:100000000C94C3030C94E4030C94E4030C94E403F5
:100010000C94E4030C94E4030C94E4030C94E403C4
:100020000C94E4030C94E4030C94E4030C94E403B4
:100030000C94E4030C94E4030C94E4030C94E403A4
:100040000C94E4030C94E4030C94E4030C94E40394
:100050000C9499070C94E4030C94E4030C94E403CB
:100060000C94250F0C94E4030C94E4030C94E40327
:100070000C940A080C94E4030C94E4030C94E30E2F
:100080000C94E4030C94E4030C94E403B015B3154E
:10009000E2161516E216E216E216DB16E216E21674
:1000A0009D16A216A716B216C7160A4F144F1C4F5C
:1000B0001E4F204F224F244F264F294F6E616E0056
:1000C000696E660000407A10F35A00A0724E18095B
:1000D0000010A5D4E80000E87648170000E40B54AF
:1000E000020000CA9A3B000000E1F505000080967E
:1000F0009800000040420F000000A08601000000B0
:10010000102700000000E803000000006400000069
:1001100000000A00000000000100000000002C7632
:10012000D888DC674F0823DFC1DFAE59E1B1B7964D
:10013000E5E3E453C63AE651997696E8E6C28426AA
:10014000EB898C9B62ED407C6FFCEFBC9C9F40F286
:10015000BAA56FA5F490055A2AF75C936B6CF96702
:100160006DC11BFCE0E40D47FEF520E6B500D0EDC7
:10017000902E0300943577050080841E080000202F
:100180004E0A000000C80C333333330F986E1283CD
:100190001141EF8D2114893BE65516CFFEE6DB18A1
:1001A000D1844B381BF77C1D901DA4BBE424203266
:1001B00084725E228100C9F124ECA1E53D274E4105
:1001C0004E494E495459494E46CDCCCC3D0AD723D1
:1001D0003C17B7D13877CC2B329595E6241FB14F19
:1001E0000A000020410000C84200401C4620BCBE5E
:1001F0004CCA1B0E5AAEC59D744572726F722C208C
:10020000696E64657465726D696E61746520626F94
:100210006F7420766563746F722025640D0A004147
:10022000540024504D544B3331342C302C312C306D
:100230002C312C302C302C302C302C302C302C30DD
:100240002C302C302C302C302C302C302C302C30CE
:100250002A32380D0A0024504D544B3330302C31A3
:100260003030302C302C302C302C302A31430D0AD9
:100270000024504D544B3235312C35373630302A2E
:1002800032430D0A0052096AD53036A538BF40A363
:100290009E81F3D7FB7CE339829B2FFF87348E430B
:1002A00044C4DEE9CB547B9432A6C2233DEE4C9588
:1002B0000B42FAC34E082EA16628D924B2765BA25F
:1002C000496D8BD12572F8F66486689816D4A45CC3
:1002D000CC5D65B6926C704850FDEDB9DA5E15469E
:1002E00057A78D9D8490D8AB008CBCD30AF7E458F7
:1002F00005B8B34506D02C1E8FCA3F0F02C1AFBD53
:100300000301138A6B3A9111414F67DCEA97F2CFF0
:10031000CEF0B4E67396AC7422E7AD3585E2F937DA
:10032000E81C75DF6E47F11A711D29C5896FB76228
:100330000EAA18BE1BFC563E4BC6D279209ADBC0D3
:10034000FE78CD5AF41FDDA8338807C731B11210EB
:10035000592780EC5F60517FA919B54A0D2DE57AC8
:100360009F93C99CEFA0E03B4DAE2AF5B0C8EBBB14
:100370003C83539961172B047EBA77D626E1691422
:100380006355210C7D637C777BF26B6FC530016711
:100390002BFED7AB76CA82C97DFA5947F0ADD4A2FD
:1003A000AF9CA472C0B7FD9326363FF7CC34A5E5C9
:1003B000F171D8311504C723C31896059A07128026
:1003C000E2EB27B27509832C1A1B6E5AA0523BD65A
:1003D000B329E32F8453D100ED20FCB15B6ACBBE7F
:1003E000394A4C58CFD0EFAAFB434D338545F9022B
:1003F0007F503C9FA851A3408F929D38F5BCB6DA40
:100400002110FFF3D2CD0C13EC5F974417C4A77EE5
:100410003D645D197360814FDC222A908846EEB8F6
:1004200014DE5E0BDBE0323A0A4906245CC2D3AC30
:10043000629195E479E7C8376D8DD54EA96C56F475
:10044000EA657AAE08BA78252E1CA6B4C6E8DD7433
:100450001F4BBD8B8A703EB5664803F60E6135575B
:10046000B986C11D9EE1F8981169D98E949B1E87AB
:10047000E9CE5528DF8CA1890DBFE6426841992D50
:100480000FB054BB1678A46AD756B7C7E8DB702004
:1004900024EECEBDC1AF0F7CF52AC6874713463088
:1004A000A8019546FDD8988069AFF7448BB15BFFF2
:1004B000FFBED75C892211906B937198FD8E4379B2
:1004C000A62108B44962251EF640B340C0515A5EC9
:1004D00026AAC7B6E95D102FD65314440281E6A1BF
:1004E000D8C8FBD3E7E6CDE121D60737C3870DD5C2
:1004F000F4ED145A4505E9E3A9F8A3EFFCD9026F1E
:10050000678A4C2A8D4239FAFF81F6718722619DF4
:100510006D0C38E5FD44EABEA4A9CFDE4B604BBBB1
:10052000F670BCBFBEC67E9B28FA27A1EA8530EFD5
:10053000D4051D880439D0D4D9E599DBE6F87CA22E
:100540001F6556ACC4442229F497FF2A43A723947D
:10055000AB39A093FCC3595B6592CC0C8F7DF4EF53
:10056000FFD15D84854F7EA86FE0E62CFE14430129
:10057000A3A111084E827E53F735F23ABDBBD2D704
:100580002A91D386EB0000891112239B322446ADB9
:10059000573665BF74488CC19D5AAFD3BE6CCAE54F
:1005A000DB7EE9F7F88110080193331A22A5562C57
:1005B00047B7753E64C99C408DDBBF52AEEDDA642F
:1005C000CBFFF976E802218B30100299132667AF32
:1005D000763444BD554AADC3BC588ED19F6EEBE70F
:1005E000FA7CC8F5D983310A2091121803A7772E17
:1005F00066B5543C45CBBD42ACD99E508FEFFB66EF
:10060000EAFDD874C904428D5316619F702004A975
:10061000153227BB364CCEC5DF5EEDD7FC6888E1CE
:10062000997AABF3BA85520C4397711E60A11428D6
:1006300005B3373A26CDDE44CFDFFD56ECE99860AE
:1006400089FBBB72AA06638F7214409D512225ABB1
:10065000343006B9174EEFC7FE5CCCD5DD6AA9E38E
:10066000B8788AF19B87730E6295501C41A3352A96
:1006700024B1163807CFFF46EEDDDC54CDEBB9626E
:10068000A8F99A708B088481951AA793B62CC2A5F5
:10069000D33EE1B7F04008C919522BDB3A644EED66
:1006A0005F766DFF7C899400859BB712A6ADD2243E
:1006B000C3BFF136E0C1184809D33B5A2AE55E6C46
:1006C0004FF77D7E6C0AA583B4188691972EE3A719
:1006D000F23CC0B5D14229CB38500AD91B666FEF26
:1006E0007E744CFD5D8BB502A499961087AFF326FE
:1006F000E2BDD034C1C3394A28D11A580BE77F6E06
:100700006EF55C7C4D0CC685D71EE597F42880A15C
:10071000913AA3B3B2444ACD5B5669DF78600CE9E5
:100720001D722FFB3E8DD604C79FF516E4A99020BD
:1007300081BBB332A2C55A4C4BD7795E68E11C68C5
:100740000DF33F7A2E0EE787F61CC495D52AA1A398
:10075000B03882B193466BCF7A5448DD59622DEBA5
:100760003C700EF91F8FF706E69DD414C5ABB1227D
:10077000A0B9923083C77B4E6AD5585C49E33D6A85
:100780002CF11E780F002092D83A11241FBECFEF13
:10079000D0E4DEBFCDBF17E0A0E0B1E0E4E0F3EFCE
:1007A00000E00BBF02C007900D92A036B107D9F749
:1007B0001AE3A0E6B7E001C01D92A83DB107E1F73A
:1007C0000E94756D0C9480790C9400000C94456423
:1007D0008091D83A80FF02C082E007C082FF02C049
:1007E00083E003C083FF08C081E0809360078091AD
:1007F00026188823F9F018C01F928F9389EF91E093
:100800009F938F930E94A77687EE95E00E94BB7618
:100810000F900F900F900F9080917307811101C07E
:10082000299A0E942A10F8CF0E946754811102C0B1
:100830000E94DA1080917307811101C02A9A0895ED
:10084000789486E797E10E949C09EAECFAE386E750
:1008500097E193838283918380830E94DF060E94C5
:100860009E0F0E94051082E09CE00E946C0B26EE19
:1008700033E042E05CE0BA018DE298E10E94BE60A4
:1008800046E757E162E07CE08DE298E10E94266253
:100890000E94BE110E94764F86E797E10E94625047
:1008A0000E94F5100C94E80310924117089580916E
:1008B0003B17813019F480E00E94790880913B1742
:1008C000823019F480E00E94950880913B178330B4
:1008D00019F480E00E94B10880913B17843019F42C
:1008E00080E00E94CC0880913B17853019F480E0AD
:1008F0000E94E60880913B17863019F480E00E9440
:10090000000980913B17873019F480E00E941A0992
:1009100080913B17883019F480E00E94340980915F
:100920003B17893019F480E00E944E0980913B17F3
:100930008A3019F480E00E94680980913B178B305F
:1009400019F480E00E94820980913B178C3019F4E1
:1009500080E00C94330A08958FEF8093A41A44E149
:1009600050E060E070E0409358175093591760933F
:100970005A1770935B1746E950E060E070E04093CF
:1009800028185093291860932A1870932B184AE05E
:1009900050E060E070E04093191850931A1860938B
:1009A0001B1870931C1890EC909342178093681753
:1009B00080E8809327181092181810923017109220
:1009C000261881E08093751780939F1A9BE090937F
:1009D0003B1780933A17089580E00895089508958D
:1009E0009FEF980F9C3010F480933B1708950C9460
:1009F000B60F0C94B00F811103C01092181808950F
:100A000081E0809318180895811103C01092301767
:100A1000089581E0809330170895811103C01092EA
:100A200075170895813011F0823011F48093751795
:100A30000895811103C0109241170895813011F07B
:100A4000823011F4809341170895811103C01092F0
:100A50009F1A0895813011F0823011F480939F1A0B
:100A60000895F894F999FECF92BD81BD60BDFA9AC0
:100A70007894F99A0895F894F999FECF92BD81BDC2
:100A8000F89A789480B50895AF92BF92CF92DF9292
:100A9000EF92FF920F931F93CF93DF93CDB7DEB703
:100AA000E0970FB6F894DEBF0FBECDBFCE01019622
:100AB0007C0100E010E05C01C8010E943B05D70109
:100AC0008D937D010F5F1F4F00311105A9F77E0146
:100AD000B1E2EB0EF11C670100E110E0C8010E94D9
:100AE0003B05F60181936F010F5F1F4F0032110527
:100AF000A9F720E830E040E050E0B501CE01419692
:100B00000E940560FE01719680E18E0F2191D70150
:100B10009D917D01291304C08E13F8CF81E001C09F
:100B200080E0E0960FB6F894DEBF0FBECDBFDF9138
:100B3000CF911F910F91FF90EF90DF90CF90BF90DA
:100B4000AF900895EF92FF920F931F93CF93DF938F
:100B5000CDB7DEB760970FB6F894DEBF0FBECDBF3E
:100B6000CE0101967C0100E010E0C8010E943B0527
:100B7000F70181937F010F5F1F4F00311105A9F726
:100B80008C818093A41A2D8130E0AAE0B0E00E940D
:100B90003273609358177093591780935A17909334
:100BA0005B172E8130E00E94327360932818709397
:100BB000291880932A1890932B182F8130E00E94D7
:100BC00032736093191870931A1880931B189093BE
:100BD0001C188885809342178985809368178A85B9
:100BE0008093271881E09B85911101C080E080935C
:100BF000181881E09C85911101C080E08093301726
:100C000081E09D85911101C080E0809326188E853A
:100C1000809375178F8580939F1A888980933B17DF
:100C200060960FB6F894DEBF0FBECDBFDF91CF91B7
:100C30001F910F91FF90EF9008950F931F93CF9303
:100C4000DF931F92CDB7DEB78C0169830E943B050D
:100C50006981861741F0C8010F90DF91CF911F91F4
:100C60000F910C9431050F90DF91CF911F910F914F
:100C70000895CF93DF93C0E0D0E060E0CE010E9402
:100C80001D062196C032D105C1F7DF91CF9108959D
:100C9000CF92DF92EF92FF920F931F93CF93DF9348
:100CA000CDB7DEB7E0970FB6F894DEBF0FBECDBF6D
:100CB0008E010F5F1F4F80E2F80111928A95E9F7CC
:100CC00081E089838A838B838091A41A8C836091CD
:100CD00058177091591780915A1790915B172AE015
:100CE000C22ED12CE12CF12CA70196010E94807319
:100CF0002D83609128187091291880912A1890915D
:100D00002B18A70196010E9480732E8360911918F9
:100D100070911A1880911B1890911C18A7019601C8
:100D20000E9480732F838091421788878091681773
:100D30008987809127188A87809118188B878091DE
:100D400030178C87809126188D87809175178E8734
:100D500080919F1A8F8780913B17888B20E830E025
:100D600040E050E0B801CE0181960E940560DE01AE
:100D70005196FE01B19680E18E0F91919D938E1355
:100D8000FCCFE12CF12CF80161918F01C7010E9489
:100D90001D06FFEFEF1AFF0A80E2E816F10499F74B
:100DA000E0960FB6F894DEBF0FBECDBFDF91CF91B6
:100DB0001F910F91FF90EF90DF90CF9008951092C8
:100DC0003A171092A31A0E944405882319F00E9432
:100DD000A20504C00E94AC040E944806109241176C
:100DE0000C9457040C94480681E0809326180C94C8
:100DF00048060E94480698E088E10FB6F894A89546
:100E0000809360000FBE90936000FFCF1092261871
:100E10000E94F90681E08093A31A08951092A31A04
:100E20000895CF92DF92EF92FF920F931F93CF938B
:100E3000DF93CDB7DEB7A0970FB6F894DEBF0FBE35
:100E4000CDBFCE0101967C0100E010E06C01C8012D
:100E50000E943B05F70181937F010F5F1F4F003216
:100E60001105A9F760E270E0C6010E94C56AA0966C
:100E70000FB6F894DEBF0FBECDBFDF91CF911F91AB
:100E80000F91FF90EF90DF90CF9008959091C80060
:100E900095FFFCCF8093CE0081E090E00895809193
:100EA000C80087FFFCCF8091CE0090E00895CF93DB
:100EB000DF931F92CDB7DEB789830E942A10898104
:100EC0009091C00095FFFCCF8093C60081E090E038
:100ED0000F90DF91CF9108958091C00087FFFCCFE4
:100EE0000E942A108091C60090E00895811103C0ED
:100EF0008091C00004C0813031F48091C800881F07
:100F00008827881F089580E008958091C00087FF9A
:100F100005C00E942A108091C60008958FEF0895A1
:100F20008091C80087FF03C08091CE0008958FEFA5
:100F300008951F920F920FB60F9211240BB60F92C5
:100F40002F933F934F935F936F937F938F939F93D1
:100F5000AF93BF93EF93FF938091C00087FF47C08B
:100F60000E942A1020912C1730912D17809128175C
:100F7000909129172817390759F420912E1730918D
:100F80002F1780912A1790912B172817390769F18D
:100F900020912E1730912F1780912C1790912D179B
:100FA00001972817390709F10E948507E0912E174C
:100FB000F0912F17808320912E1730912F17809159
:100FC0002A1790912B172817390729F48091281791
:100FD0009091291705C080912E1790912F17019697
:100FE00090932F1780932E1702C00E949007FF91B5
:100FF000EF91BF91AF919F918F917F916F915F9191
:101000004F913F912F910F900BBE0F900FBE0F90FD
:101010001F9018951F920F920FB60F9211240BB6C6
:101020000F922F933F934F935F936F937F938F9381
:101030009F93AF93BF93EF93FF938091C80087FF77
:1010400045C0209123113091241180911F1190915E
:1010500020112817390759F42091251130912611B4
:1010600080912111909122112817390769F120915F
:10107000251130912611809123119091241101970F
:101080002817390709F10E949007E0912511F09186
:1010900026118083209125113091261180912111F4
:1010A000909122112817390729F480911F119091EE
:1010B000201105C0809125119091261101969093E1
:1010C00026118093251102C00E949007FF91EF9195
:1010D000BF91AF919F918F917F916F915F914F9150
:1010E0003F912F910F900BBE0F900FBE0F901F904E
:1010F000189581110CC084E08093C50081E1809334
:10110000C4008091C0008D7F8093C000089581301D
:1011100059F484E08093CD0081E18093CC008091EC
:10112000C8008D7F8093C800089581110CC082E0B3
:101130008093C50088E08093C4008091C0008D7FBB
:101140008093C0000895813059F482E08093CD00EF
:1011500088E08093CC008091C8008D7F8093C80088
:10116000089581110CC081E08093C50083E08093D5
:10117000C4008091C0008D7F8093C00008958130AD
:1011800051F48093CD0083E08093CC008091C8001F
:101190008D7F8093C800089581110BC01092C50007
:1011A00081E88093C4008091C0008D7F8093C0004F
:1011B0000895813051F41092CD0081E88093CC00E5
:1011C0008091C8008D7F8093C800089581110BC065
:1011D0001092C50086E58093C4008091C0008D7F89
:1011E0008093C0000895813051F41092CD0086E5BF
:1011F0008093CC008091C8008D7F8093C8000895B3
:1012000081110BC01092C50080E48093C4008091CE
:10121000C0008D7F8093C0000895813051F41092FA
:10122000CD0080E48093CC008091C8008D7F8093B6
:10123000C800089581110BC01092C5008AE2809306
:10124000C4008091C0008D7F8093C00008958130DC
:1012500051F41092CD008AE28093CC008091C800B6
:101260008D7F8093C800089581110BC01092C50036
:1012700080E28093C4008091C0008D7F8093C00085
:101280000895813051F41092CD0080E28093CC001B
:101290008091C8008D7F8093C800089581110BC094
:1012A0001092C50085E18093C4008091C0008D7FBD
:1012B0008093C0000895813051F41092CD0085E1F3
:1012C0008093CC008091C8008D7F8093C8000895E2
:1012D00081110BC01092C5008FE08093C4008091F3
:1012E000C0008D7F8093C0000895813051F410922A
:1012F000CD008FE08093CC008091C8008D7F8093DB
:10130000C800089581110BC01092C5008AE0809337
:10131000C4008091C0008D7F8093C000089581300B
:1013200051F41092CD008AE08093CC008091C800E7
:101330008D7F8093C8000895CF92DF92EF92FF9245
:101340000F931F93CF93DF93CDB7DEB76C970FB694
:10135000F894DEBF0FBECDBF6C018CE1D6011D92AB
:101360008A95E9F787E2E82E81E1F82E80E096E0A1
:10137000F7019C01119221503040E1F702E917E199
:1013800080E8D8011D928A95E9F780E00E948209E1
:101390001092CD008AE08093CC00E8ECF0E08081F0
:1013A0008D7F808396E09093C20088E98093C1008E
:1013B0009093CA008093C9008EE0FE013F96DF0142
:1013C000282F1D922A95E9F79E012F5F3F4FD901E3
:1013D0001D928A95E9F783E08A8B47E557E0588F9D
:1013E0004F8B4CE657E05A8F498F9EE0D601019013
:1013F0000D929A95E1F78C8386E497E09A87898726
:101400008FE497E09C878B878EE0F901D6011E96CA
:1014100001900D928A95E1F7E8E2F7E1F182E0822E
:10142000F782E682F582E48286E297E19383828303
:10143000EFE1F1E1118300831783068315830483B1
:1014400081E198E1938382836C960FB6F894DEBFB6
:101450000FBECDBFDF91CF911F910F91FF90EF9005
:10146000DF90CF90089581110BC01092C5008AE0E3
:101470008093C4008091C00082608093C000089572
:10148000813051F41092CD008AE08093CC0080919D
:10149000C80082608093C80008950F931F93CF9374
:1014A000DF93182FC091B61AD091B71A8BA1811172
:1014B0002FC08BE290E098A38F8F1E8E1D8E1C8E06
:1014C00081E08BA38CA380917307811101C02898C0
:1014D00080917307811101C0299A209128183091B9
:1014E000291840912A1850912B18ACE2B1E00E94C3
:1014F00041736056704F8F4F9F4F20E43FE140E0B3
:1015000050E00E9480733D8B2C8B81E080936607B6
:101510000FB7F8942091191830911A1840911B18A0
:1015200050911C18ACE2B1E00E9441736056704FBC
:101530008F4F9F4F20E43FE140E050E00E948073D6
:101540003F8B2E8B0FBFE091B61AF091B71A4FB7B1
:10155000F894EE55FD4F24813581808191812817C3
:10156000390739F426813781828193812817390719
:1015700079F066817781248135812150310991E0AC
:1015800080E06217730709F090E0292F382F02C01E
:1015900021E030E04FBF232BB1F6E091B61AF09175
:1015A000B71A2FB7F894EE55FD4FA681B7811C935B
:1015B00046815781828193814817590719F48081A8
:1015C000918103C0868197810196978386832FBF7F
:1015D00081E090E0DF91CF911F910F910895E0910C
:1015E000B61AF091B71A4FB7F89423AD34AD85AD64
:1015F00096AD4FBF28173907D9F0E091B61AF09190
:10160000B71A9FB7F894A3ADB4AD21AD32ADA21710
:10161000B30719F427A930AD05C0A3ADB4AD9D0142
:101620002F5F3F4F34AF23AF8C919FBF90E0089561
:101630008FEF9FEF089587B18FEF87B910929000D9
:1016400089E18093910080E194E0909397008093EA
:10165000960080E280937100559A549A08951092F2
:1016600036171092371710923817109239171092B8
:1016700071171092721710927317109274171092BC
:101680004817109247171092800089E180938100DB
:1016900085E490E1909387008093860080E28093B8
:1016A0007C00089882B112B8EEE7F0E0808181609A
:1016B000808387E080937B008DEE80937A0008958D
:1016C0001092361710923717109238171092391758
:1016D0000E942F0B0C941B0B0F931F93CF93DF9340
:1016E000CDB7DEB72E970FB6F894DEBF0FBECDBFD5
:1016F0008C018CE195E0D801FC011D923197E9F74E
:101700001093B71A0093B61A8BE290E0D801909626
:101710009C938E935F9792961C921E929197C8010C
:101720008D9696969C938E9395979C969C938E936C
:101730009B979A969C938E939997099698969C93CB
:101740008E9397970996D8969C938E93D797DE960B
:101750009C938E93DD97DC969C938E93DB978E59AA
:101760009D4FDA969C938E93D9970996F801EE5582
:10177000FD4F9183808397838683958384838E59DD
:101780009D4F9383828389E090E0019711F1D80106
:101790009B96ED91FC919C9710829B964D915C914C
:1017A0009C9797962D913C9198974217530749F42F
:1017B00095962D913C9196979C963C932E939B9752
:1017C000E4CFF80123A534A52F5F3F4F34A723A70B
:1017D000DCCF0E94600B8EE0FE013196DF01282FE6
:1017E0001D922A95E9F793E09C832DE43AE03A872D
:1017F00029872FEE3AE03C872B87D80101900D9284
:101800008A95E1F72E960FB6F894DEBF0FBECDBFD6
:10181000DF91CF911F910F910895CF93DF93FC013A
:10182000808D8111BEC0828D811190C0DF01AE55C7
:10183000BD4F14964D915C91159716962D913C9144
:1018400017974217530749F426893789232B29F420
:101850001092660713A214A251C0938D911101C07A
:10186000148E91E0938F248935892115310579F5FE
:1018700014964D915C91159716962D913C91179762
:101880004217530741F414A22689378921503109A0
:10189000378B268B20C01496CD91DC91159712962C
:1018A0002D913C911397C217D30721F42D913C91B0
:1018B000119707C01496CD91DC9115979E012F5F6B
:1018C0003F4F15963C932E931497988105C0215055
:1018D0003109358B248B9EE7918F918D9B3181F55A
:1018E00014964D915C91159716962D913C911797F2
:1018F0004217530749F41092660713A29091730799
:1019000091116FC029986DC01496CD91DC911597F7
:1019100012968D919C911397C817D90721F48D9138
:101920009C91119706C01496CD91DC911597CE012C
:10193000019615969C938E9314978881818F04C08D
:101940009E57923008F4138E81E0828F838D278D0D
:1019500030A1882379F0848D853060F0148E2B328D
:10196000310519F08BE290E002C080E390E090A393
:10197000878F15C0828D918D982321F0948D9F5F64
:10198000948F0BC0148E2B32310519F02BE230E00E
:1019900002C020E330E030A3278F880F828F80E4DD
:1019A000808F278D30A1858D968D820F931FAC017E
:1019B0005170568F458F208D2150208F9927803868
:1019C000910530F02FEF30E0B901681B790BCB01A6
:1019D000FC01E85FFE4F80814F3F510511F008F098
:1019E0008095DF91CF910895EF92FF920F931F930F
:1019F000CF93DF93FC01262F8091A31A8823E9F06F
:101A000040916207509163074F5F5F4F50936307A8
:101A1000409362078091640786171CF46093640703
:101A20000CC04036510548F01092630710926207CF
:101A300018161CF48150809364078F01015F1A4FC0
:101A4000D801ED90FC9011971297ED92FC92A1A510
:101A5000B2A587A190A5A817B90719F485A196A1E9
:101A600004C0A1A5B2A5CD01019692A781A79C9122
:101A70009202C001112466E070E00E946C73E801DC
:101A800079836883DF01AD5EBA4F4C9111963C912A
:101A90001197CF018F5E9A4FEC01488339836E0D09
:101AA0007F1D842F932F97FD019695958795860F1F
:101AB000971F8D939C93DF01AB5EBA4F41E050E0DE
:101AC0001816190614F440E050E08D919C9111977E
:101AD000880F991F842B952B11969C938E93C3A5E9
:101AE000D4A5288323A534A587A190A52817390755
:101AF00019F485A196A103C083A594A5019694A786
:101B000083A78D919C9111979C01369527953695C9
:101B100027958227932783709927EF01C95EDA4FB3
:101B2000039769F4888199818830910510F40196B2
:101B300001C001979983888312A211A205C081A1D7
:101B400092A1019692A381A3888199810196803107
:101B5000910518F49983888322C18F7099279983FE
:101B60008883EF01C75EDA4F8881880F88839C9154
:101B700097702BEF290F233010F0933011F4816010
:101B800088838881982F969589278095817096857E
:101B9000990F892B86878E37C1F523AD34AD87A980
:101BA00090AD2817390739F425AD36AD81AD92AD2A
:101BB0002817390731F125AD36AD83AD94AD0197C6
:101BC00028173907F1F0A5ADB6AD8EE78C9325AD9A
:101BD00036AD81AD92AD2817390719F487A990ADBC
:101BE00003C085AD96AD019696AF85AF81E0818B40
:101BF0009389911103C0128A838BA2C0828B81E0EA
:101C00009FC0118A128A138A9AC08F778F3711F476
:101C1000118A0FC0928980917307992321F0811155
:101C200005C0289A03C0811101C0289881898111BB
:101C300003C0128A138AB3C08685982F9F739E3380
:101C400009F4ADC080FF03C080898068808B9785D0
:101C50009F5F97878089983008F477C092E8980F43
:101C6000923010F08B3199F523AD34AD87A990AD4A
:101C70002817390739F425AD36AD81AD92AD281757
:101C80003907E1F025AD36AD83AD94AD0197281746
:101C90003907A1F0A5ADB6AD8BE18C9325AD36AD7E
:101CA00081AD92AD2817390719F487A990AD03C00B
:101CB00085AD96AD019696AF85AF09C0118A128A9F
:101CC000138A80917307811104C0289803C081E0B2
:101CD00001C080E043AD54AD27A930AD4217530792
:101CE00039F445AD56AD21AD32AD42175307F1F091
:101CF00045AD56AD23AD34AD2150310942175307E0
:101D0000A9F09089A5ADB6AD9C9345AD56AD21AD7A
:101D100032AD4217530719F427A930AD04C025ADE1
:101D200036AD2F5F3F4F36AF25AF0AC0118A128AFA
:101D3000138A80917307811102C0289801C080E046
:101D4000108A1786882321F02AC08695808B27C0A9
:101D5000DF01A65EBA4F8D919C911197816011961B
:101D60009C938E9323AD34AD87A990AD2817390786
:101D700039F425AD36AD81AD92AD2817390741F064
:101D800025AD36AD83AD94AD01972817390739F4E9
:101D900085AD96AD94AF83AF11961C921E9281A132
:101DA00092A18130914040F012A211A2128A80913A
:101DB0007307811101C02898DF91CF911F910F9176
:101DC000FF90EF9008951F920F920FB60F9211247B
:101DD0000BB60F922F933F934F935F936F937F9325
:101DE0008F939F93AF93BF93EF93FF938091660779
:101DF000882379F08091B61A9091B71A0E940D0C41
:101E000088B980917307811101C0299A5D9A5C9805
:101E100009C080917307811101C029988FE788B9A3
:101E20005D985C9AFF91EF91BF91AF919F918F91D7
:101E30007F916F915F914F913F912F910F900BBECA
:101E40000F900FBE0F901F9018951F920F920FB614
:101E50000F9211240BB60F922F933F934F935F93E2
:101E60006F937F938F939F93AF93BF93EF93FF9362
:101E700080E286BB80916607811115C06091790070
:101E800060588091B61A9091B71A0E94F40C809114
:101E900061078F5F803618F48093610704C0109249
:101EA00061070E945B120E945A1080913617909130
:101EB0003717A0913817B09139170196A11DB11DA0
:101EC0008093361790933717A0933817B09339172C
:101ED00080914717909148170196909348178093E7
:101EE0004717803C9241B8F080917117909172171A
:101EF000A0917317B09174170196A11DB11D809325
:101F0000711790937217A0937317B0937417109270
:101F1000481710924717FF91EF91BF91AF919F9192
:101F20008F917F916F915F914F913F912F910F9082
:101F30000BBE0F900FBE0F901F9018958AB1806C4A
:101F40008AB983EA8093B00081E08093B1008091E8
:101F500027188093B300809168178093B400089588
:101F60008093271880958093B30008958093681715
:101F70008093B40008952FB7F8946091361770914C
:101F8000371780913817909139172FBF08958F9286
:101F90009F92AF92BF92CF92DF92EF92FF92CF9338
:101FA000DF9300D000D0CDB7DEB79B01AC016983D1
:101FB0003A834B835C830E94BB0F6B017C01A5E0DD
:101FC000B0E029813A814B815C810E9441734B01D1
:101FD0005C010E94BB0FDC01CB018C199D09AE098D
:101FE000BF0988159905AA05BB0598F30F900F90B6
:101FF0000F900F90DF91CF91FF90EF90DF90CF90F7
:10200000BF90AF909F908F90089588EC90E0A0E0F3
:10201000B0E080936F0790937007A0937107B0931F
:10202000720784B18F6184B985B1807E85B983ECF4
:1020300084BD81E085BD8091421787BD089581E010
:102040008093730708951092730708958093421741
:1020500087BD089580917307811111C02C9A0E9449
:10206000BB0FDC01CB0188539F4FAF4FBF4F809315
:10207000670790936807A0936907B0936A0708956C
:1020800080917307811101C02C9808952C9A0E94A9
:10209000BB0FDC01CB0188539F4FAF4FBF4F8093E5
:1020A000670790936807A0936907B0936A0708953C
:1020B0002C9808950F931F9380916B0790916C0754
:1020C000A0916D07B0916E0740916F075091700716
:1020D000609171077091720784179507A607B7077B
:1020E000D4F00E94BB0F0091670710916807209100
:1020F000690730916A07061717072807390714F48C
:102100000E94401010926B0710926C0710926D079E
:1021100010926E070BC00196A11DB11D80936B0735
:1021200090936C07A0936D07B0936E071F910F916A
:102130000895CF9381E0809373072A980E945810E6
:102140002998289868EC70E080E090E00E94C70F22
:10215000C2E02A9A62E370E080E090E00E94C70F3C
:102160002A980E94461062E370E080E090E00E94AE
:10217000C70F0E945810289A62E370E080E090E058
:102180000E94C70F2898299A62E370E080E090E0EF
:102190000E94C70F299862E370E080E090E00E94FF
:1021A000C70FC13011F0C1E0D4CF2A9A1092730743
:1021B000CF9108950E942A1080917307811101C068
:1021C0002A9864EF71E080E090E00E94C70F0E94BF
:1021D000401080917307811101C02A9A64EF71E069
:1021E00080E090E00E94C70FE5CF81B1866081B9A1
:1021F0000E94DB4F811103C081B1886181B90895CC
:1022000082B186958170089582B182FB882780F91A
:1022100008950E94DB4F811105C082B183FB88279E
:1022200080F9089580E008950E94DB4F811104C079
:1022300082B182958170089580E00895119A089581
:10224000129A08950E94DB4F811101C0139A0895DC
:102250000E94DB4F811101C0149A089511980895CE
:10226000129808950E94DB4F811101C0139A0895BE
:102270000E94DB4F811101C0149A08950E94DB4F28
:10228000811107C00E94001181110C942E110C9431
:102290001E1108950E94DB4F811107C00E94041196
:1022A00081110C9430110C94201108950E94091191
:1022B00081110C9432110C9422110E94141181117D
:1022C0000C9438110C9428118F929F92AF92BF9268
:1022D000CF92DF92EF92FF920F931F939B01AC017D
:1022E0008FB7F894C0903617D0903717E090381712
:1022F000F09039178FBFA5E0B0E00E9441732FB76F
:10230000F8948090361790903717A0903817B090B7
:1023100039172FBF950184010C191D092E093F099A
:10232000061717072807390750F31F910F91FF90E1
:10233000EF90DF90CF90BF90AF909F908F900895D7
:10234000CF93C2E080917307811101C02A986AEF90
:1023500070E080E090E00E94641180917307811129
:1023600001C02A9A64E170E080E090E00E9464116C
:10237000C13011F0C1E0E6CFCF91089584B1806AF9
:1023800084B9269881E58CBD0E9A0F98179A089506
:102390000E94A0110E94C25481110C94DA10089579
:1023A000CF938130D1F4C4E080917307811101C0D3
:1023B0002A9861E470E080E090E00E9464118091CE
:1023C0007307811101C02A9A6EE170E080E090E00D
:1023D0000E946411C15041F705C0811103C0CF9123
:1023E0000C94A011CF91089581E00E94D0110C941B
:1023F0002557809100018695817091E08927089585
:1024000081E090910001911180E00895809178071A
:1024100008950E94F911882389F041E062EB76E08B
:1024200088EB9AE10E940F35811104C081E080930E
:10243000780702C01092780780917807089540E0ED
:1024400062EB76E080E090E00E940F35811104C0DD
:102450001092780781E0089580E008950E940912A3
:1024600081110C94F41108950E941F1281110C9493
:10247000C811089580917707882321F0109277077B
:102480000E942E1280917607882321F01092760701
:102490000E94341280917507882321F010927507ED
:1024A0000E94F41180917407882321F01092740720
:1024B0000C94C8110895CF93809179078F5F809312
:1024C00079070E94F71680E00E94CD1480930001E6
:1024D0008091790762E30E944C73911116C01092AB
:1024E0007907C0917807C11107C00E94F9118823AC
:1024F00019F081E0809377070E94F911811105C0DE
:10250000CC2319F081E080937607CF9108950F9343
:102510001F93CF93DF93CDB7DEB760970FB6F894D4
:10252000DEBF0FBECDBF2FB7F89480917117909189
:102530007217A0917317B09174172FBF8D879E8764
:10254000AF87B88BBE016F5F7F4FCE010D960E94A3
:10255000106B4B81552747FD5095652F752F8BE0EC
:10256000440F551F661F771F8A95D1F78C819927D5
:1025700087FD9095A92FB92FDC0199278827482B33
:10258000592B6A2B7B2B8A81992787FD9095A92F40
:10259000B92F35E0880F991FAA1FBB1F3A95D1F7B5
:1025A000482B592B6A2B7B2B8981992787FD909586
:1025B000A92FB92FB695A79597958795482B592B95
:1025C0006A2B7B2B8F819885805D9740AA2797FD8A
:1025D000A095BA2FF9E1880F991FAA1FBB1FFA9582
:1025E000D1F7482B592B6A2B7B2B8E818F5F992734
:1025F00087FD9095A92FB92F15E1880F991FAA1F64
:10260000BB1F1A95D1F78A019B01082B192B2A2B86
:102610003B2BC901B80160960FB6F894DEBF0FBE20
:10262000CDBFDF91CF911F910F9108958EBD0DB455
:1026300007FEFDCF8EB50895169A8FEF0C941613F2
:102640000F931F93CF93DF93EC018B0184E1809371
:102650007B078FEF0E9416138F3F29F480917B0731
:102660008111F7CF1EC08E3FE1F48FEF8EBD0DB408
:1026700007FEFDCF9EB598838EBD0DB407FEFDCF3E
:1026800022969EB5FE01319790830250110971F791
:102690008FEF0E9416138FEF0E94161381E090E0D7
:1026A00002C080E090E0DF91CF911F910F910895DB
:1026B00082E380937A078FEF0E941613282F8F3FB3
:1026C00021F080917A078111F6CF81E090E02F3FD1
:1026D00011F080E090E00895CF93DF9300D0CDB764
:1026E000DEB716988FEF0E9416130E9458130097BA
:1026F00039F489839A830E941C1389819A8102C0CC
:1027000081E090E00F900F90DF91CF910895FF92BC
:102710000F931F93CF93DF93C82FD42F152F062F1E
:10272000F72E87FF09C040E050E0BA0187E30E941E
:1027300087138230A0F5CF77CC3099F48C2F80644A
:102740000E9416138F2D0E941613802F0E941613BD
:10275000812F0E9416138D2F0E941613CC2369F02F
:1027600008C00E941C130E946C13892B39F78FEF4D
:1027700016C0C83021F081E003C085E901C087E8B8
:102780000E941613CC3019F48FEF0E941613CAE082
:102790008FEF0E94161387FF02C0C150C9F7DF9167
:1027A000CF911F910F91FF9008951F93CF93DF93C7
:1027B000EC01162F0E945813009759F1812F0E94A7
:1027C00016131D3F21F1CE019E5F28812EBD0DB451
:1027D00007FEFDCF2296FE01319720812EBD0DB45C
:1027E00007FEFDCFC817D90781F78FEF0E94161398
:1027F0008FEF0E9416138FEF0E9416138F7131E036
:1028000020E0853009F030E0832F922F02C081E074
:1028100090E0DF91CF911F910895DF92EF92FF92A8
:102820000F931F93CF93DF9300D000D0CDB7DEB7C7
:102830008111A6C01CBC8091010181FD9EC084B1A4
:10284000806A84B9269881E58CBD82E58CBD1AE04A
:102850008FEF0E9416131150D9F740E050E0BA01F3
:1028600080E00E948713813009F075C084E6809370
:102870007B074AEA51E060E070E088E00E9487133D
:10288000813009F040C08E010F5F1F4F780184E056
:10289000D82ED00E8FEF0E941613F70181937F017F
:1028A000DE12F8CF8B81813009F055C08C818A3AD5
:1028B00009F051C080917B07811106C080917B0790
:1028C000882309F448C00AC040E050E060E070E4AA
:1028D00089EA0E9487138111EDCFF0CF40E050E0EC
:1028E000BA018AE30E948713811135C08FEF0E94DD
:1028F0001613F80181938F01DE12F8CF898186FDCE
:102900002CC014E02BC040E050E0BA0189EA0E94DC
:102910008713823018F011E001E002C012E009EAEA
:1029200080917B07811105C080917B07882399F0F6
:1029300009C040E050E0BA01802F0E948713811146
:10294000EFCFF2CF40E052E060E070E080E10E9423
:102950008713882319F010E001C01CE010937C0756
:102960000E941C13112341F0809101018E7F8093FE
:10297000010180E58CBD01C01CBC8091010101C03A
:1029800081E00F900F900F900F90DF91CF911F91EA
:102990000F91FF90EF90DF900895811103C0809117
:1029A0000101089581E00895EF92FF920F931F9324
:1029B000CF937B01BA01A901811138C0011511051E
:1029C000A9F18091010180FD33C080917C0783FDD6
:1029D00007C089E0440F551F661F771F8A95D1F7FE
:1029E0000230110510F4C1E101C0C2E18C2F0E9438
:1029F0008713811114C060E072E0C7010E942013A8
:102A0000892B29F08EEFF81A01501109A1F7C23174
:102A100031F440E050E0BA018CE00E9487130E943C
:102A20001C1381E0012B29F480E003C084E001C085
:102A300083E0CF911F910F91FF90EF900895CF9277
:102A4000DF92EF92FF920F931F93CF93DF93EB01EF
:102A500069017A01811156C00115110509F452C0AE
:102A60008091010180FD50C08091010182FD4EC026
:102A700080917C0783FD07C099E0CC0CDD1CEE1C27
:102A8000FF1C9A95D1F70130110599F4B701A60101
:102A900088E10E94871381112EC06EEFCE010E9443
:102AA000D51331E020E0892B09F030E0032F122FFD
:102AB00022C0867031F0A80160E070E087E90E94D2
:102AC0008713B701A60189E10E948713811113C002
:102AD0006CEFCE010E94D513892B21F0DE5F0150EF
:102AE0001109B1F76DEF80E090E00E94D513892BBA
:102AF00011F401E010E00E941C1381E0012B39F475
:102B000080E005C084E003C083E001C082E0DF9183
:102B1000CF911F910F91FF90EF90DF90CF9008958C
:102B2000EF92FF920F931F93CF93DF93CDB7DEB752
:102B300060970FB6F894DEBF0FBECDBF811147C1BD
:102B40008091010180FD45C17A01862F90E08F3090
:102B5000910508F037C1FC01EA5BFF4F0C9401744A
:102B60000E946C1324C140E050E0BA0189E00E9449
:102B70008713882311F011E026C160E170E0CE01D7
:102B800001960E942013892BB1F399819295969515
:102B900096959370888549852A859130E1F48F73E5
:102BA00090E0A0E0B0E0DC01992788270196A11D04
:102BB000B11D50E0542F4427BA01620F711D860FDA
:102BC000971FA11DB11DFAE0880F991FAA1FBB1FF7
:102BD000FA95D1F7ABC04295469546954370F4E01F
:102BE0008F9FC0011124840F911D01964F81437066
:102BF00050E0542F4427550F550F840F951FA0E028
:102C0000B0E03E81432F4F703B85331F3327331F86
:102C1000340F2370220F230F275004C0880F991FF1
:102C2000AA1FBB1F2A95D2F781C010917C0740E0F4
:102C300050E0BA0112FF2BC08DE80E94871381116A
:102C40009ACF8FEF0E94161360E170E0CE010196DB
:102C50000E942013892B09F48ECF10E38FEF0E947E
:102C600016131150D9F72B8522952F7080E190E033
:102C7000A0E0B0E004C0880F991FAA1FBB1F2A95CF
:102C8000D2F7F70180839183A283B3839CC089E04C
:102C90000E94871381116FCF60E170E0CE01019631
:102CA0000E942013892B09F466CF8B852C8511FF98
:102CB0001FC0221F2227221F022F10E00F5F1F4F6D
:102CC0008F73080F111D080F111D8E858295869533
:102CD00086958370815002C0000F111F8A95E2F71C
:102CE00020E030E0F701008311832283338323C087
:102CF000922F937022952695277030E0F8E09F9FE1
:102D0000200D311D11242F5F3F4F8C7790E095955A
:102D10008795959587950196289FA001299F500D2D
:102D2000389F500D1124CA01A0E0B0E0F701808364
:102D30009183A283B38310E046C080917C07FA019F
:102D40008083F9CF40E050E0BA0189E004C040E060
:102D500050E0BA018AE00E94871381110CCF60E134
:102D600070E022C040E050E0BA018AE30E9487137D
:102D7000811101CF87010C5F1F4F8FEF0E94161347
:102D8000F70181937F01E017F107B9F7D4CF40E055
:102D900050E0BA018DE80E9487138111ECCE8FEFCD
:102DA0000E94161360E470E0C7010E94201311E036
:102DB000892B49F0C0CF1CBC8091010181608093B8
:102DC0000101B9CF14E00E941C13812F03C084E0DD
:102DD00001C083E060960FB6F894DEBF0FBECDBF92
:102DE000DF91CF911F910F91FF90EF900895809107
:102DF0007B07882319F0815080937B0780917A07A5
:102E0000882319F0815080937A0790910101892FCE
:102E10008B7F079B03C0892F897F01C083608093CC
:102E200001010895FC016381862F90E0A0E0B0E0ED
:102E3000BA2FA92F982F88272281822BBA2FA92F4A
:102E4000982F88272181822BBA2FA92F982F882786
:102E50002081BC01CD01622B08950F93FC012781D5
:102E600030E040E050E060E070E080E090E008E0BA
:102E70000E940A74A6812A2B0E940A74A5812A2B1B
:102E80000E940A74A4812A2B0E940A74A3812A2B0F
:102E90000E940A74A2812A2B0E940A74A1812A2B03
:102EA0000E940A74E0812E2B0F910895FC0140834B
:102EB00051836283738308950F931F93CF93DF939E
:102EC000FC01D22FC32FB42FA52FCB010083980173
:102ED0004D2F5C2F6B2F7A2F08E00E9425742183E1
:102EE0000E94257422830E94257423830E942574E6
:102EF00024830E94257425830E94257426830E94C2
:102F000025742783DF91CF911F910F910895480F6A
:102F1000591FFC016193CF01E417F507D1F708951C
:102F2000DC01FB012D91819130E0B901681B710931
:102F3000CB014150510911F00097A1F308950F936F
:102F40001F93FC019A01AB0122503109410951093B
:102F50008789908DA18DB28D0297A109B10928179B
:102F600039074A075B0768F4A185B2850E9441735F
:102F700003A514A525A536A5600F711F821F931FF9
:102F800003C060E070E0CB011F910F910895FC0138
:102F90009C01255F3F4F80E0982F90FB979597F914
:102FA0008191890FE217F307B9F70895CF93DF9363
:102FB000FC01418150E04F5F5F4F65E0440F551FBA
:102FC0006A95E1F780E090E060E070E062307105C2
:102FD000A1F0DC01A170BB2780FF02C0A0E0B0E837
:102FE000EF01C60FD71F288196958795EC01C20F78
:102FF000D11DCE018A0F9B1F02C063E070E06F5F9E
:103000007F4F6417750710F3DF91CF910895CF9329
:10301000DF93DC01ED91FC9111973097D1F09F0186
:103020002F5F3F4FE90121978881803278F08A3302
:10303000B9F7908180ED890F8A3058F43296E21703
:10304000F30739F4903329F42D933C9380E090E01A
:1030500002C08FEF9FEFDF91CF9108950F931F93E1
:10306000CF93DF93EC018B01892BF1F0E881F9819B
:103070003097D1F080818823B9F02A813B81858106
:1030800096812817390781F481810E94CD1480FD33
:103090000BC02881398180E0F80131832083DF91E2
:1030A000CF911F910F91089589E020E030E0F4CF97
:1030B0000F931F93CF93DF93EA01890141E653E019
:1030C0000E948E4E8F3F910541F038F0023011057D
:1030D00058F09883898382E008C0009729F0012B7B
:1030E00019F0888381E001C080E0DF91CF911F91CA
:1030F0000F9108952F923F924F925F926F927F921D
:103100008F929F92AF92BF92CF92DF92EF92FF92F7
:103110000F931F93CF93DF93DC018D909C901197B9
:10312000FB01128E9E960D911D912D913C91D19790
:10313000012B022B032B09F4A1C1EB018C01D4015B
:103140008C91843009F09AC01D96ED90FC901E97EA
:10315000A12CB12CB0E4CB2ED12C00E010E080E00B
:1031600090E088248A94912CD70193962C9130E09A
:10317000A216B30608F044C0B0E6CB16B2E0DB06F8
:1031800008F043C096012F713327232B19F4E2E096
:10319000CE0ED11CF701EC0DFD1D4180512C542C9D
:1031A00044242081422AF2E0CF0ED11C2FEFA21A34
:1031B000B20A009729F49201385D21153840F0F0E9
:1031C000A801465E5F4F4C0F5D1F612C712CA0E083
:1031D000B0E0DC0199278827BC01CD01642975295D
:1031E000862997299401201B310B0E94581890E0E2
:1031F000009759F0080F191F412C512CC201B4CF70
:10320000892B19F40115110521F48FE38A8F01E050
:1032100010E0FE01E00FF11F128E1D86F701848180
:103220008C8784FD05C0C701C8960E942D1708C071
:1032300020E030E040E050E060E070E080E090E0CE
:10324000288339834A835B836C837D838E839F834A
:10325000D7011D968C911D9790E0982F88271C967A
:103260002C911C97822B9B878A871F968C911F9786
:1032700090E0982F88271E962C91FDC0F801E05C05
:10328000FF4F80819181A281B3818F3F9F4FAF4FCC
:10329000BF4F09F44AC0A12CB12CC12CD12CE12C78
:1032A000F12C66246A94712CD4011B96ED91FC914B
:1032B0001C97EA0DFB1D80819181009771F1C1146B
:1032C000D10429F49C01385D21153840F8F0A7019C
:1032D000465E5F4F4C0F5D1FA0E0B0E01601412C31
:1032E000512C210133242224BC01CD0162297329F0
:1032F0008429952993012E193F090E94581890E0BE
:10330000009749F0E80EF91E80E090E022E0A20E5E
:10331000B11C6C01C9CFE12CF12CCD2811F0E12CAE
:10332000F12CFE01EE0DFF1D128E20E030E080E05A
:1033300090E06EE2AC014F5F5F4FD801D296ED9105
:10334000FC91D397E80FF91F808190E080329105BE
:10335000B9F08530910511F485EE90E049305105C2
:1033600049F42C30310530F4FE01E20FF31F65877C
:103370002F5F3F4FFE01E20FF31F85872F5F3F4F07
:10338000CA014B305105B1F6FE01E20FF31F15865D
:103390008A8D811142C0232B31F0BE01665E7F4FC2
:1033A000E0E0F0E010C08FE38A8FE1E0F0E029C0B8
:1033B00090E09C01215431092A31310558F0DB019C
:1033C0008D93BD013196CB010D97DC018C9181115C
:1033D000EFCF17C0D801D2962D913C91D397D90148
:1033E0001C962C9130E0E930F10518F448E050E0EB
:1033F00002C040E150E024233523232B01F38096C3
:10340000DECFEC0FFD1F128ED801D296ED91FC910C
:10341000D3978485811101C01D86D801D296ED9184
:10342000FC91D39783858C87D2968D919C91D3976D
:103430004C960E9412174B015C0168839982AA8204
:10344000BB821C821D821E821F82D801D296ED9102
:10345000FC91D397878990E0982F88272689822B23
:103460009B878A87D296ED91FC91D397818D90E0CE
:10347000982F8827208D822B99878887DF91CF917D
:103480001F910F91FF90EF90DF90CF90BF90AF9082
:103490009F908F907F906F905F904F903F902F9074
:1034A00008950F931F93CF93DF93EC01E881F98187
:1034B0008F010F5F1F4F6081862F90E0009731F0E2
:1034C00061E673E00E94C14E009731F019830883D2
:1034D000BC0180E090E003C06FEF7FEFCB01DF9194
:1034E000CF911F910F9108950F931F93CF93DF9367
:1034F0008C01C0E0D0E0F801619171918F016115FC
:10350000710529F180E090E00E94D64EAE01417035
:103510005527C0FF02C040E050E8D695C7959B01F3
:1035200033272C0F3D1F240F351FA901417055274C
:1035300020FF02C040E050E836952795C72FDD27D1
:10354000B9016C0F7D1FEB01C40FD51FD4CFCE0185
:10355000DF91CF911F910F910895FB01480F591FE3
:103560002191DC012D93CD01A417B507C9F708956A
:10357000FB01438D50E0542F4427928D492B60E08E
:1035800070E0833079F4858990E0982F882724892A
:10359000822BA0E0B0E0DC0199278827482B592B2B
:1035A0006A2B7B2BCB01BA010895FB01228F338F4D
:1035B000DC018C91833029F4CA01AA27BB27848BB4
:1035C000958B08950F931F93CF93DF938C01EB019D
:1035D000DC018D919C91C4960E9412176E837F83AB
:1035E00088879987F80180819181C8960E942D175C
:1035F0002A873B874C875D876E877F87888B998B6F
:10360000D801ED91FC9181A182708D831E8A1F8A61
:10361000188E198EDF91CF911F910F9108958F927F
:103620009F92AF92BF92EF92FF920F931F93CF930F
:10363000DF93FC0123812223C1F1EC017C01F7E33C
:10364000EF0EF11C2BA93CA94DA95EA901E010E0E9
:10365000B70189810E941F15811129C01B828BA986
:103660009CA9ADA9BEA90B8D1C8D2D8D3E8D8BA067
:103670009CA0ADA0BEA0AC01BD01481959096A09C2
:103680007B09401751076207730778F46A8162303B
:1036900061F4A9019801280F391F4A1F5B1F01E03F
:1036A00010E0B70189810E941F1580E001C081E010
:1036B000DF91CF911F910F91FF90EF90BF90AF904E
:1036C0009F908F9008958F929F92AF92BF92FF929A
:1036D0000F931F93CF93DF93EC014A015B018BA9FA
:1036E0009CA9ADA9BEA9481759076A077B07E9F04D
:1036F000CE010E940F1BF82E811118C001E010E0CE
:10370000A5019401BE01695C7F4F89810E94D41498
:10371000882331F0FF24F39488248A94982C540150
:103720008BAA9CAAADAABEAA01C0F12C8F2DDF9155
:10373000CF911F910F91FF90BF90AF909F908F906E
:1037400008954F925F926F927F928F929F92AF9265
:10375000BF92CF92DF92EF92FF920F931F93CF937E
:10376000DF936C0148015901DB01CA010297A109ED
:10377000B1098C019D014CE0369527951795079569
:103780004A95D1F7F60147A550A961A972A9400F42
:10379000511F621F731F8C019D01E3E03695279531
:1037A00017950795EA95D1F7E801D17087709927A9
:1037B00011E001C0110F8A95EAF701E02A013B01EF
:1037C000FFEF4F1A5F0A6F0A7F0AC6010E94631B50
:1037D000811125C0F601EC0FFD1F97A9492F412348
:1037E00021E030E011F420E030E0E216F306C9F009
:1037F000912797ABF6010383F1E08F1A9108A10896
:10380000B10881F0110F31F7219611E0C11592E056
:10381000D90701F7C0E0D0E0B301A201CFCF81E02A
:1038200001C082E0DF91CF911F910F91FF90EF9047
:10383000DF90CF90BF90AF909F908F907F906F90D0
:103840005F904F9008952F923F924F925F926F92A8
:103850007F928F929F92AF92BF92CF92DF92EF9220
:10386000FF920F931F93CF93DF9300D000D01F924E
:10387000CDB7DEB7FC016A017B01208131813C8339
:103880002B83423051056105710508F464C1AB8199
:10389000BC8157964D915D916D917C915A97C4165C
:1038A000D506E606F70608F056C18C91823009F479
:1038B0005CC018F4813041F04EC1833009F47EC001
:1038C000843009F4A5C047C18601169507950C0DF3
:1038D0001D1DC801892F99278695EB81FC8143A185
:1038E00054A165A176A1480F591F611D711DCF011B
:1038F0000E94631B882321F06FEF7FEFCB0134C15F
:103900005801FFEFAF1ABF0A1170EB81FC81E00F85
:10391000F11F17A9C501892F99278695AB81BC8115
:1039200093964D915D916D917C919697480F591F9B
:10393000611D711DCD010E94631B8111DDCFB1E0BE
:10394000BB22EB81FC81EA0DFB1D87A9612F70E092
:10395000782BC0FE06C024E0769567952A95E1F79E
:1039600001C07F7080E090E0FFC077276F2D5E2D53
:103970004D2DEB81FC8183A194A1A5A1B6A1480F97
:10398000591F6A1F7B1FCF010E94631B8111B4CF97
:10399000CC0CDD1CE894C0F8F1E0DF22EB81FC8167
:1039A000EC0DFD1D90AD692F70E0762F6627EB8141
:1039B000FC81EC0DFD1D87A9682BD4CFEB81FC8128
:1039C00083A194A1A5A1B6A1B701A60117E07695A0
:1039D0006795579547951A95D1F7480F591F6A1F54
:1039E0007B1FCF010E94631B811186CFCC0CDD1C95
:1039F000CC0CDD1CFCEFCF22F1E0DF22C601C79624
:103A00002B813C81820F931F0E9412179F70ACC0C4
:103A10003284438454846584768407851089B1890F
:103A2000BD83232D342D452D562D672D702F812FCD
:103A30009B2FA0E025800E94687441F04681578149
:103A400060857185452B462B472B11F4211083C0CF
:103A5000468157816085718546015701841A950A10
:103A6000A60AB70AAB81BC8119960D90BC91A02D16
:103A7000BA83A983B2E02B1230C0232D342D452DFB
:103A8000562D672D702F812F9D81AFEF0E944A74B4
:103A900009E00E942574B22FA32FE42F152F8981EE
:103AA0009A819C0140E050E06B2F7A2F8E2F912F4E
:103AB0000E948073281539054A055B0508F44BC040
:103AC00082169306A406B50609F44AC0C701B601DA
:103AD0006F5F7F4F8F4F9F4F47C093E0291209C000
:103AE00082899389A489B58988169906AA06BB0696
:103AF00068F386899789A08DB18D892B8A2B8B2BB2
:103B000079F5EB81FC8183A194A1A5A1B6A1B701B0
:103B1000A60127E076956795579547952A95D1F7A1
:103B2000480F591F6A1F7B1FCF010E94631B811121
:103B3000E3CECC0CDD1CCC0CDD1CFCEFCF22F1E085
:103B4000DF22C601C7962B813C81820F931F0E9402
:103B500012179F7709C061E070E080E090E004C038
:103B60006FEF7FEF8FEF9FE70F900F900F900F9009
:103B70000F90DF91CF911F910F91FF90EF90DF9009
:103B8000CF90BF90AF909F908F907F906F905F90FD
:103B90004F903F902F9008954F925F926F927F9237
:103BA0008F929F92AF92BF92CF92DF92EF92FF924D
:103BB0000F931F93CF93DF93EC016A017B01088180
:103BC0001981F8018081843029F080E090E0A0E242
:103BD000B0E004C080E090E0A0E0B0E1C816D906F3
:103BE000EA06FB0610F082E0AAC0D701C6018F7179
:103BF0009927AA27BB27892B8A2B8B2BA1F7CEA22B
:103C0000DFA2E8A6F9A68E809F80A884B9848114DB
:103C10009104A104B10469F5F80180818330E8F4CE
:103C2000F80187819085A0E0B0E0B701A601E5E04A
:103C30007695679557954795EA95D1F748175907AF
:103C40006A077B0780F6F80187A190A5A1A5B2A518
:103C50008EA79FA7A8ABB9AB48C0F80187A190A5D4
:103C6000A1A5B2A51D820097A105B105C9F24C011D
:103C70005D01F80141845284612C712C39E0440CBF
:103C8000551C661C771C3A95D1F7B501A401C414E4
:103C9000D504E604F70410F1CE010E94231C4B0169
:103CA0005C016F3F7F4F8F4F9F4F09F447C082E009
:103CB00088169104A104B10408F495CFF80187890E
:103CC000908DA18DB28D88169906AA06BB0608F0C4
:103CD0008ACFC418D508E608F708D7CFC8010E94D4
:103CE0009F176EA77FA788AB99AB8AA69BA6ACA6A9
:103CF000BDA68EA59FA5A8A9B9A90097A105B10544
:103D000009F471CFB701A60129E07695679557951B
:103D100047952A95D1F7840F951FA61FB71F8EA729
:103D20009FA7A8ABB9ABF1E0DF2287E3C80ED11C97
:103D3000C00ED11EDBAACAAA80E001C081E0DF91DB
:103D4000CF911F910F91FF90EF90DF90CF90BF9098
:103D5000AF909F908F907F906F905F904F9008955D
:103D6000CF93DF93EC011B828FEF9FEFDC018BABD6
:103D70009CABADABBEABCE010E94631B811134C0C6
:103D8000FE01EA5CFD4F808190E0982F88273197F3
:103D90002081822B85359A4A49F54BE050E065E059
:103DA00076E0CE01C7960E949017892B09F18FA962
:103DB0008B3E19F0885E8230F8F443E050E061E118
:103DC00076E0CE0183599F4F0E949017892B91F086
:103DD00045E050E065E176E0CE0187579F4F0E94B5
:103DE0009017892B49F406C084E007C083E005C022
:103DF00081E003C080E001C082E0DF91CF910895AF
:103E00002F923F924F925F926F927F928F929F92EA
:103E1000AF92BF92CF92DF92EF92FF920F931F93D8
:103E2000CF93DF93CDB7DEB7E2970FB6F894DEBF3E
:103E30000FBECDBF6B01142FDB011D921C920E949F
:103E400007187C0197FD84C2FC01EE0FFF1FE152B1
:103E5000F44F208031802114310409F47BC2F60133
:103E6000318220821E7FD1018C91882369F01196C6
:103E70008C910E94CD1480FD07C0112309F46CC2FF
:103E800082FF6AC28AE02CC4F1011082E1828E2D89
:103E90000E940D1480FD62C2112311F082FDF2CF49
:103EA00040E050E0BA01C1010E94B01E823009F02A
:103EB00043C08E010F5F1F4F7801810103501E4FD9
:103EC000510123ECA21A2DEFB20A6701F8013497D1
:103ED0008081882321F0C8010E94121703C060E08E
:103EE00070E0CB01D6016D937D938D939D936D0111
:103EF000005F1F4F0A151B0549F78E010F5E1F4F0C
:103F0000D7014D905D906D907D907D01498E5A8EC8
:103F10006B8E7C8E411451046104710441F0B30135
:103F2000A201C1010E94B01E823010F411C083E0D2
:103F3000E016F10629F7D0C3198E1A8E1B8E1C8E3F
:103F4000843011F481E0CCC3823010F08DE0C8C31E
:103F5000F101EE5BFF4F813051F4910129583F4F41
:103F600081918111F3CFE217F307D1F7F9C1D101A4
:103F7000AD5BBF4F8C9190E0982F88272081822BDA
:103F80008115924019F7F101E25BFF4F8080912C7F
:103F9000982C882431978081882A8114910419F003
:103FA000A12CB12C07C0C101855A9F4F0E94121746
:103FB0004B015C01D1015B968D929D92AD92BC92BA
:103FC0005E97F101E95BFF4F0081F10102838FEF02
:103FD000800F823008F0BACFEC5BFF4F1081812F49
:103FE00090E01A969C938E931997009709F4AECFA0
:103FF0009C012150310982239323892B09F0A6CFFC
:104000003596808190E0382F2227319780812901D1
:10401000482A5A8A498A18965C924E921797C2018A
:104020008F709927892B09F091CF3396808190E08A
:10403000982F882731972081822B2C01612C712C9D
:10404000892B39F4C101895A9F4F0E9412172B0105
:104050003C01F101EA5BFF4FE081F0E0FE2FEE272B
:10406000D101AB5BBF4F8C91E82B309709F46ECF39
:10407000A02FB0E0A50194010E9441736D8F7E8F47
:104080008F8F98A36F01E12CF12CC9A2DAA2EBA2C9
:10409000FCA289899A89B4E096958795BA95E1F74B
:1040A000C80ED91EE11CF11CD701C601CD8CDE8CD7
:1040B000EF8CF8A0C80ED91EEA1EFB1E4C145D043E
:1040C0006E047F0408F442CFC301B2016C197D096C
:1040D0008E099F09212F30E040E050E00E9480735C
:1040E000211531054105510509F430CF263F0FEF69
:1040F000300740070FE0500708F028CF263F1FEF9A
:1041000031074105510540F4263F8FE0380741054E
:10411000510520F411E003C013E001C012E02901B1
:104120003A0192E0490E511C611C711CD101579655
:104130004D925D926D927C925A97298D3A8D4B8D5E
:104140005C8D5F962D933D934D935C939297DA012E
:10415000C90129A13AA14BA15CA1820F931FA41F01
:10416000B51FF10183A394A3A5A3B6A3498D5A8DCE
:104170006B8D7C8D4C0D5D1D6E1D7F1D43A754A75F
:1041800065A776A7133029F5EE59FF4F808190E09F
:10419000982F882731972081822B892B09F0D6CE42
:1041A000C988DA88CD2809F0D1CEC1018D599F4F39
:1041B0000E941217D10197966D937D938D939C93D6
:1041C0009A97E2E0440C551C661C771CEA95D1F7DF
:1041D0002DC0C988DA88CD2809F4B8CECD8CDE8C04
:1041E000EF8CF8A0C80ED91EEA1EFB1EC7A2D0A6EF
:1041F000E1A6F2A6123029F4440C551C661C771C6B
:1042000015C0A3E0B0E0A30192010E944173DC015C
:10421000CB01B695A79597958795E1E04E22552459
:1042200066247724480E591E6A1E7B1EFFEF4F0E30
:10423000F1E05F1E611C711C59E0769467945794FD
:1042400047945A95D1F784149504A604B70408F44A
:104250007DCE8FEF9FEFDC01F101838B948BA58BDB
:10426000B68B8787908BA18BB28B80E884831330C9
:1042700009F052C0E859FF4F808190E0982F8827BD
:1042800031972081822B019709F046C0498D5A8DC4
:104290006B8D7C8D4F5F5F4F6F4F7F4FC1010E94D1
:1042A000631B811139C0D10114961C92F101EA5CA3
:1042B000FD4F808190E0982F882731972081822BB5
:1042C00085359A4A49F5C101C7960E941217623591
:1042D00072458146914401F5C101855E9D4F0E9462
:1042E00012176237724781449146B1F4C101815E71
:1042F0009D4F0E941217D10153966D937D938D931C
:104300009C935697C1018D5D9D4F0E941217F1013C
:104310006787708B818B928BD1011C938091DD0B11
:104320009091DE0B01969093DE0B8093DD0B169639
:104330009C938E9315978DE797E01C969C938E9394
:104340001B978DE799E01E969C938E931D9704C052
:104350008BE0C6C18CE0C4C180E0C2C183E0C0C1B3
:10436000F101E056FF4F808190E0982F8827319728
:104370002081822B8115914009F0E8CDF101ED55A6
:10438000FF4F81E090E0008002C0880F991F0A94DF
:10439000E2F78115924009F0D9CDC10181589F4FB4
:1043A0000E942D17498C5A8C6B8C7C8C53014201D6
:1043B000C12CD12C7601498A9A8AAB8ABC8ACD8AD3
:1043C000DE8AEF8AF88E5201CB88DC88E12CF12C52
:1043D00000E010E00E9441742D8F39A3742E652EE9
:1043E000562E472E8DA39EA3562D652D742D2F3F3F
:1043F0003F4F4F4F5F4F610571058105910511F0EA
:1044000008F0A4CDC10185579F4F0E941217D1011A
:104410005B966D937D938D939C935E97F101EB5525
:10442000FF4F8081F1018283813009F08FCDEC55FF
:10443000FF4F01E010E0008002C0000F111F0A943E
:10444000E2F71A961C930E9319970115110509F4BA
:104450007DCDC1018D569F4F0E9412179B01AC016B
:104460006E3FBFEF7B078B07BFE79B0708F06ECD62
:10447000DC01CB010296A11DB11DF101878B908F4C
:10448000A18FB28F898C9A8CAB8CBC8C878E90A2BA
:10449000A1A2B2A2C10181579F4F2FA338A749A75C
:1044A0005AA70E941217860E971EA81EB91E898A47
:1044B0009A8AAB8ABC8AF10183A694A6A5A6B6A661
:1044C000C10189579F4F0E941217898C9A8CAB8C1F
:1044D000BC8C860E971EA81EB91EF10183A294A261
:1044E000A5A2B6A2A988BA88CB88DC884501560166
:1044F000C12CD12C76018BA69CA6ADA6BEA6CFA6BC
:10450000D8AAE9AAFAAAD8012FA138A549A55AA57F
:104510000E9441737B018C0120E030E0A901698B8E
:10452000FA8A0B8B1C8B2D8B3E8B4F8B588F9401F3
:10453000A50160E070E080E090E057016801E12CA7
:10454000F12C00E010E00E94417459016A017B01E6
:104550008C012D8D39A1472D562D652D742D8DA1E2
:104560009EA10E945F7408F4F1CCC10189569F4F4F
:104570000E941217D10197966D937D938D939C9312
:104580009A97C12CD12C760100E010E0011511059D
:1045900011F5F10181859285A0E0B0E0C816D90639
:1045A000EA06FB0608F0D2CC47A150A561A572A58A
:1045B000C1010E949F17AB01BC014C0D5D1D6E1D1A
:1045C0007F1DC1010E94631B8111BCCCFFEFCF1A7C
:1045D000DF0AEF0AFF0AF101E00FF11F87A9813816
:1045E00021F0005E1F4F1170D1CFC801855B9F4F36
:1045F000820D931D0E9412176B017C0162307105C0
:104600008105910508F4A2CCF1018789908DA18DD7
:10461000B28DC816D906EA06FB0608F097CCA1852C
:10462000B285A701960122503109410951090E9422
:10463000417303A514A525A536A5DC01CB01800F88
:10464000911FA21FB31F87A790ABA1ABB2ABF10123
:1046500083A194A1A5A1B6A1B701A601E7E0769533
:10466000679557954795EA95D1F7480F591F6A1FE7
:104670007B1FC1010E94631B811164CCC6018F772F
:104680009927880F991F880F991FC796820D931D30
:104690000E9412176F3FFFEF7F078F079F0771F090
:1046A0000FEFC01AD00AE00AF00A6C157D058E05DE
:1046B0009F0509F04BCC6B017C01C9CFD10153960A
:1046C0006D937D938D939C935697F1016787708BC3
:1046D000818B928B14E020CE843009F037CC32CC21
:1046E000E2960FB6F894DEBF0FBECDBFDF91CF913B
:1046F0001F910F91FF90EF90DF90CF90BF90AF9000
:104700009F908F907F906F905F904F903F902F90F1
:1047100008952F923F924F925F926F927F928F9265
:104720009F92AF92BF92CF92DF92EF92FF920F9340
:104730001F93CF93DF9300D000D0CDB7DEB71C011D
:104740006A017B012801390142305105610571057B
:1047500008F4EEC0FC018789908DA18DB28D4817B9
:1047600059076A077B0708F0E3C08081823009F4AB
:104770007AC018F4813029F0DBC0853008F495C088
:10478000D7C05A01B694A794A40EB51EC501892FAF
:1047900099278695D10193964D915D916D917C916C
:1047A0009697480F591F611D711DC1010E94631B1F
:1047B000182F8111BEC04501BFEF8B1A9B0AE1E0A3
:1047C000BE22A20CB31CD701C60181709927AA276B
:1047D000BB2789839A83AB83BC83C0FE0BC0D50102
:1047E000D7968C91282F2F70B0E14B9EC0011124D9
:1047F000822B01C0842DF50187AB81E0D101139696
:104800008C93139793964D915D916D917C919697B2
:10481000C401892F99278695480F591F611D711D65
:10482000C1010E94631B182F811183C0B1E09B223C
:10483000F101E80DF91D89819A81AB81BC81892B39
:104840008A2B8B2B41F054E07694679457944794CD
:104850005A95D1F706C067A9607F852D8F70462EC7
:10486000482A47AA60C077276F2D5E2D4D2DF10194
:1048700083A194A1A5A1B6A1480F591F6A1F7B1F50
:10488000C1010E94631B182F811153C0CC0CDD1C89
:10489000E894C0F8F1E0DF22F101EC0DFD1D47AA1C
:1048A000F101EC0DFD1D50AE3EC0F10183A194A1BC
:1048B000A5A1B6A127E076956795579547952A95C6
:1048C000D1F7480F591F6A1F7B1FC1010E94631B4C
:1048D000182F81112EC0D1018C91CC0CDD1CCC0C79
:1048E000DD1C8430A1F0BFE07B22C6018C7F91707B
:1048F000C796820D931D0E941217DC01CB018827F9
:104900009927AA27B07F482A592A6A2A7B2AECEFDE
:10491000CE22E1E0DE22C601C796B301A201820DDC
:10492000931D0E94561781E0D10113968C9301C00C
:1049300012E0812F0F900F900F900F90DF91CF9189
:104940001F910F91FF90EF90DF90CF90BF90AF90AD
:104950009F908F907F906F905F904F903F902F909F
:1049600008952F923F924F925F926F927F928F9213
:104970009F92AF92BF92CF92DF92EF92FF920F93EE
:104980001F93CF93DF9300D000D0CDB7DEB79C83C9
:104990008B836A017B0109831A83322E232E82E0E6
:1049A000882E912CA12CB12C412C512C32014394F6
:1049B000EB81FC8186899789A08DB18D0097A10537
:1049C000B105A1F182309105A105B10558F095011D
:1049D0008401081B190B2A0B3B0B0C0D1D1D2E1DF2
:1049E0003F1D04C009811A81232D322DB301A2017C
:1049F000481B590B6A0B7B0B4C0D5D1D6E1D7F1DFB
:104A0000EB81FC81808191810E94892381110FC0FB
:104A1000EB81FC8186899789A08DB18D0197A109D1
:104A2000B109868B978BA08FB18FC2CF80E00F909A
:104A30000F900F900F90DF91CF911F910F91FF90EA
:104A4000EF90DF90CF90BF90AF909F908F907F902E
:104A50006F905F904F903F902F9008952F923F92CC
:104A60004F925F926F927F928F929F92AF92BF927E
:104A7000CF92DF92EF92FF920F931F93CF93DF932A
:104A800000D000D000D0CDB7DEB71C016A017B0199
:104A900028013901DC010D90BC91A02DBE83AD83AE
:104AA000423051056105710510F482E003C1ED81CA
:104AB000FE818789908DA18DB28D481759076A07AD
:104AC0007B0798F7012B022B032B29F4C982DA828A
:104AD000EB82FC825BC0AD81BE818C91843021F47D
:104AE000F1018581823091F30FEF1FEF9801B3013F
:104AF000A2018D819E810E948923882339F3DAC027
:104B0000613071058105910581F26F3F7F4F8F4FB5
:104B10009F4F09F46EC0AD81BE818C91843009F045
:104B20006AC0ED81FE8183899489A589B689478908
:104B3000508D618D728D4250510961097109841740
:104B40009507A607B70750F40196A11DB11D838BE9
:104B5000948BA58BB68B848181608483FFEFCF1A01
:104B6000DF0AEF0AFF0AC814D904EA04FB0409F0BB
:104B70004EC075016401ED81FE818789908DA18D04
:104B8000B28D88169906AA06BB0668F4B701A6017D
:104B9000C1010E94231C4B015C0161157105810557
:104BA000910509F0ADCFAD81BE818C91843009F0C3
:104BB00080C04BC0F101858181115EC0C680D78065
:104BC000E084F184C414D504E604F70409F46DC04C
:104BD000B701A601C1010E94231C62307105810545
:104BE000910508F462CF6F3FFFEF7F078F079F07A4
:104BF000B1F581E05FC000E010E09801B701A601C7
:104C0000CD010E948923882309F48BCF53C0AD8145
:104C1000BE818C918430A1F49701860189819A81AB
:104C2000AB81BC81081B190B2A0B3B0BE12CF12C2F
:104C3000AC01BD018D819E810E94A11B81113AC0F2
:104C400089829A82AB82BC8294CF41145104610460
:104C5000710409F0AFCFD10115961C922AC02FEF35
:104C6000C21AD20AE20AF20A6C157D058E059F056A
:104C700001F56B017C01A6CF8330D9F4F1014681A7
:104C8000578160857185441655066606770688F05B
:104C900082899389A489B589840F951FA61FB71FA0
:104CA00084159505A605B70520F082E0D10115967B
:104CB0008C9380E026960FB6F894DEBF0FBECDBF72
:104CC000DF91CF911F910F91FF90EF90DF90CF90E8
:104CD000BF90AF909F908F907F906F905F904F901C
:104CE0003F902F9008958F929F92AF92BF92CF9254
:104CF000DF92EF92FF920F931F93CF93DF93EC011C
:104D00004E815F8168857985CA88DB88EC88FD885B
:104D1000C40ED51EE61EF71E4C155D056E057F05FB
:104D200091F04A015B018FEF881A980AA80AB80A25
:104D300095018401888199810E948923811105C090
:104D4000B501A401E9CF1D8280E0DF91CF911F91D1
:104D50000F91FF90EF90DF90CF90BF90AF909F901A
:104D60008F9008956F927F928F929F92AF92BF9291
:104D7000CF92DF92EF92FF920F931F93CF93DF9327
:104D800000D000D0CDB7DEB73C0149835A836B8396
:104D90007C830E940F1B49815A816B817C81811128
:104DA00039C0C3010E949F174B015C01F30163AB43
:104DB00074AB85AB96AB6301F7E3CF0ED11C40E03B
:104DC00052E060E070E0C6010E948717E12CF12CF0
:104DD000F30181859285E816F90648F081E0F30138
:104DE00021853285E216F306B1F480E014C001E0BB
:104DF00010E0A50194012E0D3F1D411D511DB6016E
:104E0000F30181810E941F158111E8CF8FEFE81A0D
:104E1000F80ADECF81E00F900F900F900F90DF9196
:104E2000CF911F910F91FF90EF90DF90CF90BF90A7
:104E3000AF909F908F907F906F9008953F924F9288
:104E40005F926F927F928F929F92AF92BF92CF921A
:104E5000DF92EF92FF920F931F93CF93DF93CDB723
:104E6000DEB72A970FB6F894DEBF0FBECDBF6C0138
:104E700049835A836B837C83DC010D90BC91A02D08
:104E8000BA87A987452B462B472BB9F41F964D901F
:104E90005D906D907C9052974114510461047104AF
:104EA000A9F157968D919D910D90BC91A02D48161A
:104EB00059066A067B0670F129C049815A816B81C7
:104EC0007C810E94231C4B015C01623071058105CD
:104ED000910508F43AC26F3F7F4F8F4F9F4F29F4DF
:104EE0006FEF7FEF8FEF9FEF3BC2E985FA858789F0
:104EF000908DA18DB28D88169906AA06BB0608F47E
:104F000029C249805A806B807C8004C0412C512C7E
:104F100032014394E985FA8583899489A589B68904
:104F2000892B8A2B8B2B11F460E010C2A985BA85DE
:104F30002C9157968D919D910D90BC91A02D243070
:104F400009F02FC1A30192012250310941095109F1
:104F50002D833E834F8358870297A109B1092817F3
:104F600039074A075B0720F01D821E821F821886C0
:104F70008D809E80AF80B88433243394E985FA8590
:104F800087A590A9A1A9B2A9B501A4011CE07695B5
:104F90006795579547951A95D1F7480F591F6A1F7E
:104FA0007B1FCF010E94631B81115DC0D501C4012D
:104FB00043E0B695A795979587954A95D1F79C01BB
:104FC0003170C40187709927F32D01C0FF0F8A95B6
:104FD000EAF78F2FA985BA8557964D915D916D910E
:104FE0007C915A977A018B01B2E0EB1AF108010922
:104FF0001109E985FA85E20FF31F97A99823B501F6
:10500000A4014F5F5F4F6F4F7F4F4E155F056007E5
:10501000710710F4880F06C040E050E0BA0120E0AC
:1050200032E080E0911106C0E2E08E0E911CA11CDE
:10503000B11C21C08D809E80AF80B8844815590571
:105040006A057B05A9F0882319F04A015B01D1CFDD
:105050002F5F3F4F211582E0380710F481E0F5CF34
:105060004A015B018BCF88248A94982C540103C099
:10507000812C912C5401D501C4010197A109B109DA
:105080008E3F9F4FAF4FBF4F08F064C1EE24E394B3
:10509000F12C01E010E020E030E0B501A4018985A9
:1050A0009A850E94A11B823009F44FC1813009F416
:1050B00017CF29813A814B815C81232B242B252B0F
:1050C00019F492E0D6011DC0F60195819230D9F411
:1050D000B301A2014F5F5F4F6F4F7F4F841695065C
:1050E000A606B70681F04681578160857185441A0E
:1050F000550A660A770AD601428A538A648A758AF3
:1051000093E015969C93F6019581923009F425C1A0
:1051100046895789608D718D09811A812B813C8167
:105120000F5F1F4F2F4F3F4F80169106A206B30609
:10513000B1F4411551056105710529F04F5F5F4FCD
:105140006F4F7F4F04C042E050E060E070E0D60156
:1051500056964D935D936D937C935997FEC0452B66
:10516000462B472B49F481E090E0A0E0B0E0F60147
:10517000868B978BA08FB18F9501840149815A81CD
:105180006B817C81C6010E94B1248111DBC081E06A
:1051900090E0A0E0B0E0F601868B978BA08FB18FF6
:1051A000A7C089809A80AB80BC80481459046A04E7
:1051B0007B0409F043C0530142012FEF821A920A87
:1051C000A20AB20A88169906AA06BB0628F092E03F
:1051D000892E912CA12CB12CB501A401C6010E94ED
:1051E000231C613071058105910509F4AEC06F3F44
:1051F0003FEF73078307930709F472CE672B682B81
:10520000692BB9F0E985FA8587859089A189B289EA
:1052100082309105A105B10588F04789508D618DD7
:10522000728D84179507A607B70740F42C013D013E
:1052300005C081149104A104B104E9F553014201B0
:10524000FFEF8F1A9F0AAF0ABF0AE985FA8587899F
:10525000908DA18DB28D88169906AA06BB0660F0C6
:10526000F2E04F1651046104710408F45DCE82E04F
:10527000882E912CA12CB12CB501A401C6010E944D
:10528000231C8B019C01611571058105910599F025
:10529000613071058105910529F06F3F7F4F8F4F78
:1052A0009F4F19F4B801C9015BC084149504A6048A
:1052B000B70431F639CE0FEF1FEF9801B501A40105
:1052C00089859A850E94892381113CC089819A81B0
:1052D000AB81BC810097A105B10551F09501840116
:1052E000AC01BD0189859A850E94892381112AC05C
:1052F000A985BA851F968D929D92AD92BC925297C8
:10530000FD0183899489A589B6894789508D618D6E
:10531000728D4250510961097109481759076A078E
:105320007B0738F00197A109B109838B948BA58B7A
:10533000B68BA985BA8514968C91149781601496C2
:105340008C9308C0813009F4CBCD61E070E080E03F
:1053500090E006C0B401C50103C0882349F2F5CF2F
:105360002A960FB6F894DEBF0FBECDBFDF91CF9166
:105370001F910F91FF90EF90DF90CF90BF90AF9073
:105380009F908F907F906F905F904F903F90089587
:105390004F925F926F927F92AF92BF92CF92DF92C5
:1053A000EF92FF920F931F93CF93DF93EC0108814D
:1053B0001981CEA0DFA0E8A4F9A480E2C80ED11C18
:1053C000E11CF11CF8018081843029F080E090E03C
:1053D000A0E2B0E004C080E090E0A0E0B0E1C81638
:1053E000D906EA06FB0620F01EA61FA618AA19AACF
:1053F0008EA59FA5A8A9B9A90097A105B10509F493
:10540000AAC05B01B701A601517066277727452B1B
:10541000462B472B09F090C00196A11DB11D8EA708
:105420009FA7A8ABB9AB4AA55BA56CA57DA5F80164
:105430004115510561057105C1F487819085A0E092
:10544000B0E0B701A60135E0769567955795479589
:105450003A95D1F7481759076A077B0708F46CC0DB
:105460001EA61FA618AA19AA76C081859285019743
:10547000A0E0B0E02601370129E0769467945794C4
:1054800047942A95D1F784219521A621B721892B0C
:105490008A2B8B2B09F050C0CE010E94231C2B01BC
:1054A0003C01623071058105910510F482E056C01F
:1054B0008FEF481658066806780611F481E04EC052
:1054C000F8018789908DA18DB28D481659066A061C
:1054D0007B0628F1AB2821F24AA55BA56CA57DA52A
:1054E000CE010E941E272B013C016115710581052B
:1054F000910599F16130710581059105B9F28FEF40
:105500004816580668067806C9F2B301A201C80118
:105510000E94B2268111D2CF8D8184608D834AA6EC
:105520005BA66CA67DA6B301A201C8010E949F17CD
:105530006EA77FA788AB99ABCEA2DFA2E8A6F9A69B
:10554000E1E0DE22F7E3CF0ED11CC00ED11EDBAAB4
:10555000CAAA80E003C084E001C087E0DF91CF9158
:105560001F910F91FF90EF90DF90CF90BF90AF9081
:105570007F906F905F904F900895CF92DF92EF925F
:10558000FF920F931F93CF93DF93EC016B01E880A1
:10559000F98040E050E0BA010E94CC1D81112FC07B
:1055A00000E010E04EA55FA568A979A9C7010E9497
:1055B000631B811124C0F7019081EAA9FBA99430F3
:1055C00031F490819095991F9927991F07C02081E8
:1055D00091E0253E11F0211190E09170992331F076
:1055E0000F5F1F4F0C151D0519F40CC000E010E0F3
:1055F00061E070E0CE010E94C829882399F28430CE
:1056000009F487E0DF91CF911F910F91FF90EF9008
:10561000DF90CF900895AF92BF92CF92DF92EF923A
:10562000FF920F931F93CF93DF93EC0108811981B1
:10563000CEA0DFA0E8A4F9A4FC01E05CFF4F40810C
:105640005181628173814F3F8FEF58076807780758
:1056500029F485EEB82EAA24A39421C0CE010E947D
:10566000CC1D81112BC0F5CFF8019081EAA9FBA9CF
:105670009430F9F490819F779083F801A3824EA132
:105680005FA168A579A54C155D056E057F05B0F491
:1056900060E070E0CE010E94C82981110CC04EA5C7
:1056A0005FA568A979A9C8010E94631B8823E1F25C
:1056B00002C0B082E2CF843009F482E0DF91CF9162
:1056C0001F910F91FF90EF90DF90CF90BF90AF9020
:1056D0000895EF92FF920F931F93CF93DF93EC0106
:1056E0000E940F1B982F81115CC08881833009F0C4
:1056F0004EC08C81813009F04AC040E052E060E049
:1057000070E07E0187E3E80EF11CC7010E94871755
:1057100085E5FE01EB5CFD4F80838AEA319680834C
:1057200082E58FAB88AF81E689AF91E49AAF22E73B
:105730007B972083319620833196908331968083A6
:105740004B895C896D897E89CE01815E9D4F0E9467
:1057500056174F85588969897A89CE018D5D9D4F8D
:105760000E9456178F8D98A1A9A1BAA19C01AD01E5
:105770002F5F3F4F4F4F5F4F2BAB3CAB4DAB5EAB03
:1057800001E010E0B70189810E941F151C8240E0F2
:1057900050E060E089810E94901591E0811101C084
:1057A00090E0892FDF91CF911F910F91FF90EF90A3
:1057B0000895CF92DF92EF92FF920F931F93CF93B2
:1057C000DF938C01DC01ED91FC91E584F684C70147
:1057D0000E94D617F70182839383C180F801E05CB1
:1057E000FF4F4081518162817381C8010E94CC1DAD
:1057F000C82FD12CD1E0C1112AC0D8019E964D915D
:105800005D916D917C91D1978D919C910E94631BCC
:10581000C82F81111CC040E250E0B701F80182A9F5
:1058200093A90E94AD1AD801ED91FC91D383C114C4
:10583000D10469F0B0E2EB0EF11C60E070E0C80149
:105840000E94C829C82FE1E0CE1AD108D4CF8C2FEE
:10585000C33008F082E0DF91CF911F910F91FF904C
:10586000EF90DF90CF900895CF92DF92EF92FF926A
:105870000F931F93CF93DF93EC0188819981FC01F3
:10588000058516854EA55FA568A979A90E94631BA9
:10589000811191C06AA97BA9FB018081853809F03B
:1058A00063C040E250E0C8010E94AD1AF801E180F7
:1058B000F12CFFEFEF1AFF0AF5E0EE0CFF1CFA9552
:1058C000E1F7C701805691098130924008F04CC041
:1058D00060E070E0CE010E94C829843009F444C021
:1058E000811169C04EA55FA568A979A988819981B0
:1058F0000E94631B81115FC06AA97BA9FB018081A3
:10590000803C91F540E250E0C80180960E94AD1ABB
:10591000F80183A190E08C966FE070E00E945873CC
:10592000E5E0660F771FEA95E1F7E616F706E0F087
:1059300050E4C52ED12C60E070E0CE010E94C82951
:10594000843091F0811137C04EA55FA568A979A96F
:10595000888199810E94631B81112DC06AA97BA94E
:10596000FB018081813C11F082E025C0F0E6CF167A
:10597000F2E0DF0638F440E250E0C8018C0D9D1DD6
:105980000E94AD1A20E2C20ED11CCE14DF0498F2A0
:1059900081E6C81682E0D80668F4C8010E94D617CE
:1059A000F801238130E0322F22274281242B8217F5
:1059B0009307D1F680E0DF91CF911F910F91FF9077
:1059C000EF90DF90CF9008954F925F927F928F92E9
:1059D0009F92AF92BF92CF92DF92EF92FF920F937E
:1059E0001F93CF93DF93EC016B01E880F9800FEFF9
:1059F0001FEF84E0B82E9DE0792E4E0160E4860E04
:105A0000911C4EA55FA568A979A9411551056105AD
:105A1000710509F4CFC0C7010E94631BB82E811124
:105A2000CBC0EAA9FBA98081882309F4CCC0D701A7
:105A30009C91943019F5C114D10421F0833809F0F8
:105A4000AFC0C6C0853809F0ABC08EA19FA1A8A584
:105A5000B9A5FE01E05CFF4F80839183A283B383ED
:105A6000CE010E94342C8111B1C0D7011D96ED9159
:105A7000FC911E9784818F738C83AAC093859F733A
:105A80009C83853E09F48BC08E3209F488C021E0E6
:105A900030E0492F4F71483011F020E030E02C15F4
:105AA0003D0509F07CC09F3009F068C086FF0EC03C
:105AB0000585182F1F7B4EA15FA168A579A5D4018C
:105AC0004D935D936D937C93139702C0811367C0D0
:105AD0008585081364C0D7011B96AD90BC901C97B8
:105AE000838D90E0982F8827228D822B892B09F0B7
:105AF00056C0808190E08F7B0197789E9001799EBF
:105B0000300D1124AAE14A2EA2E05A2E41E050E0C5
:105B1000D2018D912D01BF01680F711DDB0111961E
:105B20008C91119790E0982F88276C91862B4115C6
:105B3000510579F02F3F310590F5A901440F551F0C
:105B40004A0D5B1DDA018D939C93AC012F5F3F4F93
:105B500002C0019621F567E2461662E05606C1F6DC
:105B6000808186FF2EC02F3F3105C8F4220F331FDE
:105B7000F501E20FF31F1182108223C0111105C03D
:105B8000CF010E94C717081719F1C05CDF4F8FEFD4
:105B90009FEFDC0188839983AA83BB8319C01FEF21
:105BA00060E070E0CE010E94C829B82E882309F475
:105BB00028CF02C0BB2061F01EA61FA618AA19AAF2
:105BC00007C01150EDCF84E0B82EF6CFB82EF4CF39
:105BD0008B2DDF91CF911F910F91FF90EF90DF9070
:105BE000CF90BF90AF909F908F907F905F904F909D
:105BF00008952F923F924F925F926F927F928F9271
:105C00009F92AF92BF92CF92DF92EF92FF920F934B
:105C10001F93CF93DF93CDB7DEB72F970FB6F894CE
:105C2000DEBF0FBECDBF9F878E87DC018D909C901D
:105C300040E050E0BA010E94CC1D81117FC1F40107
:105C40008081843009F06CC0838594850E94741A29
:105C50005C0160E070E08E859F850E94E42C382E08
:105C600081115CC0D4011D96ED91FC911E9785A118
:105C700090E0982F882724A1822B8A159B0549F74D
:105C8000C3A0D12C00E010E080E4E82EF12C0C152C
:105C90001D05B1F1C7018F719927892B19F4B2E065
:105CA000EB0EF11CD4011D96ED91FC911E97EE0DAB
:105CB000FF1D618170E0762F66278081682B80E070
:105CC00090E00E94D64E2B013C01F401438554859F
:105CD0009801220F331FFA01E20FF31F60817181D7
:105CE00080E090E00E94D64E461657066806790678
:105CF00009F0AFCFF2E0EF0EF11C0F5F1F4FC7CFDF
:105D0000000F111FD4011B96ED91FC911C97E00F21
:105D1000F11F80819181892B09F09BCF832D0EC1CA
:105D2000AE84BF8420E4A20EB11C8FEF9FEFDC0194
:105D3000F50180839183A283B3832FEF29833FEF03
:105D40003D8744244A94542C32012E853F852C5C97
:105D50003F4F3B872A87AE85BF859E964D915D91CB
:105D60006D917C91D197C4010E94631B8111E6C0A3
:105D7000EE85FF85E2A8F3A8D7018C91882309F46A
:105D8000D5C01B963C91932F9F739483853E09F455
:105D9000B9C033FF04C09F3009F0B4C003C09F30C6
:105DA00009F098C0AE85BF85DF969C91DF9796FD80
:105DB000B3C086FF11C0F701F585F9838F7B8D870E
:105DC00096968D919D910D90BC91A02DF5018083AB
:105DD0009183A283B38303C02D85821399C0D70119
:105DE0001D968C912981281395C0D4011B96CD90C6
:105DF000DC901C97F701838D90E0982F8827328DD7
:105E0000832B892B09F086C080818F7390E00197E6
:105E1000FDE0F89F8001F99F100D11242AE132E086
:105E20003B832A8341E050E0AA81BB818D91BB83F3
:105E3000AA83F701E80FF11D818190E0982F882750
:105E400030811C01232A4115510559F10F3F1105DD
:105E500008F060C0B10180E090E00E94D64E6C83F3
:105E60007D838E839F8398012F5F3F4F39872887DB
:105E7000000F111FF601E00FF11F80819181BC011D
:105E800080E090E00E94D64E2C813D814E815F8162
:105E90002617370748075907E9F5A101088519852D
:105EA00003C023202094B1F52A813B812752324040
:105EB00009F0BACFD7018C9186FF3CC0452BD1F1B8
:105EC000000F111FF601E00FF11F80819181892BD6
:105ED00089F120C02D85211106C0C7010E94C71776
:105EE0003981381729F1AE85BF85DF968C9180FD09
:105EF00009C04BE050E06A857B85C7010E9490177E
:105F0000892BB1F0F501408251826282738202C016
:105F10003FEF12C02FEF2D8760E070E08E859F85E8
:105F20000E94C829882309F416CF08C084E006C05F
:105F300080E004C03D8531503D87EECF2F960FB6EF
:105F4000F894DEBF0FBECDBFDF91CF911F910F91AF
:105F5000FF90EF90DF90CF90BF90AF909F908F9089
:105F60007F906F905F904F903F902F9008952F9269
:105F70003F924F925F926F927F928F929F92AF92D9
:105F8000BF92CF92DF92EF92FF920F931F93CF9326
:105F9000DF93CDB7DEB7CE54D1090FB6F894DEBF8C
:105FA0000FBECDBFDC016D907C901197DF962C91D8
:105FB000207A09F0D0C2D3011B96ED91FC911C9779
:105FC000E12CF12C21913191232B21F0BFEFEB1A21
:105FD000FB0AF8CF4C01F3018081843009F032C113
:105FE000C7010E966FE070E00E9458738B016E5FE0
:105FF0007F4FC4010E94BD2A8111AEC29401205C72
:106000003F4F0F5F174F45E0000F111F4A95E1F713
:10601000F40186A197A1A0A5B1A5801B910BA109B0
:10602000B109F90180839183A283B383D4011596CA
:106030008C91159782FFAFC08B7F15968C93833020
:1060400071F0F40142A553A564A575A50FEF1FEFEC
:106050009801C4010E94B124882339F07DC2C40193
:106060000E947326811178C2ECCFF401868197815A
:10607000A085B185892B8A2B8B2B09F48CC080815C
:1060800091819A838983828D938DA48DB58D8F8321
:106090009887A987BA87068D178D20A131A10E8315
:1060A00000270B871C872D873E871F86188A198A31
:1060B0001A8A1F8A188E198E1A8E42A153A164A1C2
:1060C00075A125964CAF5DAF6EAF7FAF2597CE0122
:1060D00001960E94CC1D81113FC2CE0101960E9403
:1060E000342C811139C2D3011996AD90BC901A9706
:1060F000C501A0E0B0E029E0880F991FAA1FBB1FCF
:106100002A95D1F75C016D019C01A60160E070E069
:1061100080E090E0F401A284B384C484D584E68452
:10612000F784008911890E9441742287338744874C
:10613000558766877787808B918BD3011D96ED916C
:10614000FC911E9789019A01AB01BC01CF01C89651
:106150000E945C17F40102851385248535854685E8
:10616000578560897189D3011D968D919C911E97E9
:1061700088960E945C17D3011D96ED91FC911E97A5
:10618000D40115968C91816081A3CE0101960E9465
:10619000D92B8111E1C1F301E384F48405851685CF
:1061A00040E450E060E070E0C8010E94871785E895
:1061B000D8018C9380EC90968C9341E050E020E0E5
:1061C00030E080E490E0B1ECF801E80FF91FB08313
:1061D000FC013196E00FF11F029610824115510526
:1061E00059F0F701E20FF11DE20FF11D40815181DD
:1061F0004115510509F02F5FF801E80FF91F4083A1
:1062000051830296BC016F717727672B39F7A1E0A4
:10621000A30FF701E20FF11DE20FF11D6081718103
:10622000672B11F03A2FD0CFF80123A33E5F3183C3
:10623000C7010E94741AD80194968C9394979596EE
:106240009C9387C16401B4E3CB0ED11C4CE050E0B9
:10625000B601CE0101960E94AD1A8C8580FFAEC0BA
:1062600080E4F40187AF212C312C2101239485E4B3
:10627000A82EB12CAC0EBD1EF8E0AF0EB11C8101F2
:10628000D3011B962C911B971C963C914BE050E040
:10629000BE016F5F7F4FC6012E962FAF2E972F96B0
:1062A0003FAF2F970E94AD1A2E962FAD2E972F96A7
:1062B0003FAD2F97B6E02B1631044104510418F17D
:1062C000F901B201A101819191910097D9F020E1EA
:1062D00030E0440F551F661F771FDC01A170BB27FC
:1062E0004A0F5B1F611D711D9695879560FF06C063
:1062F000A1E24A27A0E15A27A1E06A2721503109EB
:1063000041F7E1CF8A01F50127E030E0902F9F703F
:1063100080E3890F8A3310F087E3890F2150310918
:106320008293A4E016950795AA95E1F7011511054A
:1063300069F7E5E4F0E0EC0FFD1FE20FF31FBEE7A5
:10634000B083F60180E090E08217930721F4F60114
:10635000E80FF91F0CC041914032C9F30196F4CF08
:1063600080E28193CF018C199D09089768F4283049
:106370003105B0F7A5E4B0E0AC0FBD1FA20FB31F0D
:106380008C912F5F3F4FEDCFC4010E94F92D8111F9
:106390000EC0EFEF2E1A3E0A4E0A5E0AF4E62F16E2
:1063A00031044104510409F06ACF87E0D5C084303C
:1063B00009F0D2C08C85D401DF968C938C8581FF47
:1063C0000AC0C7010C966DE070E00E9458738B0103
:1063D0000F5F1F4F02C001E010E0B801C4010E942E
:1063E000BD2A8111B9C00150110909F487C0F40117
:1063F00046A157A160A571A5C801E5E0880F991FC6
:10640000EA95E1F7481B590B61097109C4010E9423
:10641000CC1D8111A1C0C6010E94C717F82E6FE0E4
:10642000562E7DE0A72EBB24B394D4019E964D91A9
:106430005D916D917C91D197C3010E94631B811185
:106440008BC0E02ED401D296ED91FC91D397D3016D
:106450001B966D917C911C97F58653861486128E3F
:10646000138E9801332721503109A29EC001A39EAB
:10647000900D11245AE1252E52E0352E20E030E017
:106480002F3FBFEF3B0749F09C01220F331F260F20
:10649000371FD9012D913C910196D1014D911D01DC
:1064A000DF01A40FB11D2C9311963C9321153105EA
:1064B00011F42FEF3FEFB7E22B16B2E03B0601F7E6
:1064C0002F3F3F4F49F0880F991FDB01A80FB91FDD
:1064D0008D919C91892B19F48E2D8064E82EE08299
:1064E000D3011396BC9260E070E0C4010E94C829F9
:1064F000811132C00150110909F097CFD4019E9645
:106500004D915D916D917C91D197C3010E94631B68
:10651000811122C040E250E060E070E0F40182A905
:1065200093A90E9487174BE050E0B601D401D296A0
:106530008D919C91D3970E94AD1AD401D296ED9182
:10654000FC91D397DF968C918871848781E0F30169
:10655000838380E001C086E0C25BDF4F0FB6F89412
:10656000DEBF0FBECDBFDF91CF911F910F91FF9086
:10657000EF90DF90CF90BF90AF909F908F907F90E3
:106580006F905F904F903F902F9008952F923F9281
:106590004F925F926F927F928F929F92AF92BF9233
:1065A000CF92DF92EF92FF920F931F93CF93DF93DF
:1065B000CDB7DEB72C970FB6F894DEBF0FBECDBFB8
:1065C0008C01DC010D90BC91A02DBC83AB83FB0141
:1065D0002E2F9F2F81918F32D9F38C35C9F3422E04
:1065E000592EF8011682178210861186168A178A8C
:1065F000108E118EF2018081803280F098012C5C27
:106600003F4F3E832D83245F3F4F38872F832B815D
:106610003C81235F3F4F3A8729878AC080E8D801B1
:10662000DF968C9340E050E0BA01C8010E94CC1D77
:10663000DDC1C114D10409F008C18E9709F405C168
:10664000929182918E9721F041E0E41AF108C1F70E
:106650004BE050E060E270E08D819E810E948717E0
:1066600058E0A52EB12C20E030E0212C46018FEF20
:10667000881A980ACC0CDD1CF301EC0DFD1D8081FD
:106680009181009709F0E5C0F80184A9853E11F4D5
:1066900085E084ABF8E0AF16B10411F4220C220CB3
:1066A000822D8C708C3009F467C1822D8370833009
:1066B00009F462C131FE64C1D801DF963C92C80181
:1066C0000E94F92DF80197AD811167C192FD8EC12D
:1066D000D801848184FF7CC1EB81FC81808184307E
:1066E00009F060C116968D919D910D90BC91A02DE1
:1066F000F801828F938FA48FB58F82859385A485AF
:10670000B58588272581822B868F978FA0A3B1A37B
:10671000EF81F88580819181A281B381F80182A304
:1067200093A3A4A3B5A3B80189859A850E94E21A10
:106730005A824982D801ED91FC9163847484E12CE2
:10674000F12CCE0101960E94511A6F3FBFEF7B07DB
:106750008B079B0709F41FC161157105E1E08E07E6
:10676000910558F0F701EE0FFF1FE60DF71D91831D
:10677000808397012F5F3F4F7901AB016032710534
:1067800058F16F32710541F16C35710529F16038AE
:10679000710558F49B01EBE1F6E04191442329F0A7
:1067A00050E042175307C9F7F6C03FEFE316F10474
:1067B00008F0F1C0F701EE0FFF1FE60DF71D718322
:1067C0006083C70101967C01BCCF2C3561F49FEF3B
:1067D000491A590A5A82498249805A80D2012C9119
:1067E0002F3299F7F4CF4032510510F0312C02C00E
:1067F000E4E03E2EF701EE0FFF1FE60DF71DE1145A
:10680000F10459F0929182918032910511F08E97A6
:1068100021F4B1E0EB1AF108F2CFF701EE0FFF1F00
:10682000E60DF71D11821082E114F10409F4B3C0E2
:10683000D301C12CD12C8D919D918032910509F00D
:10684000F8CE2FEFC21AD20AF6CF332D3360332E93
:10685000F7CE8032910539F08E32910549F48E14CD
:106860009F0409F4BDC0932D9360392E6401FECEC0
:106870002A153B0520F48E149F04F9F4ABC0ABE05D
:10688000AA16B10439F4B32DB3603B2E9BE0A92EB8
:10689000B12CFACE8E149F0439F0E32DE3603E2E26
:1068A000E814F90408F4F0CE220C220C47018BE026
:1068B000A82EB12C28E030E0D9CF8038910578F1AE
:1068C000F32DF260DF2EBC0180E090E041E653E062
:1068D0002B873C870E948E4E2B853C8587FF09C005
:1068E0008F779927FC01E656FE4F808190E03D2C82
:1068F00016C08F3F9105A1F098F0A50141505109B4
:106900002417350728F0232D2360322E9501AECFB2
:10691000F801E20FF31F94AB2F5F3F4F25C0D32C3C
:10692000009749F0E4E2F6E04191442351F050E051
:1069300048175907C9F74D2D4360D42E8FE590E0D5
:1069400013C0AC01415451094A31510518F4A22D2C
:10695000A2602A2EAC01415651094A31510520F45A
:10696000B22DB1602B2E8097F801E20FF31F84AB9C
:106970002F5F3F4F3D2C7ACF232D2260322E9ACEAF
:1069800020FE03C0332D3061332E22FE95CE432DE1
:106990004860342E91CE86E029C0843039F592FFCC
:1069A00017C024C0D80196966D917C91979771700D
:1069B000695C7F4F2B813C81620F731F0E94B81A64
:1069C000D80116966D937D938D939C931997B0CEB5
:1069D00085E00CC0BBE0AB16B10409F065CF53CF26
:1069E000EBE0AE16B10409F05FCF4DCF2C960FB699
:1069F000F894DEBF0FBECDBFDF91CF911F910F91F5
:106A0000FF90EF90DF90CF90BF90AF909F908F90CE
:106A10007F906F905F904F903F902F900895CF930D
:106A2000DF93CDB7DEB727970FB6F894DEBF0FBE62
:106A3000CDBF9C838B837E836D837A836983CE01F4
:106A400001964F830E9407184F8197FD22C0880F3F
:106A5000991FFC01E152F44F0190F081E02D309735
:106A600009F01082EB81FC81309709F01082FC0163
:106A7000E152F44F2B813C8131832083442359F030
:106A800040E0BE016D5F7F4FCE0105960E94001F62
:106A900003C08BE001C080E027960FB6F894DEBFFC
:106AA0000FBECDBFDF91CF9108952F923F924F92AD
:106AB0005F926F927F928F929F92AF92BF92CF928E
:106AC000DF92EF92FF920F931F93CF93DF93CDB797
:106AD000DEB7C655D1090FB6F894DEBF0FBECDBFE5
:106AE00029967FAF6EAF2997009709F40FC3142F33
:106AF0004C01042F0F73F02E402FBE016B5B7F4FB4
:106B0000CE01895B9F4F0E94001F811109C3279608
:106B10008EAD9FAD27979A83898329966EAD7FAD01
:106B20002997CE0101960E94C632E82F811105C037
:106B300021968FAD219787FDE6E0812F8C7109F4B6
:106B4000E8C0EE2369F0E43029F4CE0101960E94FA
:106B5000B72FE82F1F2D1860F12EEE2339F0E3C276
:106B60008D81817109F0D8C212FDD2C2F3FEDDC061
:106B70002796EEADFFAD27978081843009F071C074
:106B8000D401ED93FC93B401CF010D960E94E21A5B
:106B90002796EEADFFAD2797858596854EE150E0AF
:106BA00060E070E002960E9487172796EEADFFAD79
:106BB0002797858596854AE150E060E070E08696EB
:106BC0000E9487172796EEADFFAD27970584F685BF
:106BD000E02D80E284830E948712AB01BC012796DE
:106BE000EEADFFAD27978585968508960E945617CE
:106BF0002796EEADFFAD27970584F685E02D81E061
:106C000081A3CE0101960E94D92BE82F81118BC25E
:106C1000F4014681578160857185411551056105F3
:106C2000710509F482C000E010E09801C4010E94DF
:106C30002E25E82F27962EAD3FAD2797D401169627
:106C40004D915D916D917C91199741505109610968
:106C50007109D9011F964D935D936D937C93529763
:106C600062C06BA97CA90E94B81A2B013C010E944A
:106C70008712AB01BC018BA99CA90E960E945617E6
:106C8000EBA9FCA980E283876BA97CA920E030E016
:106C9000A90127968EAD9FAD27970E94D51AEBA923
:106CA000FCA9148E158E168E178E2796EEADFFADAD
:106CB000279781E083834114510461047104A9F191
:106CC000A3A8B4A8C5A8D6A800E010E09801B30115
:106CD000A201CE0101960E942E25E82F811123C228
:106CE000B601A50127968EAD9FAD27970E94631B25
:106CF000E82F2796AEADBFAD2797F1E04F1A5108A8
:106D0000610871081F964D925D926D927C92529728
:106D10000AC0E11108C28D8184FDFCC111FF05C0CC
:106D200080FDFAC102C0E111FEC1F3FE03C00F2DC8
:106D30000064F02E2796EEADFFAD279743A954A926
:106D400065A976A9D401D8964D935D936D937C93F4
:106D5000DB970BA91CA9DD961C930E93DC97808111
:106D6000843049F54F81588569857A855A964D93C7
:106D70005D936D937C935D974B855C856D857E857A
:106D800044278E81482B5E964D935D936D937C9343
:106D9000919725964CAD5DAD6EAD7FAD25979296E2
:106DA0004D935D936D937C939597B401CF010D96B0
:106DB0000E94E21A26C0B8010E94B81AF401668344
:106DC000778380879187C8014C960E9412178B01A8
:106DD0009C01D4011A966C931A971B961C931B97CF
:106DE0001C962C931C971D963C931D971E961C92E7
:106DF0001E971F961C921F9750961C925097519663
:106E00001C922796EEADFFAD2797D4011196FC9307
:106E1000EE938581968113969C938E931297969606
:106E2000FC92969797961C929797D4961D921D92D6
:106E30001D921C92D79798961C92989799961C929F
:106E400099979A961C929A979B961C929B979C96C0
:106E50001C929C979D961C929D979E961C929E9725
:106E60009F961C929F97F5FE59C11A967C901A978F
:106E70001B96BC916296BFAF6297D4011C96BC91E1
:106E80006396BFAF6397D4011D96BC916496BFAF64
:106E90006497D4011E96BC916596BFAF6597D401E7
:106EA0001F96BC916696BFAF6697D40150966C90C2
:106EB00050975196BC916796BFAF6797272D629602
:106EC0003FAD629763964FAD639764965FAD6497ED
:106ED00065966FAD659766967FAD6697862D9B2FFD
:106EE000A0E00E94687409F419C1D40198967C92BC
:106EF000989799963C9399979A964C939A979B96C4
:106F00005C939B979C966C939C979D967C939D9786
:106F10009E966C929E979F969C9381859285A0E009
:106F2000B0E029E0880F991FAA1FBB1F2A95D1F74F
:106F3000F40126803780408451848C019D012A967B
:106F40008FAF2A972B961FAF2B972C962FAF2C978E
:106F50002D963FAF2D97272D62963FAD6297639692
:106F60004FAD639764965FAD649765966FAD659717
:106F700066967FAD6697862D67969FAD67972A9632
:106F8000AFAC2A972B96BFAC2B972C96CFAC2C97F7
:106F90002D96DFAC2D97E12CF12C00E010E00E9443
:106FA0005F7409F008F454C0B201A101C4010E9449
:106FB000231C1B012C01623071058105910538F0FD
:106FC0006F3F7F4F8F4F9F4F21F0E0E003C0E2E023
:106FD00001C0E1E0272D62963FAD629763964FAD09
:106FE000639764965FAD649765966FAD6597669697
:106FF0007FAD6697862D67969FAD67972A96AFAC53
:107000002A972B96BFAC2B972C96CFAC2C972D960E
:10701000DFAC2D97E12CF12C00E010E00E945674BB
:10702000722E62963FAF629763964FAF63976496F6
:107030005FAF649765966FAF659766967FAF66970B
:10704000682E67969FAF6797EE2309F484CF01C03F
:10705000E0E0D401D0962D923D924D925C92D39770
:10706000E11161C0272D62963FAD6297317040E01B
:1070700050E060E070E080E090E0A0E00E94687482
:1070800009F44CC0B201A10127968EAD9FAD2797A0
:107090000E949F176B017C01672B682B692B09F4F9
:1070A00041C0272D62963FAD629763964FAD6397BF
:1070B00064965FAD649765966FAD659766967FAD94
:1070C0006697862D67969FAD679709E00E942574A5
:1070D0002A962FAF2A972B963FAF2B972C964FAF20
:1070E0002C972D965FAF2D972D960CAD1DAD2EAD27
:1070F0003FAD2D97C00ED11EE21EF31ED401D496D3
:10710000CD92DD92ED92FC92D79708C089E00FC036
:10711000E8E009C0E4E007C0E7E005C080E007C0A0
:10712000E82F01C0E2E0D4011D921C928E2FCA5AB2
:10713000DF4F0FB6F894DEBF0FBECDBFDF91CF910A
:107140001F910F91FF90EF90DF90CF90BF90AF9085
:107150009F908F907F906F905F904F903F902F9077
:1071600008952F923F924F925F926F927F928F92EB
:107170009F92AF92BF92CF92DF92EF92FF920F93C6
:107180001F93CF93DF93CDB7DEB72E970FB6F8944A
:10719000DEBF0FBECDBF4C017C876B873A013E87B7
:1071A0002D87D9011D921C92BE016F5F7F4F0E94F7
:1071B0002E18811193C1F40187A181118FC186A17D
:1071C00080FF8BC12285338544855585668577850B
:1071D00080899189A0A4B1A4C2A4D3A4E4A4F5A4F5
:1071E00006A517A50E945674F22FE32F6A017B01B2
:1071F0008C01930140E050E060E070E080E090E0BE
:10720000AF2EBE2E0E945F7409F008F4D6C0CF01E5
:10721000692E782ED2C0D4019896FC9198979996B1
:10722000EC9199979A965C909A979B96CC909B97A5
:107230009C96DC909C979D96EC909D979E96FC90DA
:107240009E979F964C903E2F31702F2F40E050E03C
:1072500060E070E080E090E0A0E00E94687409F0D7
:1072600010C13E2F452D5C2D6D2D7E2D8F2D942D23
:1072700009E00E9425742B833C834D835E836F83DA
:10728000788789879A8789819A81DC0119960D917F
:107290001C911A97015011092B813C810223132361
:1072A0000115110509F48EC0C980DA80F40140A9E6
:1072B00051A962A973A9C6010E949F1761157105A2
:1072C0008105910509F49FC01B012C01200E311E80
:1072D000411C511C7301EF2CFF24E694E114F104CE
:1072E00009F4C8C0D60119968D919C911A979701FF
:1072F000200F311F8217930718F47C01E01AF10A5E
:107300008701A20191016B857C85F60181810E9434
:10731000D414811183C0E981FA81838181118AC0EB
:10732000FE2CEE24FF0C6E187F08AD85BE858D9176
:107330009C9111978E0D9F1D8D939C93EB85FC85E1
:10734000EE0DFF1DFC87EB87970140E050E060E009
:1073500070E080E090E0D4019896AC909897999670
:10736000BC9099979A96CC909A979B96DC909B9715
:107370009C96EC909C979D96FC909D979E960C9168
:107380009E979F961C919F970E94417498962C936C
:10739000989799963C9399979A964C939A979B961F
:1073A0005C939B979C966C939C979D967C939D97E2
:1073B0009E968C939E979F969C936114710409F0FE
:1073C0002ACF89C02F2F3E2F452D5C2D6D2D7E2D70
:1073D0008F2D942DA0E00E94687441F4D40116967C
:1073E0006D917D918D919C91199708C0F40140A9F0
:1073F00051A962A973A9C4010E94231C62307105BE
:107400008105910528F482E0D40197968C9366C09B
:107410006F3FBFEF7B078B079B0721F481E0F401EF
:1074200087A35CC0D401D0966D937D938D939C937C
:10743000D3973ACF83A994A9A5A9B6A9821993098C
:10744000A409B509A70160E070E084179507A607B5
:10745000B70708F065CFBF01695C7F4F982F882779
:10746000990F40E052E02B853C85820F931F0E94CC
:10747000AD1A56CFD401D4962D923D924D925C9286
:10748000D797F40180A591A5917020E032E0281BE8
:10749000390B73012615370508F47901D401D49608
:1074A0004D915D916D917C91D79789819A810E94D0
:1074B000631B8111B3CFF40160A571A57170695C84
:1074C0007F4F89819A81680F791FA7018B859C85E1
:1074D0000E94AD1A28CF80E001C087E02E960FB63B
:1074E000F894DEBF0FBECDBFDF91CF911F910F91FA
:1074F000FF90EF90DF90CF90BF90AF909F908F90D4
:107500007F906F905F904F903F902F9008952F92B3
:107510003F924F925F926F927F928F929F92AF9223
:10752000BF92CF92DF92EF92FF920F931F93CF9370
:10753000DF93CDB7DEB767970FB6F894DEBF0FBE07
:10754000CDBF4C017C876B871A013E872D87D901FF
:107550001D921C92BE016F5F7F4F0E942E188111F9
:1075600046C2F40187A1811142C286A181FF3EC2B9
:10757000E981FA818081843009F463C1D40198964D
:107580000C91989799961C9199979A962C919A9705
:107590009B963C91C101A0E0B0E0800F911FA21F1B
:1075A000B31F80179107A207B30708F04AC118015B
:1075B0002094309446C1D4019896FC91989799965E
:1075C000EC9199979A96AC909A979B96BC909B97C2
:1075D0009C96CC909C979D96DC909D979E961C9136
:1075E0009E979F967C903E2F31702F2F40E050E069
:1075F00060E070E080E090E0A0E00E94687409F034
:10760000C6C13E2FA501B601812F972D09E00E942A
:1076100025742B833C834D835E836F8378878987B2
:107620009A8789819A81DC011996ED90FC901A97CE
:10763000B1E0EB1AF1082B813C81E222F322E11444
:10764000F10409F403C189819A81FC0103A914A9F9
:1076500025A936A9D401D4964D915D916D917C9167
:10766000D797041715072607370709F446C1E9819C
:10767000FA81FC83EB83D401D0964D915D916D919D
:107680007C91D397CF010E949F17611571058105E9
:10769000910509F410C12B013C014E0C5F1C611CCB
:1076A000711C6101CD2CDD24C694C114D10409F4F0
:1076B0002AC1EB81FC818185928596012E0D3F1DAB
:1076C0008217930718F46C01CE18DF088601A30116
:1076D00092016B857C85AB81BC8111968C910E9457
:1076E0001F158111F2C089819A81FC0143A954A917
:1076F00065A976A94419550966097709860120E02C
:1077000030E0401751076207730778F4542F44277D
:10771000550F6B857C85640F751F40E052E0C7965E
:107720000E94AD1AE981FA8113828601102F002789
:10773000110F201A310AAD85BE858D919C9111974C
:10774000800F911F8D939C93EB85FC85E00FF11FBB
:10775000FC87EB87980140E050E060E070E080E05B
:1077600090E0D4019896AC9098979996BC90999790
:107770009A96CC909A979B96DC909B979C96EC90CF
:107780009C979D96FC909D979E960C919E979F9698
:107790001C919F970E94417498962C939897999664
:1077A0003C9399979A964C939A979B965C939B9748
:1077B0009C966C939C979D967C939D979E968C939C
:1077C0009E979F969C939F971A96BC91BB83F401BA
:1077D000F385FF87D4011C96BC91B88BF401F58525
:1077E000F98BD4011E96BC91BA8BF401F785FB8B03
:1077F000D4015096BC91BC8BF401F189FD8B290119
:107800003A01B62FA72F8E8B9F8BAB80BF84C88881
:10781000D988EA88FB880C891F2F0E945F7430F496
:1078200025013601BE2DAF2D0E8BFF8BF401428654
:10783000538664867586B687A787AE89A08BBF8975
:10784000B18B2114310409F0B6CE27C02F2F3E2F63
:10785000A501B601812F972DA0E00E94687481F4E4
:10786000D40116966D917D918D919C91199761151A
:10787000710581059105D1F440E050E0BA0105C0E1
:10788000F40140A951A962A973A9C4010E941E274D
:10789000611571058105910549F4D40196968C9185
:1078A0009697806496968C9380E0A1C061307105B4
:1078B0008105910521F482E0F40187A398C06F3F10
:1078C000FFEF7F078F079F0729F481E0D401979688
:1078D0008C938DC0F40160AB71AB82AB93AB06812E
:1078E000178120853185012B022B032B09F0ABCEAC
:1078F0006683778380879187A6CE0E940F1B88239B
:1079000009F4B5CEE2CFD40198962C919897999628
:107910003C9199979A964C919A979B965C919B97DC
:107920009C966C919C979D967C919D971A96AC9095
:107930001A971B96BC901B971C96CC901C971D9673
:10794000DC901D971E96EC901E971F96FC901F973B
:1079500050960C91509751961C9151979E968C91F0
:107960009E979F969C910E945F7460F08B819C8192
:107970000E940F1B8111A9CFE981FA8143AA54AA61
:1079800065AA76AAF40144AA55AA66AA77AAD401E0
:1079900098968D919C9199979170E0E0F2E0E81BA8
:1079A000F90B8101E215F30508F48F01D401D49697
:1079B0004D915D916D917C91D79789819A810E94BB
:1079C000631B811182CFF40180A591A59170C796A8
:1079D00029813A81A8016B857C85820F931F0E94C3
:1079E000AD1AE981FA8121E02383A3CE87E067966F
:1079F0000FB6F894DEBF0FBECDBFDF91CF911F91C0
:107A00000F91FF90EF90DF90CF90BF90AF909F903D
:107A10008F907F906F905F904F903F902F90089540
:107A2000CF92DF92EF92FF920F931F93CF93DF934A
:107A300000D0CDB7DEB7FC012281338137FD31C0E4
:107A40008C01C480D5807901FFEFEF1AFF0AFC0199
:107A5000E20FF31F66838CE3E816F104CCF09E017D
:107A60002F5F3F4FA701B8016A5F7F4FF801808108
:107A700091810E94873A81E090E029813A812E1518
:107A80003F0511F480E090E0EE24FF24E81AF90AA3
:107A9000F801F382E282FFEFCF1ADF0AF801D58204
:107AA000C4820F900F90DF91CF911F910F91FF90A3
:107AB000EF90DF90CF9008950F931F93CF93DF93B4
:107AC00000D0CDB7DEB7FC014281538157FF03C020
:107AD0008FEF9FEF18C08C01BC016A5F7F4F9E0142
:107AE0002F5F3F4FFC01808191810E94873A811175
:107AF000EFCFF8012281338189819A8128173907D4
:107B000039F7848195810F900F90DF91CF911F916C
:107B10000F9108958F929F92AF92BF92EF92FF9232
:107B20000F931F93CF93DF93CDB7DEB7C654D10920
:107B30000FB6F894DEBF0FBECDBF7C01BE016B5BFC
:107B40007F4F0E942E18811125C1D70196969C91D6
:107B500096FF20C10E9487124B015C0127968EADD3
:107B60009FAD2797FC012081D701243009F0D0C0B8
:107B700015968C91833071F0F70140A951A962A943
:107B800073A90FEF1FEF9801C7010E94B12488234A
:107B900039F000C1C7010E9473268111FBC0ECCFF0
:107BA000D7018D919C9111979A8389835A968D91D3
:107BB0009D910D90BC91A02D8F839887A987BA873E
:107BC000F701068D178D20A131A10E8300270B87A9
:107BD0001C872D873E871F86188A198A1A8A1F8A52
:107BE000188E198E1A8E42A153A164A175A12596F3
:107BF0004CAF5DAF6EAF7FAF2597CE0101960E946F
:107C0000CC1D8111C7C0CE0101960E94342C811178
:107C1000C1C02796EEADFFAD2797A585B685149612
:107C20008C911497806214968C9325853685D701A4
:107C300015968C918160D90191968C93D7011696F7
:107C40004D915D916D917C91199785859685C4962E
:107C50000E945617F70102851385248535854685D0
:107C60005785608971892796EEADFFAD2797858589
:107C70009685C8960E945C17D7011A960C911A97A0
:107C80001B961C911B971C962C911C971D963C9142
:107C90001D971E964C911E971F965C911F975096AC
:107CA0006C91509751967C912796EEADFFAD27973A
:107CB0008585968588960E945C172796EEADFFAD68
:107CC000279785859685B501A4010C960E945617C5
:107CD0002796EEADFFAD2797A585B68555961C92E4
:107CE0000584F685E02D108A118A128A138ACE0146
:107CF00001960E94D92B81114DC027968EAD9FAD64
:107D000027970E94692BF70196A19F7B96A342C0FB
:107D1000D8964D915D916D917C91DB970E94631B8C
:107D2000811138C0F70104AD15ADD8011B968C91B7
:107D30001B9780621B968C932681378140855185E5
:107D4000B801808191810E94D51AF701428553853F
:107D500064857585C8014C960E945617B501A4012B
:107D6000C80146960E945617D80152961C92529707
:107D700053961C9227968EAD9FAD279721E0FC016C
:107D800023830E94692BD70196969C9196979F7B9F
:107D900096969C93CA5BDF4F0FB6F894DEBF0FBE7A
:107DA000CDBFDF91CF911F910F91FF90EF90BF90CA
:107DB000AF909F908F9008950F931F93CF93DF9371
:107DC00000D0CDB7DEB78C010E948A3D81110BC077
:107DD000BE016F5F7F4FC8010E942E18811103C042
:107DE000F801118210820F900F90DF91CF911F91B7
:107DF0000F9108952F923F924F925F926F927F92D0
:107E00008F929F92AF92BF92CF92DF92EF92FF92AA
:107E10000F931F93CF93DF93CDB7DEB7A2970FB623
:107E2000F894DEBF0FBECDBF1C010B871C872D87CA
:107E30003E874F87588B4B01BE016F5F7F4F0E947B
:107E40002E1881111CC3D10197968C91811117C3F3
:107E5000E981FA818081843041F0E981FA81FAA3D5
:107E6000E9A38081843089F42DC0D101D0964D9151
:107E70005D916D917C91D3970FEF1FEF9801C10138
:107E80000E94B124882349F3FAC22B853C854D8595
:107E90005E856F857889C4012F3F3F4F4F4F5F4FFD
:107EA000610571058105910569F060F0EFEFEB87E1
:107EB000FFEFFC870FEF0D871FEF1E871F86188AC5
:107EC000812C912CD1011A964C901A971B965C909C
:107ED0001B971C966C901C971D967C901D971E9668
:107EE000EC911E971F96FC911F975096BC91BD8BED
:107EF000D1015196BC91BE8B2B853C854D855E850D
:107F00006F857889C401520163017F010D891B2FA0
:107F10000E945F7469F060F0D10196968C9181FDAA
:107F200007C04B865C866D867E86EF87F88B48019E
:107F3000F101F0A5FB83D10199964C9099979A96FF
:107F40005C909A979B966C909B979C967C909C9744
:107F50009D96BC91BD8BF101F6A5FE8BF101B7A5F5
:107F600010A611A612A613A614A615A616A617A645
:107F70002B853C854D855E856F857889C401A0E0A1
:107F80000E94687421F4412C512C3201FEC1E9A1F8
:107F9000FAA14185528560E070E08A019B0189E089
:107FA000000F111F221F331F8A95D1F7098B1A8BDF
:107FB0002B8B3C8B2B81342D452D562D672D7D89A8
:107FC0008E899B2FA0E00E94687409F497C02989CC
:107FD0003A894B895C8959016A01E12CF12C8701AE
:107FE0002B81342D452D562DAFEF0E944A742D8BD9
:107FF0003E8B4F8B588F2B013C012B853C854D854B
:108000005E856F857889C4010E944A74AB82BC8208
:10801000CD82DE82EF82F88609871A87E12CF12C67
:1080200000E010E00E94A473298F3A8F4B8F5C8F81
:108030006D8F7E8F8F8F98A32D893E894F89588DA4
:10804000B201C3010E94A47359016A017B018C0132
:10805000298D3A8D4B8D5C8D6D8D7E8D8F8D98A188
:108060000E945F7408F44AC009891A892B893C89E7
:108070000150110921093109A02EA094B12EB0940C
:10808000C22EC094D32ED0943D89A3224E89B4220F
:108090005F89C522688DD622D1019896AC929897B7
:1080A0009996BC9299979A96CC929A979B96DC92C5
:1080B0009B979C964C929C979D965C929D979E96C2
:1080C0006C929E979F967C929F972B853C854D85C1
:1080D0005E856F857889C401720183010E945674A0
:1080E0002B873C874D875E876F87788B4C01D096B6
:1080F0004D905D906D907C90D39732C0F101468099
:10810000578060847184411451046104710419F52D
:1081100040E050E0BA01C1010E941E272B013C0142
:10812000613071058105910529F482E0D1019796AE
:108130008C93A5C16F3FBFEF7B078B079B0721F493
:1081400081E0F10187A39BC1D10116966D937D93C8
:108150008D939C931997F10140AA51AA62AA73AA20
:10816000411451046104710409F40DCF29893A893D
:108170004B895C8989019A0140E050E0BA010B8388
:108180001C832D833E834F83588769877A872B858D
:108190003C854D855E856F857889C401AB80BC8048
:1081A000CD80DE80E12CF12C00E010E00E945F74B5
:1081B00009F008F4A5C02B853C854D855E856F854B
:1081C0007889C401AB80BC80CD80DE80E12CF12CAD
:1081D00000E010E00E9456742B873C874D875E8735
:1081E0006F87788B4C019501A60160E070E080E01C
:1081F00090E0D1019896AC9098979996BC909997F9
:108200009A96CC909A979B96DC909B979C96EC9034
:108210009C979D96FC909D979E960C919E979F96FD
:108220001C910E944174298B3D8BB42FA52F698F1F
:108230007E8B8F8B9A8FF10120A731A742A753A77E
:1082400064A775A786A797A7F6A1F88FF1FF27C0A7
:10825000F101A284B384C484D584E684F7840089C0
:1082600011895A2F0E945F7471F068F0228733875A
:10827000B487A58766877787808B918BE88DE064CC
:10828000D1019696EC93B301A201C1010E941E2771
:108290002B013C01672B682B692B41F429C0B301EA
:1082A000A201C1010E94231C2B013C01BFEF4B1610
:1082B0005B066B067B0609F443CFE2E04E165104E1
:1082C0006104710408F431CFE981FA818789908DC6
:1082D000A18DB28D481659066A067B0608F025CF97
:1082E000D101D0964D925D926D927C92D3974FCFF3
:1082F0001B861C861D861E861F86188A812C912C43
:108300002B853C854D855E856F857889C401F1019B
:10831000A0A4B1A4C2A4D3A4E4A4F5A406A517A55F
:108320000E94417420A731A742A753A764A775A74D
:1083300086A797A72B853C85317040E050E060E030
:1083400070E080E090E0A0E00E94687409F41BCE29
:10835000B301A20189819A810E949F176B017C0160
:10836000672B682B692B09F4E0CE2B853C854D8566
:108370005E856F857889C40109E00E942574290112
:108380003A014C0C5D1C6E1C7F1CD1019896FC912F
:1083900098979996EC9199979A96BC91BB83D10145
:1083A0009B96BC91BB87D1019C968C909C979D9687
:1083B0009C909D979E96BC91BC87D1019F96BC9145
:1083C000BD87D1011A96AC901A971B96BC901B974B
:1083D0001C96CC901C971D96DC901D971E96EC90D9
:1083E0001E971F96FC901F9750960C915097519690
:1083F0001C9151972F2F3E2F4B815B85B4018C85AB
:108400009D850E945F74F9F0F0F01A96FC931A971C
:108410001B96EC931B971C964C931C971D965C9394
:108420001D971E968C921E971F969C921F97509692
:108430008C93509751969C93519796968C919697C2
:10844000806496968C933E2F31702F2F40E050E041
:1084500060E070E080E090E0A0E00E94687471F05D
:10846000F10184A995A9A6A9B7A9481659066A06D3
:108470007B0621F044AA55AA66AA77AA80E0A296B4
:108480000FB6F894DEBF0FBECDBFDF91CF911F9125
:108490000F91FF90EF90DF90CF90BF90AF909F90A3
:1084A0008F907F906F905F904F903F902F900895A6
:1084B0000F931F93CF93DF9300D000D0CDB7DEB7DB
:1084C0007C836B83009709F467C08C0140E0BE0198
:1084D0006F5F7F4FCE0103960E94001F811158C02D
:1084E00089819A81F801918380836B817C81C801A5
:1084F0000E94C632811156C0F80187AD87FD38C091
:10850000848184FF44C029813A81F9018081F80186
:10851000843029F586819781A085B185828F938FDC
:10852000A48FB58F428553856485758544278581E1
:10853000482B468F578F60A371A3D801A05CBF4F13
:108540008D919D910D90BC91A02D82A393A3A4A386
:10855000B5A3B801C9010D960E94E21A09C062A92B
:1085600073A90E94B81AF801668377838087918780
:10857000E981FA8185819681F8019383828340E0C5
:1085800050E0BA01C8010E94CC1D843039F485E066
:10859000F8011182108209C089E007C08111F8CF6B
:1085A00080E003C08430A1F7F2CF0F900F900F90BE
:1085B0000F90DF91CF911F910F9108950F931F930B
:1085C000CF93DF9300D0CDB7DEB78C01BE016F5FD4
:1085D0007F4F0E942E18811103C0F8011182108272
:1085E0000F900F90DF91CF911F910F910895CF922F
:1085F000DF92EF92FF921F93CF93DF9300D0CDB71E
:10860000DEB77C016B01BE016F5F7F4F0E942E18A9
:10861000182F81111EC0C114D10439F440E050E07C
:10862000BA01C7010E94CC1D13C060E070E0C70111
:108630000E94E42C982F9B7F59F4B601C7010E9439
:108640007A1860E070E0C7010E94C829843009F000
:10865000182F812F0F900F90DF91CF911F91FF90D6
:10866000EF90DF90CF900895EF92FF921F93CF93FA
:10867000DF93CDB7DEB7C654D1090FB6F894DEBF8D
:108680000FBECDBF27969FAF8EAF27977B0140E0EF
:10869000BE016F5F7F4FCE018B5B9F4F0E94001F1B
:1086A000182F81111AC027966EAD7FAD2797CE0186
:1086B00001960E94C632182F81110FC021968FADEE
:1086C000219787FD09C0E114F10439F0B701CE010B
:1086D00001960E947A1801C016E0812FCA5BDF4F15
:1086E0000FB6F894DEBF0FBECDBFDF91CF911F91C3
:1086F000FF90EF9008952F923F924F925F926F926A
:108700007F928F929F92AF92BF92CF92DF92EF9221
:10871000FF920F931F93CF93DF93CDB7DEB7E1970F
:108720000FB6F894DEBF0FBECDBF9AA789A77DA76D
:108730006CA78A0140E0BE01695D7F4FCE0189963A
:108740000E94001F8BA781111BC1EFA1F8A5D801C2
:10875000ED93FC9383899489A589B6894788508CC9
:10876000618C728C5301420122E0821A9108A108A7
:10877000B10888169906AA06BB0638F0ECA5FDA537
:1087800080839183A283B383FBC080818130B9F55C
:10879000FA83E98342E0442E512C612C712CC12CC8
:1087A000D12C7601B301A201CE0101960E94231CB7
:1087B0006F3FFFEF7F078F079F0709F4CBC0613042
:1087C00071058105910509F4C7C0672B682B692BDA
:1087D00029F42FEFC21AD20AE20AF20A8FEF481ADE
:1087E000580A680A780AEFA1F8A58789908DA18DAB
:1087F000B28D481659066A067B06A0F2B1C08430D5
:1088000009F04FC047A550A961A972A900E010E086
:10881000C12CD12C760138E0232E312C0115110505
:1088200079F42A013B019FEF491A590A690A790A2A
:108830008FA198A50E94631B811191C0B301A20171
:10884000EFA1F8A5E00FF11FE7A924013501C1014F
:10885000881999094114510461047104A9F0E0FDDB
:1088600005C0AFEFCA1ADA0AEA0AFA0AE695B1E0D9
:108870004B1A5108610871089C01240D351D232BEA
:1088800049F75301420103C0812C912C54010F5F21
:108890001F4F117081149104A104B10409F0BECFDF
:1088A0005FC083A094A0A5A0B6A000E010E0C12CFA
:1088B000D12C760101151105A9F4D501C401019649
:1088C000A11DB11D8EA79FA7A8ABB9ABB501A4018F
:1088D0008FA198A50E94631B811141C08EA49FA403
:1088E000A8A8B9A8EFA1F8A56081C801C796623011
:1088F000B1F4DF01A80FB91F11968C9190E0982F69
:108900008827E00FF11F67A9862B892B29F49FEF99
:10891000C91AD90AE90AF90A0E5F1F4F12C08E0F51
:108920009F1F0E941217DC01CB01BF70892B8A2B7D
:108930008B2B29F4AFEFCA1ADA0AEA0AFA0A0C5F9B
:108940001F4F1170B1E04B1A51086108710809F00E
:10895000B1CF06C021E001C022E02BA701C08BA748
:10896000ACA5BDA5CD92DD92ED92FC921397EFA13F
:10897000F8A5C38AD48AE58AF68A848181608483D3
:108980008BA5E1960FB6F894DEBF0FBECDBFDF9189
:10899000CF911F910F91FF90EF90DF90CF90BF90FC
:1089A000AF909F908F907F906F905F904F903F908F
:1089B0002F9008952F923F924F925F926F927F92E5
:1089C0008F929F92AF92BF92CF92DF92EF92FF92DF
:1089D0000F931F93CF93DF9300D01F92CDB7DEB7D5
:1089E0004C01BE016F5F7F4F0E942E18811185C020
:1089F000F40177A071107CC086A181FF7BC030A4F8
:108A000041A452A463A4B4A5A5A526A4F7A5FB83FD
:108A1000F401A284B384C484D584E684F7840089F5
:108A20001189232D342D452D562D6B2F7A2F822D14
:108A30009B810E945F7408F05FC0A0E00E94687490
:108A400089F4468157816085718500E010E09801C6
:108A5000C4010E942E25782EF401168217821086FA
:108A600011862FC0F40140A951A962A973A9C401BC
:108A70000E94231CAB01BC014F3FFFEF5F076F0754
:108A80007F0741F0413051056105710531F482E005
:108A9000782E17C07724739414C0E981FA818789EE
:108AA000908DA18DB28D481759076A077B0748F44E
:108AB000F40100A911A922A933A9C4010E942E25FD
:108AC000782EF40180A5828781A5838782A584877B
:108AD00083A5858784A5868785A5878786A5808BBE
:108AE00087A5818B86A1806486A3772029F077A251
:108AF000872D03C087E001C080E00F900F900F909A
:108B0000DF91CF911F910F91FF90EF90DF90CF9069
:108B1000BF90AF909F908F907F906F905F904F909D
:108B20003F902F900895CF92DF92EF92FF920F9394
:108B30001F93CF93DF93CDB7DEB7C25BD1090FB6DA
:108B4000F894DEBF0FBECDBFCF54DF4F998388832B
:108B5000C15BD04042E0BE0161557F4FCE018F54D2
:108B60009F4F0E94001F8111CEC0C155DF4F8881E9
:108B70009981CF5AD04027969FAF8EAF2797CF5479
:108B8000DF4F68817981C15BD040CE018B5B9F4F05
:108B90000E94C6328111B7C0CC57DF4F8881C458BC
:108BA000D04087FD06C02A968FAD2A9780FD88C0E9
:108BB00002C086E0A8C0C155DF4FE881F981CF5AD5
:108BC000D040C757DF4FF983E883C958D040808130
:108BD000843081F4BE0167577F4FCF010D960E940C
:108BE000E21AC157DF4FC880D980EA80FB80CF5896
:108BF000D04008C0E9966EAD7FADE9970E94B81AE3
:108C00006B017C012A968FAD2A9784FF5BC0C1550A
:108C1000DF4FE881F981CF5AD040FA83E983CF82D0
:108C2000D886E986FA8680818430B1F5CD56DF4F4B
:108C30008881C359D0408B87CC56DF4F8881C45977
:108C4000D0408C87CB56DF4F8881C559D0408D8767
:108C5000CA56DF4F8881C659D0408E87C956DF4F2C
:108C60008881C759D0408F87C856DF4F8881C8593F
:108C7000D040888BC756DF4F8881C959D040898B37
:108C8000C656DF4F8881CA59D0408A8BC257DF4F02
:108C90008881CE58D0408E8340E050E0BA01CE01AA
:108CA00001960E94CC1D81112EC060E070E0CE01C3
:108CB00001960E94E42C882319F0843019F023C017
:108CC00087E021C0CE018B5B9F4F0E940B2B81114F
:108CD0001AC0C114D104E104F10449F4C155DF4FB5
:108CE00088819981CF5AD0400E94692B0CC000E046
:108CF00010E09801B701A601CE0187579F4F0E944F
:108D00002E25882359F3CE54DF4F0FB6F894DEBFDB
:108D10000FBECDBFDF91CF911F910F91FF90EF90CC
:108D2000DF90CF9008954F925F926F927F928F92D3
:108D30009F92AF92BF92FF920F931F93CF93DF93B7
:108D4000CDB7DEB7CE56D1090FB6F894DEBF0FBE51
:108D5000CDBFAF969FAF8EAFAF9742E0BE016559D2
:108D60007F4FCE0183599F4F0E94001FF82E811123
:108D70002FC1AD968EAD9FADAD979A838983AF9687
:108D80006EAD7FADAF97CE0101960E94C6328823AB
:108D900009F41AC1843009F01AC1AD968EAD9FADA9
:108DA000AD9727969FAF8EAF279740E050E0BA016E
:108DB000CE018B5B9F4F0E941E274B015C01672BEE
:108DC000682B692B79F081E088169104A104B10425
:108DD00061F0EFEF8E169E06AE06BE0641F4FF244C
:108DE000F39405C047E0F42E02C032E0F32E0E9457
:108DF00087122B013C01F110DCC0B501A401AD9636
:108E00008EAD9FADAD970E94B226F82E8111D1C0D4
:108E1000AD968EAD9FADAD97FC012081243009F455
:108E200047C04BE050E060E270E0C7960E948717B1
:108E3000AD968EAD9FADAD971EE2FC0117ABEE5B1C
:108E4000FF4F20E12083B301A201835B9F4F0E946B
:108E50005617AD968EAD9FADAD97BC01695C7F4F47
:108E6000A50194010E94D51AAD968EAD9FADAD9728
:108E7000BC01695C7F4F40E250E0895A9F4F0E94DD
:108E8000AD1AAD968EAD9FADAD97FC01E85AFF4F80
:108E900010832F81388549855A85BC01695A7F4FD7
:108EA0000E94D51AAD96EEADFFADAD9781E08383FC
:108EB000CE0101960E94B72FF82E81117AC0AD968F
:108EC000EEADFFADAD978081843009F050C085854F
:108ED0009685B301A2010C960E945617AD96EEAD91
:108EE000FFADAD9785859685B501A401C4960E9416
:108EF0005617AD96EEADFFADAD974185528560E05A
:108F000070E099E0440F551F661F771F9A95D1F7BF
:108F100085859685C8960E945617AD96EEADFFAD35
:108F2000AD974185528560E070E029E0440F551F00
:108F3000661F771F2A95D1F78585968588960E94AA
:108F40005617AD96EEADFFADAD97A585B68583E01E
:108F500091968C930584F685E02D80E18483CE0183
:108F600001960E94D92BF82E811132C01BC08BA90B
:108F70009CA9B301A20146960E9456176BA97CA931
:108F8000A5019401AD968EAD9FADAD970E94D51A07
:108F9000EBA9FCA980E18387AD96EEADFFADAD975F
:108FA00081E08383AD968EAD9FADAD970E94692B16
:108FB0000EC000E010E09801B501A401CE018B5B6A
:108FC0009F4F0E942E2504C088E0F82E01C0F82E85
:108FD0008F2DC259DF4F0FB6F894DEBF0FBECDBF45
:108FE000DF91CF911F910F91FF90BF90AF909F9015
:108FF0008F907F906F905F904F900895DF92EF92E7
:10900000FF920F931F93CF93DF93CDB7DEB7CE5C64
:10901000D1090FB6F894DEBF0FBECDBFC553DF4FE9
:1090200099838883CB5CD040C353DF4F79836883B7
:10903000CD5CD040CE0183539F4F0E94071842E081
:10904000BE0167537F4FCE0185539F4F0E94001F83
:1090500081117BC1C753DF4F88819981C95CD040A2
:1090600027969FAF8EAF2797C553DF4F68817981D1
:10907000CB5CD040CE018B5B9F4F0E94C6328111EA
:1090800064C1CC57DF4F8881C458D040807A09F042
:1090900057C1C753DF4FE881F981C95CD040808157
:1090A000843009F08CC06585768540E450E0CE01BF
:1090B00087579F4F0E94AD1A44E450E0BE016B5B9E
:1090C0007F4FCE0101960E94AD1AC353DF4F6881D6
:1090D0007981CD5CD040CE0101960E94C6328111CB
:1090E00021C04F81588569857A852F968CAD9DADBD
:1090F000AEADBFAD2F97481759076A077B0709F038
:1091000021C14FA158A569A57AA5AF968CAD9DAD9B
:10911000AEADBFADAF97481759076A077B0709F097
:1091200011C103C0843009F010C1CE0101960E9424
:10913000B72F81110AC1C753DF4FE881F981C95C9C
:10914000D0400584F685E02DE180F3A005A110E074
:10915000102F002784A1082B40E450E0BE01675780
:109160007F4FCF010E94AD1AC753DF4FE881F981CD
:10917000C95CD0400584F685E02DE182C753DF4FFE
:10918000E881F981C95CD040A585B6859396FC92AB
:10919000A585B68594960C93949795961C93058413
:1091A000F685E02D848184FD02C080628483CE0137
:1091B00001960E94D92B882309F4B2C0C6C0E99653
:1091C0006EAD7FADE99740E250E0CE0187579F4FEB
:1091D0000E94AD1A44E450E0BE016B5B7F4FCE01AC
:1091E00001960E94AD1AC353DF4F68817981CD5C2F
:1091F000D040CE0101960E94C632811121C04F811C
:10920000588569857A852F968CAD9DADAEADBFAD85
:109210002F97481759076A077B0709F093C04FA19A
:1092200058A569A57AA5AF968CAD9DADAEADBFAD85
:10923000AF97481759076A077B0709F083C003C037
:10924000843009F082C0CE0101960E94B72F8111AF
:109250007CC00BA91CA969E870E06C0F7D1F635FDF
:109260007F4F43E150E0C8010D960E94AD1ACC56E5
:10927000DF4F8881C459D04084FF8062F801838722
:10928000C753DF4FE880F980C95CD040DD24D39418
:10929000F701D382F801838584FF42C02F964CAD3D
:1092A0005DAD6EAD7FAD2F978F819885A985BA850D
:1092B000481759076A077B0799F1B801F7018081C0
:1092C0000E94B81AAB01BC01C7010E949F17AB01F5
:1092D000BC014115510561057105B1F1C7010E943D
:1092E000631BC753DF4FE881F981C95CD04081110E
:1092F0002CC0DF01A85ABF4F8C918E3289F42F8188
:10930000388549855A85BF01695A7F4FCF010E9430
:10931000D51AC753DF4FE881F981C95CD040D382A9
:10932000CE018B5B9F4F0E940B2B81110EC0C75348
:10933000DF4F88819981C95CD0400E94692B05C0AC
:1093400086E003C088E001C082E0C253DF4F0FB661
:10935000F894DEBF0FBECDBFDF91CF911F910F916B
:10936000FF90EF90DF9008952F923F924F925F927F
:109370007F928F929F92AF92BF92CF92DF92EF92A5
:10938000FF920F931F93CF93DF93CDB7DEB7C854EF
:10939000D1090FB6F894DEBF0FBECDBF29969FAF9F
:1093A0008EAF29977B014A0140E0BE016B5B7F4F86
:1093B000CE01895B9F4F0E94001F782E8111C1C092
:1093C000E114F10409F48AC027968EAD9FAD27976A
:1093D0009A8389831F82188619861A8640E050E096
:1093E000BA01CE0101960E94CC1D811173C061E0CB
:1093F00070E0CE0101960E94E42C81116BC027968B
:10940000EEADFFAD27978081843009F04DC0C12CAF
:10941000D12C00E010E0A12CB12CEBA9FCA981819A
:1094200090E0A816B906C0F52FEFA21AB20AC5013E
:10943000880F991FE80FF91F418150E0542F4427EE
:109440008081482BC114D10429F4CA01985D81158B
:109450009840F0F060E070E0C601A0E0B0E0DC0110
:10946000992788271A012B01282A392A4A2A5B2A98
:10947000C201B10124E030E0A701400F511F0E945A
:10948000581890E0009731F0080F191F40E050E0A5
:109490006A01C3CF00E010E0CD2811F000E010E039
:1094A000F701E00FF11F19C08BA99CA9F7013B96AA
:1094B000A701DC012D91CD01DA012D93AD01AE178D
:1094C000BF07B9F71082EE15FF0541F08291803297
:1094D000C9F304C08430A1F5F7011082811491040E
:1094E00081F127968EAD9FAD2797DC015F964D9158
:1094F0005D916D917C9192970E94631B782E8111F2
:1095000020C027968EAD9FAD2797FC012081233088
:1095100029F0243031F027E230E005C023E430E0C8
:1095200002C024E630E0295C3F4F820F931F0E9467
:109530001217D4016D937D938D939C93139701C063
:10954000782E872DC85BDF4F0FB6F894DEBF0FBEB5
:10955000CDBFDF91CF911F910F91FF90EF90DF90E2
:10956000CF90BF90AF909F908F907F905F904F90E3
:109570003F902F9008958F929F92AF92BF92EF925B
:10958000FF920F931F93CF93DF93CDB7DEB7CE55E6
:10959000D1090FB6F894DEBF0FBECDBF6F969FAF57
:1095A0008EAF6F9742E0BE01655A7F4FCE01835A5E
:1095B0009F4F0E94001F81112AC16D96EEADFFAD35
:1095C0006D9780819E012B5B3F4F7901843009F0BC
:1095D00045C046E150E060E070E0C9010E94871795
:1095E00000E010E06F96EEADFFAD6F9780818032A6
:1095F00008F476C0CE01835A9F4F0E94511A61151C
:10960000710531E083079105C0F06F3FEFEF7E07F2
:109610008E079E0711F486E0FAC00A301105D8F7CC
:109620004C01AA24BB24F801EE0FFF1FEE0DFF1D15
:10963000808291820F5F1F4F05C061157105810502
:10964000910549F3AB01EFE8F1E02191222309F400
:10965000B7C030E024173507C1F7DDCF4BE050E04D
:1096600060E270E0C9010E94871700E010E06F9689
:10967000EEADFFAD6F9780818032F8F0CE01835A56
:109680009F4F0E94511A61157105F1E08F079105F6
:1096900010F60E94D64E41E653E00E948E4E00978F
:1096A00009F4B9CFE8E8F1E02191222309F496C04A
:1096B00030E028173907C1F7AECFF7018081853E2A
:1096C00009F4A9CFE00FF11F8F010E191F09EE1544
:1096D000FF0521F082918032B9F302C000E010E072
:1096E0006D968EAD9FAD6D979A8389831F82188684
:1096F00019861A8640E050E0BA01CE0101960E9418
:10970000CC1D811184C061E070E0CE0101960E9401
:10971000E42C811115C06D96EEADFFAD6D972081E3
:109720008BA99CA9243011F4FC012DC0012B21F040
:109730004BE050E0B70136C025EEFC01208334C079
:10974000843009F064C001151105C1F161E070E0D9
:10975000CE0101960E94BD2A811159C040E250E01D
:1097600060E070E08BA99CA90E9487176D96EEAD12
:10977000FFAD6D978081EBA9FCA9843061F483E88B
:109780008083EBA9FCA901838BA99CA946E150E049
:10979000B701029607C088E083874BE050E0B7012D
:1097A0008BA99CA90E94AD1A6D968EAD9FAD6D9749
:1097B00021E0FC0123830E94692B29C080E027C09F
:1097C0000B30110508F027CFF801EE0FFF1FEE0D4B
:1097D000FF1D608371830F5F1F4F04CF8F3F910583
:1097E00091F088F00A30110508F015CFF701E00F6D
:1097F000F11F90830F5F1F4FF701E00FF11F808370
:109800000F5F1F4F34CF0B301105B0F304CFC25A96
:10981000DF4F0FB6F894DEBF0FBECDBFDF91CF9103
:109820001F910F91FF90EF90BF90AF909F908F90FE
:1098300008958F929F92AF92BF92CF92DF92EF9254
:10984000FF920F931F93CF93DF9300D000D000D0EF
:10985000CDB7DEB77C014A015B0181E0A81AB108EF
:109860008701C12CD12CCA14DB04D4F49E012B5FD8
:109870003F4F41E050E0BE016F5F7F4FC4010E9447
:10988000B1388D819E81019759F489810F5F1F4FF7
:10989000F801319780839FEFC91AD90A8A3019F7E6
:1098A000F8011082CD2811F0C70102C080E090E0DD
:1098B00026960FB6F894DEBF0FBECDBFDF91CF91D5
:1098C0001F910F91FF90EF90DF90CF90BF90AF90DE
:1098D0009F908F900895EF92FF921F93CF93DF9305
:1098E000CDB7DEB7C654D1090FB6F894DEBF0FBEB0
:1098F000CDBF182F7B0146E450E060E070E0CE0160
:1099000001960E948717FA82E982612FCE010196A3
:109910000E94103DCE0101960E945C3DCA5BDF4F64
:109920000FB6F894DEBF0FBECDBFDF91CF911F9170
:10993000FF90EF900895EF92FF920F931F93CF93B4
:10994000DF93CDB7DEB7C654D1090FB6F894DEBFAA
:109950000FBECDBF7C018B0146E450E060E070E0BB
:10996000CE0101960E9487171A8309838701F801A7
:1099700061918F01CE010196662319F00E94103D7E
:10998000F6CF0E945C3DCA5BDF4F0FB6F894DEBF96
:109990000FBECDBFDF91CF911F910F91FF90EF9040
:1099A00008952F923F924F925F926F927F928F9283
:1099B0009F92AF92BF92CF92DF92EF92FF920F935E
:1099C0001F93CF93DF93CDB7DEB7CC56D1090FB637
:1099D000F894DEBF0FBECDBFCD57DF4FE880F980D2
:1099E000C358D04046E450E060E070E0CE010196FC
:1099F0000E948717CF57DF4F88819981C158D04087
:109A00009A8389836E0125E8C20ED11C1E0187E46A
:109A1000280E311CD7016C91662309F461C16532AF
:109A200021F0BFEFEB1AFB0AACC0F7011181103334
:109A300031F43396D70112961C9101E00BC0F70167
:109A40001D3219F0329600E005C03396D701129608
:109A50001C9102E01A3219F0812C912C0CC0D60115
:109A60008D909C907F01BFEFEB1AFB0A1081F601ED
:109A700032966F0114C07F0180ED810F8A3078F437
:109A80003AE0432E489CC001499C900D11244C01A2
:109A9000810E911C20E3821A91081191ECCF812F45
:109AA0008F7D8C3431F40460D7011C91F70131961D
:109AB0007F01112309F414C18FE9810F8A3118F451
:109AC00020EE210F01C0212F2F34E9F050F4233470
:109AD00009F449C0243409F45CC0223409F457C0A5
:109AE0004FC0253509F455C0283509F447C0233542
:109AF00009F046C05601F2E0AF0EB11CD6016D90E0
:109B00007C90F30102C038E045C0CF018619970967
:109B100021912111FACF6C0101FD0EC06C01BFEF44
:109B2000CB1ADB0A8815990538F460E2CE0101965C
:109B30000E94103DC601F2CFF30161913F016623FF
:109B400069F0CE0101960E94103DF6CF60E2CE0191
:109B500001960E94103DFFEFCF1ADF0AC814D90406
:109B6000A8F3650157CF560122E0A20EB11CD60121
:109B70006C91CE0101960E94103DF3CF30E10AC0F6
:109B8000612FCE0101960E94103D5601EACF32E0CE
:109B900001C03AE002FF0CC05601B4E0AB0EB11CAC
:109BA000F6016081718182819381243401F515C0B1
:109BB000C60102965C01243449F4D6018D919C9132
:109BC000BC01882777FD8095982F07C0F60180811A
:109BD0009181BC0180E090E00AC097FF08C0909599
:109BE0008095709561957F4F8F4F9F4F0860A99624
:109BF0003FAE2EAEA997C12CD12C432E512C612CF7
:109C0000712CAD964CAE5DAE6EAE7FAEAD97AD969F
:109C10002CAD3DAD4EAD5FADAD970E9480732B0175
:109C20003C01E62FCA01B901AAE04A1651046104B9
:109C3000710430F0183711F0E7E001C0E7E2E40DFD
:109C4000BFEFCB1ADB0AE05DA996AEADBFADA99719
:109C5000ED93A996BFAFAEAFA997232B242B252B4D
:109C600021F0B0E2CB16D10491F603FF09C0F10157
:109C7000EC0DFD1D2DE2422E4082C60101966C01C5
:109C800000FD03C090E2792E02C080E3782E01FD32
:109C90000EC0C6018C010F5F1F4F8815990540F457
:109CA000672DCE0101960E94103DC801F3CF8601B9
:109CB000C20CD31CD6016E916D01CE0101960E949B
:109CC000103DC214D304B1F70815190508F049CFA7
:109CD000672DCE0101960E94103D0F5F1F4FF4CFFC
:109CE000CE0101960E945C3DC459DF4F0FB6F89437
:109CF000DEBF0FBECDBFDF91CF911F910F91FF90BF
:109D0000EF90DF90CF90BF90AF909F908F907F901B
:109D10006F905F904F903F902F900895CF92DF9279
:109D2000EF92FF92603871058105910510F4CB0127
:109D300023C06115710521E082079105D8F44136F1
:109D40005340C1F4E5EDF4E020E030E0C190D19063
:109D5000E12CF12C6C157D058E059F0529F02F5FF8
:109D60003F4F2038310591F7B90160587F4FCB0143
:109D7000992702C080E090E0FF90EF90DF90CF90B5
:109D800008958038910588F06136734061F48F3F03
:109D9000910509F040F4880F991FFC01EB52FC4F2C
:109DA00080819181089580E090E00895CF93DF93C2
:109DB0006115710521E08207910508F058C0EB019B
:109DC000611570418105910518F0A7E2B2E002C06B
:109DD000A3EEB2E04D915C9111974115510509F444
:109DE00043C0C417D50708F43FC01496FD0132974D
:109DF00020813181E32FFF273327B901640F751FBD
:109E0000C617D70748F5E930F10570F5EB5AFF4F53
:109E10000C940174CE01841B950B880F991FA80F19
:109E2000B91FCD91DC9120C09E01241B350B217000
:109E30003327C21BD30B18C0609716C0A09714C05D
:109E4000E09712C06A9710C028960EC0C055D1097D
:109E50000BC0C056DC4108C0EF2B09F0BBCF220F6E
:109E6000331FA20FB31FB6CFBE0180E090E0DF9199
:109E7000CF9108958F929F92AF92BF92CF92DF922F
:109E8000EF92FF920F931F939B01AC018FB7F89451
:109E9000C0903617D0903717E0903817F0903917E8
:109EA0008FBFA5E0B0E00E9441732FB7F894809077
:109EB000361790903717A0903817B09039172FBFEA
:109EC000950184010C191D092E093F090617170772
:109ED0002807390750F31F910F91FF90EF90DF9003
:109EE000CF90BF90AF909F908F90089581B1877E63
:109EF00081B9149A039B5EC004995CC080E00E9403
:109F0000CC0868EC70E080E090E00E943A4F8FE16E
:109F100092E09F938F930E94A7768BE296E00E9437
:109F2000BB7664E670E080E090E00E943A4F8CE3FC
:109F300096E00E94BB7664E670E080E090E00E94CC
:109F40003A4F85E596E00E94BB7664E670E080E0DB
:109F500090E00E943A4F8CE696E00E94BB7664E661
:109F600070E080E090E00E943A4F85E896E00E9421
:109F7000BB7664E670E080E090E00E943A4F85E9AD
:109F800096E00E94BB7664E670E080E090E00E947C
:109F90003A4F89EA96E00E94BB7664E670E080E082
:109FA00090E00E943A4F0B9A139881E08093E10B66
:109FB0000F900F9008958091E10B08958FB7F8945A
:109FC00040913617509137176091381770913917B3
:109FD0008FBF2FB7F8948091361790913717A091C3
:109FE0003817B09139172FBF841B950BA60BB70BF1
:109FF000843F9140A105B10560F308950D9880B1AB
:10A0000085FB882780F90895159A08951598089575
:10A01000809102010895CF93DF93CDB7DEB72C97DF
:10A020000FB6F894DEBF0FBECDBF8091000C90E05C
:10A030008C599F4F98878F838091131881508E83FE
:10A04000809112188C8380912C188B8380914F17EC
:10A050008A838091271789838FEF9FEF9C878B8757
:10A06000CE0101960E94EC6B2FB7F89460937117A4
:10A070007093721780937317909374172FBF81E0BA
:10A080008093010C2C960FB6F894DEBF0FBECDBFA7
:10A09000DF91CF9108958091020181110C940450B9
:10A0A0000C9406509F938F93809176179091771719
:10A0B0000E969F938F930E9452760F900F900F9061
:10A0C0000F900895CF93909377178093761780E839
:10A0D000EFEEFCE1DF01982F1D929A95E9F7EFE68C
:10A0E000FDE1DF011D928A95E9F710924917109260
:10A0F0004A1710924B1710924C171092601710923B
:10A100006117109262171092631710923D17109208
:10A110003E1710923F17109240171092010C0E94A8
:10A12000FE4F882359F1C1E0C093E30B0D9A809153
:10A13000751781508230E8F481E00E94CC080E94BB
:10A14000DE4F81E792E00E9452500E94DE4F81E094
:10A150000E944E090E94DE4F86E592E00E94525016
:10A1600082E292E00E945250C0930201CF910C947F
:10A17000045010920201CF910C9406501092E30B00
:10A1800010920201CF910895803350F08A3310F479
:10A19000805308959FEB980F963010F487530895DD
:10A1A00080E008952F923F924F925F926F927F923C
:10A1B0008F929F92AF92BF92CF92DF92EF92FF92D7
:10A1C0000F931F93CF93DF93CDB7DEB76F970FB683
:10A1D000F894DEBF0FBECDBF082F809141178130AC
:10A1E00071F48FE69DE19F938F938EEA96E09F93A3
:10A1F0008F930E94A7760F900F900F900F908091F1
:10A200004117823031F4602F70E08FE69DE10E94AB
:10A210007A6A053008F4E0C210E0680124E0C21A4E
:10A22000D108F601E159F24E80818A3209F0D4C298
:10A230000159124EF801339780810E94C45030E1D9
:10A24000839F70011124F801329780810E94C450CD
:10A25000F701E80FF11DCF0141E0242F30E02C156C
:10A260003D053CF4F901E159F24E208182274F5F10
:10A27000F4CF892B09F0B0C263EB76E08FE69DE165
:10A280000E94F275892B09F4D4C16CE270E08FE66C
:10A290009DE10E94DC756CE270E001960E94DC7525
:10A2A000FC0181818D8B82818E8B1F8A83818A8BB9
:10A2B00084818B8B1C8A86818E8387818F838085A6
:10A2C0008887818589871A866CE270E0CF010196C4
:10A2D0000E94DC75FC01F181F88F6CE270E0019660
:10A2E0000E94DC75FC0181818B8782818C87838150
:10A2F0008D871E8684818F878581888B198A8781C7
:10A30000898380858A8381858B8382858C831D8266
:10A310006CE270E0CF0101960E94DC75FC01F181D6
:10A32000F98F6CE270E001960E94DC7501969B8FBC
:10A330008A8F0E94D2748150863020F481E080930D
:10A34000B51A02C01092B51A8091B51A882309F483
:10A3500070C1CE0145960E94D2748C0190934E1725
:10A3600080934D17CE0142960E94D2749D8F8C8FA0
:10A370009093A11A8093A01ACE0106960E94D274DF
:10A38000BC01882777FD8095982F0E94397220E0C4
:10A3900030E44CE156E40E94967120E030E040E762
:10A3A00052E40E94C5722B013C01609364177093C4
:10A3B00065178093661790936717CE010B960E94DE
:10A3C000D2741C0190935F1780935E17CE010F9695
:10A3D0000E94D2749F8F8E8F90935D1780935C172D
:10A3E000CE0101960E94D274BC01882777FD80952A
:10A3F000982F0E94397220E030E44CE156E40E942C
:10A40000967120E030E040E752E40E94C5724B01B3
:10A410005C0160935417709355178093561790936F
:10A420005717B801882777FD8095982F0E943972B9
:10A430006B017C012C8D3D8DB901882777FD8095BE
:10A44000982F0E94397220E030E040E752E40E94E9
:10A4500096719B01AC01C701B6010E942A716B0184
:10A460007C0120E030E041E655E4C301B2010E94E6
:10A4700096719B01AC01C701B6010E942A716093DD
:10A48000691770936A1780936B1790936C17B101DB
:10A49000882777FD8095982F0E9439722B013C0107
:10A4A000EE8DFF8DBF01882777FD8095982F0E9444
:10A4B000397220E030E040E752E40E9496719B013F
:10A4C000AC01C301B2010E942A712B013C0120E0C2
:10A4D00030E041E655E4C501B4010E9496719B014C
:10A4E000AC01C301B2010E942A7160936D17709391
:10A4F0006E1780936F17909370176CE270E08A8DDF
:10A500009B8D0E94DC758C010F5F1F4FC8010E945C
:10A51000D2748093A21A6CE270E0C8010E94DC75CC
:10A520008C010F5F1F4FC8010E94CE7460932118E9
:10A530007093221880932318909324186CE270E093
:10A54000C8010E94DC758C010F5F1F4FC8010E947B
:10A55000CE746093311770933217809333179093B2
:10A5600034176CE270E0C8010E94DC756CE270E0A8
:10A5700001960E94DC7501960E94CE746093431789
:10A580007093441780934517909346172091311785
:10A590003091321740913317509134170E942A712D
:10A5A00060935017709351178093521790935317DD
:10A5B000F88DF0933517298D209325186091691730
:10A5C00070916A1780916B1790916C17FE3429F087
:10A5D00020E030E040E85FEB04C020E030E040E8FD
:10A5E0005FE30E94C5726093691770936A17809346
:10A5F0006B1790936C1760916D1770916E17809127
:10A600006F1790917017398D353429F020E030E0C4
:10A6100040E85FEB04C020E030E040E85FE30E94E8
:10A62000C57260936D1770936E1780936F17909338
:10A6300070176AEB76E08FE69DE10E94F275892B38
:10A6400009F4CAC08091B51A882309F4B5C06CE238
:10A6500070E08FE69DE10E94DC758C010F5F1F4F5B
:10A660008091010C811108C0C8010E94CE740E9423
:10A6700008722B013C0103C0412C512C32016CE2C9
:10A6800070E0C8010E94DC756CE270E001960E94E7
:10A69000DC756CE270E001960E94DC756CE270E0A3
:10A6A00001960E94DC756CE270E001960E94DC75F8
:10A6B0006CE270E001960E94DC758C010F5F1F4F09
:10A6C000C8010E94CE746093491770934A17809313
:10A6D0004B1790934C1726E53EE04DEE5FE30E944A
:10A6E000C57260936017709361178093621790939F
:10A6F00063176CE270E0C8010E94DC758C010F5F8B
:10A700001F4FC8010E94CE7460933D1770933E178F
:10A7100080933F17909340176CE270E0C8010E944D
:10A72000DC752091010C211108C001960E94CE74A5
:10A730000E9408724B015C0103C0812C912C5401D2
:10A740008091010C811148C0C301B20120E137E2C0
:10A7500040E050E00E94807320932C1824E6C22E23
:10A76000D12CE12CF12CA70196010E94807320933B
:10A770004F17C301B201A70196010E948073609335
:10A780002717C501B40120E137E240E050E00E9404
:10A79000807320931218A70196010E948073209362
:10A7A0001318C501B401A70196010E94807360933C
:10A7B000000C0E940B5010C01092491710924A17BB
:10A7C00010924B1710924C1710926017109261174D
:10A7D00010926217109263176F960FB6F894DEBF4F
:10A7E0000FBECDBFDF91CF911F910F91FF90EF90E2
:10A7F000DF90CF90BF90AF909F908F907F906F90A1
:10A800005F904F903F902F900895CF938A3001F53D
:10A81000EFEEFCE1AFE6BDE18DE1EF36F80719F0B0
:10A8200081918D93F9CFC0E8EFEEFCE1DF018C2F31
:10A830001D928A95E9F78091E20B0E94D250EFE6D3
:10A84000FDE1DF011D92CA95E9F71092E20B0CC001
:10A85000E091E20BE7FD08C091E09E0F9093E20BC0
:10A86000F0E0E151F34E8083CF9108954FB7F89413
:10A87000209123113091241180912511909126115E
:10A880004FBF2817390711F19FB7F894E0912311B2
:10A89000F09124112091211130912211E217F30738
:10A8A00029F420911F113091201107C0E09123114C
:10A8B000F09124119F012F5F3F4F3093241120937B
:10A8C000231180819FBF0E940554D0CF0895EF923D
:10A8D000FF920F931F93CF93DF931F92CDB7DEB7F5
:10A8E00085E1E82EF12C8091EA0B811129C09FB7F8
:10A8F000F89400913617109137172091381730913E
:10A9000039179FBF9FB7F89440913617509137176A
:10A9100060913817709139179FBF401B510B620B24
:10A92000730B443F51406105710560F389830E94B8
:10A930003A1291E0E91AF1088981E114F10499F6DB
:10A940000F90DF91CF911F910F91FF90EF9008959D
:10A95000EF92FF920F931F937B0123E0EE0CFF1CFD
:10A960002A95E1F700E010E09C0140E850E062E544
:10A970007EE185EA9AE10E94635B1F910F91FF904F
:10A98000EF9008958091EA0B089562E57EE182E6FA
:10A990009EE10E94875880E1E4EFFDE1A4E0BEE182
:10A9A00001900D928A95E1F70895CF93DF93EC0122
:10A9B000A4E0BEE1FC019C01205F3F4F8D9190819E
:10A9C00089278193E217F307C9F7BE0182E69EE16A
:10A9D0000E94C75980E1FE01A4E0BEE101900D9202
:10A9E0008A95E1F7DF91CF9108950F931F93CF934D
:10A9F000DF93CDB7DEB760970FB6F894DEBF0FBE1A
:10AA0000CDBF8C0180E1F801DE01119601900D921D
:10AA10008A95E1F7B80182E69EE10E94E05AE4E0FF
:10AA2000FEE1D8019801205F3F4F81919C918927D9
:10AA30008D93A217B307C9F780E1FE013196A4E018
:10AA4000BEE101900D928A95E1F760960FB6F894F9
:10AA5000DEBF0FBECDBFDF91CF911F910F91089543
:10AA60001F93CF93DF9300D0CDB7DEB70E940612BD
:10AA7000182F882309F476C041E061EC76E084E188
:10AA80009EE10E9455358093EF1D8430D9F584E115
:10AA90009EE10E94DC3E46E061EC76E084E19EE1CE
:10AAA0000E9455358093EF1D811123C01092E60B53
:10AAB0001092E70B1092E80B1092E90B1092121F04
:10AAC0001092131F1092141F1092151F1A821982D0
:10AAD0009E012F5F3F4F44E050E062E17FE184E15F
:10AAE0009EE10E94873A8093EF1D84E19EE10E94DF
:10AAF000DC3E41E061EC76E084E19EE10E94553568
:10AB00008093EF1D8091EF1D81112CC01A82198254
:10AB10009E012F5F3F4F44E050E062E17FE184E11E
:10AB20009EE10E94B1388093EF1D84E19EE10E9476
:10AB3000DC3E8091EF1D811115C089819A810497B7
:10AB400089F48091121F9091131FA091141FB0914E
:10AB5000151F8093E60B9093E70BA093E80BB0933F
:10AB6000E90B05C084E19EE10E94DC3E10E0812FEC
:10AB70000F900F90DF91CF911F910895CF93DF93A6
:10AB800000D0CDB7DEB742E061EC76E084E19EE133
:10AB90000E9455358093EF1D811138C08091E60BDE
:10ABA0009091E70BA091E80BB091E90B0496A11DE1
:10ABB000B11D8093E60B9093E70BA093E80BB09345
:10ABC000E90B8093121F9093131FA093141FB0934F
:10ABD000151F1A8219829E012F5F3F4F44E050E0FB
:10ABE00062E17FE184E19EE10E94873A8093EF1D5C
:10ABF00084E19EE10E94DC3E8091EF1D811106C040
:10AC000089819A81049711F481E001C080E00F905E
:10AC10000F90DF91CF9108952F923F924F925F92C4
:10AC20006F927F928F929F92AF92BF92CF92DF925C
:10AC3000EF92FF920F931F93CF93DF9300D01F9259
:10AC4000CDB7DEB70E940612882309F484C00E94A3
:10AC5000BE558B83882309F47EC041E069ED76E020
:10AC600084E19EE10E9455358093EF1D811173C0F0
:10AC700040901E1E50901F1E6090201E7090211E3E
:10AC80004091E60B5091E70B6091E80B7091E90B56
:10AC90008A019B0140E050E060E070E084E19EE1C9
:10ACA0000E94FA3E8093EF1D81114FC0D301C20173
:10ACB0000497A109B1091C012D0120913C1E30917E
:10ACC0003D1E40913E1E50913F1E6091401E70916E
:10ACD000411E8091421E9091431E51016201E12C60
:10ACE000F12C00E010E00E945F7478F51A8219825E
:10ACF0009E012F5F3F4F44E050E062E17FE184E13D
:10AD00009EE10E94B1388093EF1D84E19EE10E9494
:10AD1000DC3E8091EF1D81111EC06091121F709169
:10AD2000131F8091141F9091151F6093F01D709355
:10AD3000F11D8093F21D9093F31D0E94C57481E074
:10AD40008093E50B1092E40B0BC084E19EE10E941E
:10AD5000DC3E0E94DA1084E19EE10E94DC3E1B8210
:10AD60008B810F900F900F90DF91CF911F910F91DA
:10AD7000FF90EF90DF90CF90BF90AF909F908F901B
:10AD80007F906F905F904F903F902F900895CF935A
:10AD90000E940612C82F811102C0C0E00FC041E01E
:10ADA00062EF76E084E19EE10E9455358093EF1DCD
:10ADB0008111F3CF84E19EE10E94DC3E8C2FCF9184
:10ADC00008951F93CF93DF9300D0CDB7DEB70E94D5
:10ADD0000612182F882389F141E06BE077E084E1C7
:10ADE0009EE10E9455358093EF1D811126C01A8285
:10ADF00019829E012F5F3F4F40E150E062E17FE109
:10AE000084E19EE10E94B1388093EF1D84E19EE1D0
:10AE10000E94DC3E8091EF1D81110FC089819A81D3
:10AE2000409759F4A2E5BEE1E2E1FFE180E18E0F37
:10AE300091919D938E13FCCF01C010E0812F0F9054
:10AE40000F90DF91CF911F9108951092EA0B0E940D
:10AE5000C756882331F0809126188823F1F00C948E
:10AE600006070E94E156882369F00E943055882326
:10AE700049F00E940C56882329F00E94F40681E0D4
:10AE80008093EA0B80912618882339F08091EA0B91
:10AE900081110C9499100C94DA1008950F931F935C
:10AEA000CF93DF931091E50B112389F0C4EFDDE11F
:10AEB0000C2F005F0E94C17469930C13FBCF90911B
:10AEC000E40B9F5F9093E40B97FD0E940C56812F3B
:10AED000DF91CF911F910F91089584EF9DE1089527
:10AEE00080E1E5EAFAE1A4EFBDE101900D928A95D7
:10AEF000E1F70895FC018081918190839281918393
:10AF000093819283838308954F925F926F927F9291
:10AF10009F92AF92BF92CF92DF92EF92FF920F93E8
:10AF20001F93CF93DF9300D000D0CDB7DEB78C0155
:10AF3000D62EBA01C22EE22EF12C5701AA0CBB1C50
:10AF4000AA0CBB1CA5010E94D375A00EB11EF50171
:10AF5000349780819181A281B38189839A83AB8365
:10AF6000BC832C2DBC2CA12CBD1408F0B2C02C111C
:10AF700045C0CE0101960E947A5749805A806B8065
:10AF80007C80872D9927AA27BB27FC01EB57FC4F14
:10AF90002491462D50E0FA01EB57FC4F4491852D4A
:10AFA00090E0FC01EB57FC4F8491552466247724F4
:10AFB000F201EB57FC4F449050E060E070E0BA01C2
:10AFC00055274427722B442990E0F82FEE27CF0114
:10AFD000AA2797FDA095BA2F482B592B6A2B7B2BBC
:10AFE00049835A836B837C83EA2DF0E0EB52FA4F5E
:10AFF000E081E427E983A39420E042C0243009F0F3
:10B000003FC048E0C4123CC089819A81AB81BC81B9
:10B010004B2F552766277727FA01EB57FC4F3491C2
:10B020004A2F50E0FA01EB57FC4F4490492F50E073
:10B03000FA01EB57FC4F94909927AA27BB27FC01F4
:10B04000EB57FC4F8491512C612C712C320155240B
:10B050004424732AB301A201482BDB01CA01492D04
:10B0600050E0F42FEE27AF01662757FD6095762F4D
:10B07000842B952BA62BB72B89839A83AB83BC8318
:10B080008B2D90E0FC01EE19FF09EE0FFF1FEE0F74
:10B09000FF1FE00FF11F4080518062807380498163
:10B0A0005A816B817C814425552566257725498306
:10B0B0005A836B837C83880F991F880F991FF8012F
:10B0C000E80FF91F4083518362837383B3942F5F2A
:10B0D0004BCF0F900F900F900F90DF91CF911F915A
:10B0E0000F91FF90EF90DF90CF90BF90AF909F9027
:10B0F0007F906F905F904F900895AB0128E06CE3D4
:10B100000C948457AB0126E064E30C948457AB01A4
:10B1100024E06CE20C9484579C0190E1915050F033
:10B12000D901A90FB11DEC91F0E0EB57FC4FE49170
:10B13000EC93F4CF08959C0190E1915050F0D90127
:10B14000A90FB11DEC91F0E0EB57FD4FE491EC93AA
:10B15000F4CF0895FC018181958191839185958338
:10B160009585918785878281928592838287868162
:10B170009685968386878381978593839385978722
:10B180009781938787830895FC01838197819383B7
:10B19000938597839785938787878281928592830A
:10B1A000828786819685968386878181958591831E
:10B1B0009185958795819187858308958F929F9238
:10B1C000BF92CF92DF92EF92FF920F931F93CF9394
:10B1D000DF93BC0184E0D82EDA94BFEFDB1609F4CC
:10B1E0004FC084E0D89EF00111247B01EE0EFF1EBB
:10B1F000D7011C91512F550F550B5B71912F990F52
:10B200005927EF012196C60FD71F0881402F440F01
:10B21000440B4B71202F220F4227DF011296A60FFD
:10B22000B71F2C91C22EC02633964F01860E971E53
:10B23000F4013081922F990F990B9B71822F880F07
:10B240009827832F880F880B8B71B32EBB0C8B250F
:10B25000BC2CB326B526B426F701B08223272127BC
:10B26000422749274883202F21273227392738278B
:10B270003C939C2D912795278927D4018C93ACCFA3
:10B28000DF91CF911F910F91FF90EF90DF90CF90C2
:10B29000BF909F908F900895CF92DF92EF92FF9290
:10B2A0000F931F93CF93DF93DC01EB0194E0915058
:10B2B000E8F084E0989F900111248D01020F131F84
:10B2C0002C0F3D1FF801C080D180E280F380F9018E
:10B2D00040815181628173814C255D256E257F25DA
:10B2E000F8014083518362837383E1CFDF91CF9173
:10B2F0001F910F91FF90EF90DF90CF900895CF9224
:10B30000DF92EF92FF920F931F93CF93DF938C0105
:10B31000EB01C42EBC01CE010E944C59EE24E394F3
:10B32000F12CCE01EC14B8F40E948C58CE010E948E
:10B33000AA58CE010E94DE58B70184E0660F771F3D
:10B340008A95E1F7600F711FCE010E944C598FEF73
:10B35000E81AF80AE6CF0E948C58CE010E94AA583B
:10B36000B80180E1E89E600D711D1124CE01DF91CE
:10B37000CF911F910F91FF90EF90DF90CF900C94A1
:10B380004C594EE00C947F594CE00C947F594AE0A4
:10B390000C947F5920E0882369F0982F9170919543
:10B3A00096232927962F990F990B9B71660F692772
:10B3B0008695F1CF822F08953F924F925F926F92C0
:10B3C0007F928F929F92AF92BF92CF92DF92EF9235
:10B3D000FF920F931F93CF93DF9300D000D01F9263
:10B3E000CDB7DEB77C0194E0915008F484C084E0CE
:10B3F000989F900111243B832A8349018E0C9F1C46
:10B40000F4011081612F8EE09D830E94CA59382E6D
:10B41000AA80BB80FFEFAF1ABF0AAE0CBF1CF501BC
:10B420005080652D8BE00E94CA593826CA80DB8087
:10B43000F2E0CF0ED11CCE0CDF1CF6016080662D31
:10B440008DE00E94CA5938262A813B812D5F3F4FEB
:10B450002E0D3F1DF9017080672D89E029833C8303
:10B460000E94CA593826612F89E00E94CA59482E85
:10B47000652D8EE00E94CA594826662D8BE00E94F9
:10B48000CA594826672D8DE00E94CA594826612F67
:10B490008DE00E94CA59082F652D89E00E94CA5983
:10B4A0000827662D8EE00E94CA590827672D8BE079
:10B4B0000E94CA590827612F8BE00E94CA59182F91
:10B4C000652D8DE00E94CA591827662D89E00E94DB
:10B4D000CA591827672D8EE00E94CA59F40130829C
:10B4E000F5014082F6010083812729813C81F90121
:10B4F00080839D8179CF0F900F900F900F900F90C8
:10B50000DF91CF911F910F91FF90EF90DF90CF903F
:10B51000BF90AF909F908F907F906F905F904F9073
:10B520003F900895BF92CF92DF92EF92FF920F93D8
:10B530001F93CF93DF937C01EB01B42EC42ED12C4B
:10B54000BC0180E1489F600D711D1124CE010E9455
:10B550004C5900E010E00F5F1F4FCE010B15C0F4F7
:10B560000E94C458CE010E949B58B601601B710B0B
:10B570009B0184E0220F331F8A95E1F7B701620F28
:10B58000731FCE010E944C59CE010E94DC59E3CFBB
:10B590000E94C458CE010E949B58B701CE01DF9192
:10B5A000CF911F910F91FF90EF90DF90CF90BF90C0
:10B5B0000C944C594EE00C94925A4CE00C94925AD4
:10B5C0004AE00C94925ABF92CF92DF92EF92FF9290
:10B5D0000F931F93CF93DF93CDB7DEB7C054D1093C
:10B5E0000FB6F894DEBF0FBECDBF7C018E010F5F9A
:10B5F0001F4F80E4F80111928A95E9F74130F2E09B
:10B600005F0738F09A0140E050E0C8010E940560F1
:10B610000AC0495F5F4F93E0569547959A95E1F7C9
:10B62000C8010E94D3756801F80196E380E4B82E42
:10B63000B00E808189278193BE12FBCFC7010E9483
:10B640009A5DB801C7010E94C05D9AE6F60180814B
:10B65000892781936F01BE12F9CFF4E1EF0EF11C3F
:10B66000C7010E949A5DB801C7010E94C05DC05C1D
:10B67000DF4F0FB6F894DEBF0FBECDBFDF91CF9185
:10B680001F910F91FF90EF90DF90CF90BF900895A2
:10B690000C94C05D0C94485F0F931F93CF93DF937E
:10B6A0008C01EB010E94FD5F649640E850E0B80118
:10B6B000CE010E94485FBE01C801DF91CF911F916A
:10B6C0000F910C94FD5F2F923F924F925F926F9279
:10B6D0007F928F929F92AF92BF92CF92DF92EF9222
:10B6E000FF920F931F93CF93DF93CDB7DEB7C7556C
:10B6F000D1090FB6F894DEBF0FBECDBF5C01490182
:10B70000170128018E010F5F1F4F80E4F80111928D
:10B710008A95E9F74130F2E05F0738F09A0140E09E
:10B7200050E0C8010E9405600AC0495F5F4FE3E036
:10B7300056954795EA95E1F7C8010E94D37567963B
:10B740001FAF0EAF6797F80196E320E4200F6896CD
:10B750002FAF689780818927819368962FAD68976E
:10B760002E13F8CFCE018F5B9F4F0E949A5DB801D8
:10B77000CE018F5B9F4F0E94C05D72016101340159
:10B78000C114F2E0DF06E104F10470F0B301CE0170
:10B790008F5B9F4F0E94C05D80E4680E711CE2E0E9
:10B7A000DE1AE108F108ECCFB201A1015170662761
:10B7B0007727D201C10129E0B695A795979587957E
:10B7C0002A95D1F71C0136E0220C331C3A95E1F79B
:10B7D000280C391CB101CE018F5B9F4F0E94485F3E
:10B7E0009AE66796EEADFFAD6797808189278193D2
:10B7F0006796FFAFEEAF679768962FAD68972E13E9
:10B80000F0CFBE016F5B7F4FC5010E94FD5FCE018F
:10B810008F5B9F4F0E949A5DB801CE018F5B9F4F57
:10B820000E94C05D40E850E0B501CE018F5B9F4FA4
:10B830000E94485FBE016F5B7F4FC5010E94FD5FA4
:10B84000C95ADF4F0FB6F894DEBF0FBECDBFDF91F0
:10B85000CF911F910F91FF90EF90DF90CF90BF900D
:10B86000AF909F908F907F906F905F904F903F90A0
:10B870002F9008958F929F92AF92BF92CF92DF92B6
:10B88000EF92FF920F931F934B015C018094909471
:10B89000A094B09467017801C820D920EA20FB2049
:10B8A000DC01CB0182239323A423B523BC01CD016A
:10B8B0006C297D298E299F291F910F91FF90EF9070
:10B8C000DF90CF90BF90AF909F908F9008958F9210
:10B8D0009F92AF92BF92EF92FF920F931F934701F7
:10B8E000580180949094A094B09482229322A42230
:10B8F000B522DC01CB018E219F21A023B123BC0105
:10B90000CD01682979298A299B291F910F91FF90E0
:10B91000EF90BF90AF909F908F900895AF92BF929D
:10B92000CF92DF92EF92FF920F931F9359016A011A
:10B93000AE24BF24C026D1266A257B258C259D25D3
:10B940001F910F91FF90EF90DF90CF90BF90AF903D
:10B950000895CF92DF92EF92FF920F931F936701AA
:10B960007801C094D094E094F094DC01CB018C2950
:10B970009D29AE29BF29BC01CD01622773278427E9
:10B9800095271F910F91FF90EF90DF90CF90089532
:10B990002F923F924F925F926F927F928F929F92DF
:10B9A000AF92BF92CF92DF92EF92FF920F931F93CD
:10B9B000CF93DF93CDB7DEB72C970FB6F894DEBFE9
:10B9C0000FBECDBF4B01C22E0987DE2C28E0EFED64
:10B9D000F5E0DE01119601900D922A95E1F7437092
:10B9E000642F70E01C0124E0429F200C311C1124C4
:10B9F000D1014D905D906D907C905B01BFEFAB1AD3
:10BA0000BB0AE3E0AE22BB24AA0CBB1CAA0CBB1CE5
:10BA1000A80EB91EFB013396E370FF27EE0FFF1F40
:10BA2000EE0FFF1FE80FF91FE080F1800281138104
:10BA30006E5F7F4F63707727660F771F660F771FE4
:10BA4000FC01E60FF71F2081318142815381D5012E
:10BA50006D917D918D919C91FE013196ED0DF11DC1
:10BA6000ED0DF11D0190F081E02D09952985B4E0DF
:10BA70002B9FF0011124EB57FB4F259135914591F8
:10BA8000549129873A874B875C87D4010D911D918A
:10BA90002D913C91400E511E621E731E460E571E84
:10BAA000681E791E29853A854B855C85420E531E9A
:10BAB000641E751EB301A2010C2C04C0440F551F57
:10BAC000661F771F0A94D2F78C2D81958F7104C061
:10BAD00076946794579447948A95D2F7442A552AC6
:10BAE000662A772AF50180819181A281B381480E6F
:10BAF000591E6A1E7B1ED1014D925D926D927C9201
:10BB000013972C960FB6F894DEBF0FBECDBFDF9112
:10BB1000CF911F910F91FF90EF90DF90CF90BF904A
:10BB2000AF909F908F907F906F905F904F903F90DD
:10BB30002F900895FC01108A118A128A138A81E0DD
:10BB400093E2A5E4B7E680839183A283B38389E877
:10BB50009BEAADECBFEE84839583A683B7838EEF1B
:10BB60009CEDAAEBB8E980879187A287B38786E727
:10BB700094E5A2E3B0E184879587A687B787089507
:10BB80002F923F924F925F926F927F928F929F92ED
:10BB9000AF92BF92CF92DF92EF92FF920F931F93DB
:10BBA000CF93DF93CDB7DEB7A1970FB6F894DEBF82
:10BBB0000FBECDBF6C015B01FC0180819181A28130
:10BBC000B38189839A83AB83BC8384819581A68169
:10BBD000B7818D839E83AF83B88780859185A28549
:10BBE000B38589879A87AB87BC8784859585A68529
:10BBF000B7858D879E87AF87B88B87E08D8F8CE068
:10BC00008E8F81E18F8F86E188A32E01FDE14F0E9B
:10BC1000511C342D3195812C912C1201612C712CE9
:10BC200014E0032F020DF10121911F01B301680DF2
:10BC3000791D6A0D7B1DE12C412FCE01019639A3A0
:10BC40000E94C85C1150F4E06F0E711C39A11111F3
:10BC5000E8CF3C5F80E1880E911CE0E48E169104F1
:10BC6000E1F685E0898F89E08A8F8EE08B8F84E111
:10BC70008C8F88248394912C2E01F9E14F0E511C56
:10BC80008FE0F82EF4183401120114E03F2D380D26
:10BC9000032F020DF10121911F01B3016F7077276E
:10BCA000660F771F660F771F6A0D7B1DEE24E394E6
:10BCB000412FCE01019639A30E94C85C1150F5E0D6
:10BCC0006F0E711C39A11111E3CF84E0880E911C15
:10BCD000E1E18E169104B9F684E08D8B8BE08E8BBA
:10BCE00080E18F8B87E1888F65E0862E912C2E0175
:10BCF000F5E14F0E511C85E2F82EF41834011201C3
:10BD000014E03F2D3819032F020DF10121911F017D
:10BD1000B3016F707727660F771F660F771F6A0D65
:10BD20007B1D52E0E52E412FCE01019639A30E94E2
:10BD3000C85C1150F3E06F0E711C39A11111E3CFF3
:10BD400084E0881A9108E5EF8E16EFEF9E06B1F6B3
:10BD500086E0898B8AE08A8B8FE08B8B85E18C8BE8
:10BD6000812C912C2E01F1E14F0E511C80E3F82E15
:10BD7000F4183401120114E03F2D3819032F020D7D
:10BD8000F10121911F01B3016F707727660F771FB3
:10BD9000660F771F6A0D7B1D93E0E92E412FCE01C0
:10BDA000019639A30E94C85C1150F7E06F0E711C18
:10BDB00039A11111E3CF84E0881A9108E0EF8E16C3
:10BDC000EFEF9E06B1F6F6014081518162817381E9
:10BDD00089819A81AB81BC81840F951FA61FB71FF3
:10BDE00080839183A283B383448155816681778167
:10BDF0008D819E81AF81B885840F951FA61FB71FC7
:10BE000084839583A683B783408551856285738536
:10BE100089859A85AB85BC85840F951FA61FB71FA2
:10BE200080879187A287B387448555856685778506
:10BE30008D859E85AF85B889840F951FA61FB71F76
:10BE400084879587A687B78780899189A289B389D6
:10BE50000196A11DB11D808B918BA28BB38BA196F6
:10BE60000FB6F894DEBF0FBECDBFDF91CF911F910B
:10BE70000F91FF90EF90DF90CF90BF90AF909F9089
:10BE80008F907F906F905F904F903F902F9008958C
:10BE90006F927F928F929F92AF92BF92CF92DF92DA
:10BEA000EF92FF920F931F93CF93DF93CDB7DEB73F
:10BEB000C054D1090FB6F894DEBF0FBECDBF8C01C0
:10BEC0006B014A017A015B01E114E2E0FE0650F0E9
:10BED000B501C8010E94C05D82E0F81A90E4A90E85
:10BEE000B11CF2CF5401AB2CBB24A69446E0AA0CA3
:10BEF000BB1C4A95E1F7AC0CBD1C6401F1E0DF22EC
:10BF0000CE0101967C0180E4F70111928A95E9F750
:10BF1000360153E0769467945A95E1F7A301B50191
:10BF2000C7010E94D375F7E08F229924F701E60D2F
:10BF3000F71D8114910469F0D501A60DB71D80E8A5
:10BF400090E002C0959587958A94E2F79C91892BA1
:10BF500001C080E8808388E0680E711C90E4691657
:10BF60007104A8F0B701C8010E94C05DF801808982
:10BF70009189A289B3890197A109B109808B918B1D
:10BF8000A28BB38B88E3F70111928A95E9F7F80148
:10BF900080899189A289B38929E0880F991FAA1FF6
:10BFA000BB1F2A95D1F78C0D9D1DA11DB11D9C01B4
:10BFB000AD0189AF3AAF4BAF5CAF1DAE1EAE1FAE49
:10BFC00021961FAE2197B701C8010E94C05DC05CD9
:10BFD000DF4F0FB6F894DEBF0FBECDBFDF91CF911C
:10BFE0001F910F91FF90EF90DF90CF90BF90AF9097
:10BFF0009F908F907F906F900895DC0190E1FB01FE
:10C0000001900D929A95E1F708958F929F92AF92C9
:10C01000BF92CF92DF92EF92FF920F931F93CF9335
:10C02000DF93CDB7DEB768970FB6F894DEBF0FBECB
:10C03000CDBF7C018B01CE0101962D8B3E8B4F8BAA
:10C04000588F0E949A5D2D893E894F89588D4901EC
:10C050005A016801811482E09806A104B104A8F095
:10C06000B601CE0101962D8B3E8B4F8B588F0E94CF
:10C07000C05D80E4C80ED11C82E0981AA108B10806
:10C08000588D4F893E892D89E5CFDA01C90191701C
:10C09000AA27BB27BA01A90129E07695679557958C
:10C0A00047952A95D1F79A0146E0220F331F4A950A
:10C0B000E1F7B801620F731FAC01CE0101960E9437
:10C0C000485FBE016F5F7F4FC7010E94FD5F6896AA
:10C0D0000FB6F894DEBF0FBECDBFDF91CF911F9199
:10C0E0000F91FF90EF90DF90CF90BF90AF909F9017
:10C0F0008F900895CF92DF92EF92FF920F931F934C
:10C10000CF93DF931F92CDB7DEB77C01262F82E855
:10C11000860F87010B591D4F823010F06B3149F4A7
:10C12000F801608171818BE190E029830E946F7634
:10C130002981D701A559BD4F3C9111964C9111977A
:10C14000822F90E0FC01E327EE0FFF1FEB57FA4F21
:10C1500025913491C42ED12C2C253D252D933C9333
:10C16000F801608171810F90DF91CF911F910F9144
:10C17000FF90EF90DF90CF900C946F76CF93DF938A
:10C18000E2E7F2E0DC01EF011D922197E9F7FC0103
:10C19000EB59FD4F518340833297718360833A9608
:10C1A0003183208332972FEF3FEF31832083329703
:10C1B00031832083389681E08083DF91CF91089589
:10C1C0003F924F925F926F927F928F929F92AF9227
:10C1D000BF92CF92DF92EF92FF920F931F93CF9374
:10C1E000DF932C013C012BE9621A2DEF720A6C01DE
:10C1F00040E9C41A4DEFD40AEC01C159DD4F8C015E
:10C2000009591D4F7C0187E9E81A8DEFF80A33249C
:10C210003394AA24AA94BA2C4201A3E98A1AADEF56
:10C220009A0AF301808191810E9414768F3FFFEF7B
:10C230009F0709F45CC0F601208121112CC08E37C4
:10C240009105F1F4D8018D919C91049788F0F70144
:10C2500080819181883B904F21F08091181888232C
:10C2600039F0D401ED91FC91309711F0C20109959C
:10C270003882F701B182A082D8011D921C92D1CFE1
:10C280008F37910511F41882CCCF8B31910519F4B9
:10C29000F6013082C6CF2881222331F1D8012D91B9
:10C2A0003C912336B2E03B07F0F4A9014F5F5F4FAA
:10C2B000F80151834083F201E20FF31F8083D7011D
:10C2C0002D913C91F901E827FF27EE0FFF1FEB5757
:10C2D000FA4F85919491232F332782279327F701D3
:10C2E0009183808301C01882D6011C929ACFDF917E
:10C2F000CF911F910F91FF90EF90DF90CF90BF9063
:10C30000AF909F908F907F906F905F904F903F90F5
:10C3100008956F927F928F929F92AF92BF92CF9229
:10C32000DF92EF92FF920F931F93CF93DF93EC0175
:10C330003B014A017C018FE8E81A8DEFF80AF7010A
:10C3400010825E01F5E9AF1AFDEFBF0A8FEF9FEF94
:10C35000F501918380836E01FBE9CF1AFDEFDF0ABF
:10C36000F601608171818EE790E00E946F76830113
:10C37000860C971C0815190549F0F80161918F0189
:10C38000CE010E947A600E943F6AF4CFF50160817D
:10C3900011816095CE010E947A60612F6095CE0177
:10C3A0000E947A60F601608171818EE790E00E94C0
:10C3B0006F7681E0F7018083DF91CF911F910F911C
:10C3C000FF90EF90DF90CF90BF90AF909F908F90B5
:10C3D0007F906F9008952FB7F89460913617709101
:10C3E000371780913817909139172FBF0895FC01A6
:10C3F0002FB7F894A681B7816D937C9346815781BE
:10C40000828193814817590719F48081918103C073
:10C41000868197810296978386832FBF0895FC01BA
:10C420002FB7F894A481B58182819381A817B907A9
:10C4300019F48081918104C0A481B581CD01029657
:10C44000958384838D919C912FBF0895CF93DF9323
:10C4500090939C3A80939B3A50937717409376172A
:10C4600070939E3A60939D3A80E797E1E2E2FFE1A4
:10C47000DF019C011D9221503040E1F7C8EDD6E369
:10C4800088E0DE01E82F1D92EA95E9F7A7E1B8E31D
:10C49000FD0111928A95E9F7E0EDF6E3D183C083BF
:10C4A000D783C683D583C48384EF96E39383828343
:10C4B000E2ECFAE3B183A083B783A683B583A483B8
:10C4C00083E398E393838283DF91CF9108951F9351
:10C4D000CF93DF9300D0CDB7DEB70E940612182F9E
:10C4E000882309F476C041E060E277E082E996E3D0
:10C4F0000E945535809312388430D9F582E996E34D
:10C500000E94DC3E46E060E277E082E996E30E942A
:10C51000553580931238811123C01092EC0B109284
:10C52000ED0B1092EE0B1092EF0B1092133810924D
:10C53000143810921538109216381A8219829E01FA
:10C540002F5F3F4F44E050E063E178E382E996E3F8
:10C550000E94873A8093123882E996E30E94DC3E7B
:10C5600041E060E277E082E996E30E9455358093EE
:10C5700012388091123881112CC01A8219829E01C2
:10C580002F5F3F4F44E050E063E178E382E996E3B8
:10C590000E94B1388093123882E996E30E94DC3E13
:10C5A00080911238811115C089819A81049789F48C
:10C5B0008091133890911438A0911538B0911638A5
:10C5C0008093EC0B9093ED0BA093EE0BB093EF0BDD
:10C5D00005C082E996E30E94DC3E10E0812F0F90B7
:10C5E0000F90DF91CF911F910895CF93DF9300D0EB
:10C5F000CDB7DEB742E060E277E082E996E30E94E1
:10C60000553580931238811138C08091EC0B909190
:10C61000ED0BA091EE0BB091EF0B0196A11DB11D9A
:10C620008093EC0B9093ED0BA093EE0BB093EF0B7C
:10C630008093133890931438A0931538B09316381C
:10C640001A8219829E012F5F3F4F44E050E063E160
:10C6500078E382E996E30E94873A8093123882E970
:10C6600096E30E94DC3E80911238811106C08981D8
:10C670009A81049711F481E001C080E00F900F903F
:10C68000DF91CF9108951F93CF93DF93CDB7DEB79E
:10C690006A970FB6F894DEBF0FBECDBF0E94061298
:10C6A000811102C010E0E6C068EF76E38BE397E00B
:10C6B0000E943443809312388450823060F068EFD7
:10C6C00076E385E497E00E943443809312388450E7
:10C6D000823090F409C08BE397E00E9493468093E8
:10C6E0001238882361F3DECF85E497E00E949346F9
:10C6F000809312388111D6CF0E946762182F882349
:10C7000089F2EFE9FAE380E2DF01282F1D922A95F2
:10C71000E9F79091EF0B9F939091EE0B9F9390917F
:10C72000ED0B9F939091EC0B9F9325E437E03F93A3
:10C730002F9323E537E03F932F931F928F93FF931F
:10C74000EF930E94EB760E94F56246E06FE97AE390
:10C7500082E996E30E945535809312380FB6F8941B
:10C76000DEBF0FBECDBF81119DCF84ED93ECA2EB58
:10C77000B1EA898B9A8BAB8BBC8B82E090E09A8F6D
:10C78000898F84E090E0988F8F8B1D861E861F8690
:10C79000188A19861A861B861C8683E692E0A0E01A
:10C7A000B0E08D839E83AF83B88783E090E0A0E004
:10C7B000B0E089839A83AB83BC831E8A1D8A9E0165
:10C7C0002B5E3F4F44E050E0BE016F5E7F4F82E939
:10C7D00096E30E94873A9E012B5E3F4F42E050E075
:10C7E000BE01675E7F4F82E996E30E94873A9E0111
:10C7F0002B5E3F4F42E050E0BE01695E7F4F82E911
:10C8000096E30E94873A9E012B5E3F4F44E050E042
:10C81000BE01635F7F4F82E996E30E94873A9E01E3
:10C820002B5E3F4F44E050E0BE01675F7F4F82E9DF
:10C8300096E30E94873A9E012B5E3F4F44E050E012
:10C84000BE016B5F7F4F82E996E30E94873A9E01AB
:10C850002B5E3F4F44E050E0BE016F5F7F4F82E9A7
:10C8600096E30E94873A82E996E30E94DC3E81E0EB
:10C870008093F00B812F6A960FB6F894DEBF0FBE3F
:10C88000CDBFDF91CF911F9108956F927F928F92CC
:10C890009F92AF92BF92CF92DF92EF92FF920F934F
:10C8A0001F93CF93DF93CDB7DEB76E970FB6F89493
:10C8B000DEBF0FBECDBF8C010E94C2549801295922
:10C8C0003D4F6901811112C0609176177091771701
:10C8D00080EC90E00E946F766091761770917717E8
:10C8E00080E090E00E946F76780179C0D901ED90E8
:10C8F000FC90B3E3EB16F10408F430C1F80190802A
:10C90000B70162517109FE01319680E1DF011D928C
:10C910008A95E9F7D801A60FB71F5F0140E1842E81
:10C920008E0E8D9181938E12FCCFC8010E94A85467
:10C93000E5EAFAE1D5019D915D01819198130EC15F
:10C940008A12F8CFD8011196E5EAFAE130E1A32E78
:10C95000AE0E8D918193AE12FCCF0E9470570E9453
:10C96000C554C701839724E0969587952A95E1F7EA
:10C97000B82E3801812C8B14C0F4D3015196E5EA0E
:10C98000FAE18D918193AE12FCCF85EA9AE10E9483
:10C99000F554D301E5EAFAE181918D93AE12FCCF13
:10C9A0008394B0E16B0E711CE6CFE1E2EE1AF10860
:10C9B000E918F108D601ED92FC9286CFF70181913A
:10C9C0007F01803CD9F48BED90E00E946F766091FE
:10C9D0007617709177178CED90E00E946F76D601F4
:10C9E0008D919C91029760917617709177179701BE
:10C9F000201B310B2817390708F30FC08B3D59F462
:10CA00008BED90E00E946F766091761770917717AA
:10CA10008DED90E0E2CF90E0E0CF80EC90E00E94DE
:10CA20006F7680913017882309F498C00E9406120F
:10CA3000882309F493C08091F00B882309F48AC0FD
:10CA400042E36FE97AE382E996E30E9455358093E9
:10CA50001238811183C01E8E1D8E2FB7F8948091DD
:10CA6000711790917217A0917317B09174172FBF1F
:10CA700080589C4BA249B74C898F9A8FAB8FBC8F43
:10CA80000E94EB6120EC32E140E050E00E948073B4
:10CA90006E5F7F4F8F4F9F4F25E030E040E050E0CA
:10CAA0000E948073A8EEB3E00E9441736D8B7E8B71
:10CAB0008F8B988FF601808191810297A0E0B0E082
:10CAC000898B9A8BAB8BBC8B89839A83AB83BC831A
:10CAD0009E01235E3F4F44E050E0BE01675E7F4F02
:10CAE00082E996E30E94873A9E01235E3F4F44E02D
:10CAF00050E0BE016B5E7F4F82E996E30E94873A69
:10CB00009E01235E3F4F44E050E0BE016F5E7F4FC9
:10CB100082E996E30E94873A9E01235E3F4F44E0FC
:10CB200050E0BE016F5F7F4F82E996E30E94873A33
:10CB3000D6014D915C91425051099E01235E3F4FB9
:10CB4000B80182E996E30E94873A82E996E30E945F
:10CB5000DC3E04C00E944363811172CF6E960FB613
:10CB6000F894DEBF0FBECDBFDF91CF911F910F9123
:10CB7000FF90EF90DF90CF90BF90AF909F908F90FD
:10CB80007F906F9008952F923F924F925F926F9295
:10CB90007F928F929F92AF92BF92CF92DF92EF924D
:10CBA000FF920F931F93CF93DF93CDB7DEB76697B6
:10CBB0000FB6F894DEBF0FBECDBF8091EB0B811195
:10CBC000BCC181E08093EB0B212C312CE12CF12CAA
:10CBD00085EA9AE130E1C32EC80E8091FF0B90E008
:10CBE0002816390608F090C180ED96E30E940F6286
:10CBF0005C0182EC9AE30E940F628C01029708F4B8
:10CC00007FC10E94C254882309F4C0C0802F8F7056
:10CC100090E1D92ED81AD91201C0D12C6D2C712CCB
:10CC2000060D171D24E0169507952A95E1F70B8B45
:10CC30000E944E57882309F4A6C00E94C554D09282
:10CC400037380E946D57E8E3F8E39C01205F3F4FBF
:10CC5000DC014D91CD014193A217B307C9F798E4C8
:10CC6000492E98E3592E812C912C1127C801019748
:10CC70009D8B8C8BA0E1B0E0A619B7093D0180E146
:10CC8000482F4D198B89881608F052C08C899D89D0
:10CC90008816990614F0D11017C0E5EAFAE195015B
:10CCA000255A3A41C9018E0F9F1F60E777E10E9424
:10CCB0005873DC01AE5DB04E8C918193CE12F2CFF1
:10CCC00090E1A90EB11C20C020E0822F90E08615D3
:10CCD000970584F4FC01EB55F54E8A0D9B1D60E72A
:10CCE00077E10E945873DC01AE5DB04E8C91808379
:10CCF0002F5FEBCF842F9FEFE82FF0E0EB55F54E41
:10CD000090838F5F8031C1F785EA9AE14E8B0E9454
:10CD1000D554D201E5EAFAE14E8981918D93CE1284
:10CD2000FCCFAFEF8A1A9A0AB0E14B0E511CAACF82
:10CD300084E0000F111F8A95E1F7580191E1A90ED7
:10CD4000B11CB50187E398E30E94A854F501E95CA2
:10CD5000F74CA5EABAE18D918193CA12FCCFA801E4
:10CD60004F5D5F4F87010F5F1F4F4436A2E05A07A8
:10CD700040F467E378E380919B3A90919C3A0E945B
:10CD800089617801BDC00E94DA10BAC0E7E3F8E318
:10CD9000950127533843C9018E0F9F1F60E777E144
:10CDA0000E945873DC01AE5DB04E8C918193CF012F
:10CDB000875398438017910770F380913017882329
:10CDC00009F492C00E940612882309F48DC0809154
:10CDD000F00B882309F484C042E36FE97AE382E927
:10CDE00096E30E9455358093123881117DC01A8ACE
:10CDF000198A2FB7F8948091711790917217A091AA
:10CE00007317B09174172FBF80589C4BA249B74C31
:10CE10008D879E87AF87B88B0E94EB6120EC32E153
:10CE200040E050E00E9480736E5F7F4F8F4F9F4FB6
:10CE300025E030E040E050E00E948073A8EEB3E0CF
:10CE40000E94417369877A878B879C87C801A0E01D
:10CE5000B0E08D839E83AF83B88789839A83AB8349
:10CE6000BC839E012F5E3F4F44E050E0BE01635FF4
:10CE70007F4F82E996E30E94873A9E012F5E3F4FE3
:10CE800044E050E0BE01675F7F4F82E996E30E9475
:10CE9000873A9E012F5E3F4F44E050E0BE016B5F3A
:10CEA0007F4F82E996E30E94873A9E012F5E3F4FB3
:10CEB00044E050E0BE016F5F7F4F82E996E30E943D
:10CEC000873A9E012F5E3F4FA80167E378E382E92E
:10CED00096E30E94873A82E996E30E94DC3E04C012
:10CEE0000E944363811178CFA80167E378E38091C2
:10CEF0009B3A90919C3A0E948961BFEFEB1AFB0A22
:10CF00008FEF281A380A69CE8091FF0B90E0E8165F
:10CF1000F90658F480917307811101C0299A809114
:10CF200073078111F7CF289AF5CF1092FF0B10925B
:10CF3000FE0B1092FD0B1092EB0B66960FB6F89459
:10CF4000DEBF0FBECDBFDF91CF911F910F91FF903C
:10CF5000EF90DF90CF90BF90AF909F908F907F9099
:10CF60006F905F904F903F902F900895CF92DF92F7
:10CF7000EF92FF928091FF0B882309F440C0E0916B
:10CF80009D3AF0919E3A8289811139C08091A41A0C
:10CF90008F3F31F4FF90EF90DF90CF900C94C365FA
:10CFA000209158173091591740915A1750915B179B
:10CFB000A5E0B0E00E944173C090F10BD090F20B5D
:10CFC000E090F30BF090F40BC60ED71EE81EF91E8E
:10CFD0000E94EB61C616D706E806F90684F40E94A3
:10CFE000C1748091A41A6817A8F20E94EB61609343
:10CFF000F10B7093F20B8093F30B9093F40BFF9073
:10D00000EF90DF90CF900895609176177091771729
:10D0100080EC90E00E946F766091761770917717A0
:10D0200084E190E00E946F76609176177091771797
:10D0300081E090E00E946F7660917617709177178B
:10D0400080EC90E00C946F76609176177091771772
:10D0500080EC90E00E946F76609176177091771760
:10D0600082E190E00E946F7680916407609176176C
:10D0700070917717803C59F48BED90E00E946F76A9
:10D0800060917617709177178CED90E00EC08B3D14
:10D0900059F48BED90E00E946F7660917617709155
:10D0A00077178DED90E001C090E00E946F7660915F
:10D0B00076177091771780EC90E00C946F76CF9391
:10D0C000DF939091BF3A992309F446C0803C09F060
:10D0D00051C080910301811142C01092BF3A8091EA
:10D0E000FF0B8F3008F0C8C18091FD0B9091FE0BB3
:10D0F0008037974108F0C0C16091F90B7091FA0B2D
:10D100008091FB0B9091FC0B019710F48FE697E157
:10D110006817790709F4B0C16817790728F4861BE6
:10D12000970BEC01219605C0861B970BEC01CF589D
:10D13000D84EC230D10508F49FC18091FF0B8F5F9C
:10D140008093FF0B80ED96E30E94F761BE0182ECB5
:10D150009AE30E94F76121C0803C09F08DC181E013
:10D160008093BF3A8EEF809303011092C13A1092E0
:10D17000C03A82C12091C03A3091C13A203492E045
:10D18000390708F079C190910301232B79F49E3F70
:10D1900069F48093030181116FC18091FB0B909121
:10D1A000FC0B9093FA0B8093F90B66C1911146C06A
:10D1B0008B3D21F481E080939A3A5EC190919A3A36
:10D1C000992349F08C3D21F08D3D19F48BED01C080
:10D1D00080EC10929A3A9091FF0B9F3008F04CC16E
:10D1E0002091FD0B3091FE0B2037374108F044C1F0
:10D1F0002091FD0B3091FE0B2F5F3F4F3093FE0BC4
:10D200002093FD0B2091FB0B3091FC0BA9014F5F8C
:10D210005F4F5093FC0B4093FB0BF901EE5DF04E1A
:10D2200080838091FB0B9091FC0B8037974109F034
:10D2300023C11092FC0B1092FB0B1EC1913079F4AC
:10D24000282F30E0AAE0B0E00E94327360932818E3
:10D250007093291880932A1890932B180DC194303D
:10D2600079F4282F30E0AAE0B0E00E943273609396
:10D27000191870931A1880931B1890931C18FCC0EF
:10D28000933079F4282F30E0AAE0B0E00E943273A6
:10D29000609358177093591780935A1790935B17A0
:10D2A000EBC0923019F48093A41AE6C0973021F4B1
:10D2B000DF91CF910C94F206913139F48A3909F05B
:10D2C000DBC0DF91CF910C94F9069830A1F48B3D2F
:10D2D00009F470CF90919A3A992349F08C3D21F04E
:10D2E0008D3D19F48BED01C080EC10929A3ADF91DC
:10D2F000CF910C9426109930A1F48B3D09F45ACFAC
:10D3000090919A3A992349F08C3D21F08D3D19F482
:10D310008BED01C080EC10929A3ADF91CF910C9482
:10D32000F7049A30A1F48B3D09F444CF90919A3AD6
:10D33000992349F08C3D21F08D3D19F48BED01C00E
:10D3400080EC10929A3ADF91CF910C94F9049B30C3
:10D35000A1F48B3D09F42ECF90919A3A992349F08C
:10D360008C3D21F08D3D19F48BED01C080EC1092C5
:10D370009A3ADF91CF910C94FB049C30A1F48B3D41
:10D3800009F418CF90919A3A992349F08C3D21F0F5
:10D390008D3D19F48BED01C080EC10929A3ADF912B
:10D3A000CF910C9404059D30A1F48B3D09F402CF7C
:10D3B00090919A3A992349F08C3D21F08D3D19F4D2
:10D3C0008BED01C080EC10929A3ADF91CF910C94D2
:10D3D0000D059034A1F48B3D09F4ECCE90919A3A6E
:10D3E000992349F08C3D21F08D3D19F48BED01C05E
:10D3F00080EC10929A3ADF91CF910C9419059E30EF
:10D40000A1F48B3D09F4D6CE90919A3A992349F034
:10D410008C3D21F08D3D19F48BED01C080EC109214
:10D420009A3ADF91CF910C942505903121F4DF9148
:10D43000CF910C94F004903F19F40E94110718C08A
:10D44000923131F48130C1F4DF91CF910C94246892
:10D45000933151F4811104C0DF91CF910C940E07E8
:10D46000DF91CF910C940A07943131F4811104C0FB
:10D47000DF91CF910C940468DF91CF9108954FB75D
:10D48000F89420912C1730912D1780912E179091A0
:10D490002F174FBF2817390761F19FB7F894E09114
:10D4A0002C17F0912D1720912A1730912B17E21786
:10D4B000F30729F4209128173091291707C0E0912C
:10D4C0002C17F0912D179F012F5F3F4F30932D1791
:10D4D00020932C1780819FBF0E945F680E94EB61A0
:10D4E0006093F50B7093F60B8093F70B9093F80B0A
:10D4F000C6CF0895EF92FF920F931F93CF93DF93C0
:10D500007C018B01609176177091771780EC90E029
:10D510000E946F76609176177091771780E490E0A3
:10D520000E946F76E7010E0D1F1D609176177091B6
:10D530007717C017D107F9F08991803C59F48BED2A
:10D5400090E00E946F7660917617709177178CED5E
:10D5500090E00EC08B3D59F48BED90E00E946F7609
:10D5600060917617709177178DED90E001C090E093
:10D570000E946F76DACF80EC90E0DF91CF911F911F
:10D580000F91FF90EF900C946F76EF92FF920F93B4
:10D590001F93CF93DF937C018B016091761770917D
:10D5A000771780EC90E00E946F766091761770910B
:10D5B000771780EF90E00E946F76E7010E0D1F1D38
:10D5C0006091761770917717C017D107F9F089919C
:10D5D000803C59F48BED90E00E946F766091761755
:10D5E000709177178CED90E00EC08B3D59F48BED68
:10D5F00090E00E946F7660917617709177178DEDAD
:10D6000090E001C090E00E946F76DACF80EC90E06D
:10D61000DF91CF911F910F91FF90EF900C946F7657
:10D62000CF92DF92EF92FF920F931F93CF93DF93EE
:10D63000CDB7DEB728970FB6F894DEBF0FBECDBFCB
:10D640008B01FC01608171818281938120E831E549
:10D6500041E050E00E94807369017A012CE330E0E0
:10D6600040E050E00E94617929833A834B835C83D8
:10D6700089819A81AB81BC81F80160836CE370E0A1
:10D680000E946C73DC01CB01F801A1838283C60187
:10D69000069667E070E00E94587384832DEA3EE8A6
:10D6A00040E050E0C701B6010E94617929833A83C6
:10D6B0006D837E838F83988789819A8124E6289F52
:10D6C0006001299FD00C11246D817E818F81988506
:10D6D00025EB35E040E050E00E94617929833A83F0
:10D6E0006D837E83E980FA80EE0CFF1CEE0CFF1C3C
:10D6F000EC0CFD1C8D819E81F5E6EF16F10410F017
:10D70000019604C024E6E216F10419F021E030E0AD
:10D7100002C020E030E0A90144595E4F4817590784
:10D7200068F46DE671E0821B930B0E946C73DC0160
:10D73000CB01E80EF91ECD0120E030E044E6E40E16
:10D74000F11CF801F782E68291878087255C3F4FC4
:10D750008217930748F46FE170E00E946C73DC015C
:10D76000CB01F801858322C069E970E0821B930B2D
:10D770000E946C73DC01CB01F82EFF0CFF0CF80E3D
:10D780006DE370E0CD010E946C73DC01CB01E82EEB
:10D79000EE0C6FE170E0CD010E946C73DC01CB01F7
:10D7A00022E0280FF20EFE0CF801F582A383F801A7
:10D7B0001386128683818F5F838328960FB6F89431
:10D7C000DEBF0FBECDBFDF91CF911F910F91FF90B4
:10D7D000EF90DF90CF900895CF92DF92EF92FF927B
:10D7E0000F931F93CF93DF9300D000D0CDB7DEB758
:10D7F0008C010E94A56C69837A838B839C83F801DA
:10D800008285938597FF0EC0E091D43AF091D53A86
:10D81000309741F060ED7AE3CE0101960995F80169
:10D8200093878287F801828593851816190694F4E8
:10D83000AA2797FDA095BA2F49815A816B817C81D7
:10D840006A017B01C81AD90AEA0AFB0AC982DA828C
:10D85000EB82FC8289819A81AB81BC814091D03A74
:10D860005091D13A6091D23A7091D33A841B950B82
:10D87000A60BB70B89839A83AB83BC83B801CE0117
:10D8800001960E94546C69817A818B819C810F90F2
:10D890000F900F900F90DF91CF911F910F91FF90FC
:10D8A000EF90DF90CF900895CF92DF92EF92FF92AA
:10D8B0000F931F93CF93DF9300D000D0CDB7DEB787
:10D8C0006C017B01E091D43AF091D53A309729F080
:10D8D00060ED7AE309958C0102C00FEF1FEFF601AE
:10D8E00040815181628173818091D03A9091D13A87
:10D8F000A091D23AB091D33A480F591F6A1F7B1FAB
:10D90000101611064CF4C801AA2797FDA095BA2F4E
:10D91000480F591F6A1F7B1F49835A836B837C837F
:10D92000B701CE0101960E94106BF70113870287A1
:10D930000F900F900F900F90DF91CF911F910F914B
:10D94000FF90EF90DF90CF9008958F929F92AF92CB
:10D95000BF92CF92DF92EF92FF920F931F93CF93DC
:10D96000DF93EC01EE81FF818F0104561109B9F0BC
:10D97000CF01855691096C0197FF03C023E0C20EC9
:10D98000D11CD594C794D594C7946CE97FEF0E94BD
:10D990006C73C60ED71E8FEFC81AD80A02C0C12CEE
:10D9A000D12CEE24D7FCE094FE2C2DE631E0D801FA
:10D9B0000E944279C60ED71EE81EF91E8B81992758
:10D9C00087FD90958C01015011092D8122302CF496
:10D9D000222379F1015E1F4F2CC0CF018459984F4B
:10D9E0000E94616DE82FF0E0FB96E00FF11F8D8142
:10D9F000992787FD909502978530910514F0E75699
:10DA0000FF4F65E070E00E946C739C0197FF02C0BD
:10DA10002F5F3F4F359527959DE3929FA001939FE0
:10DA2000500D11248F01040F151F80FF02C0015EED
:10DA30001F4FA801662757FD6095762F9A01AB010D
:10DA40002C0D3D1D4E1D5F1D60E871E581E090E0ED
:10DA50000E9451796B017C01AA81BB27A7FDB0957B
:10DA600020E13EE00E9442794B015C01A981BB2785
:10DA7000A7FDB0952CE330E00E944279DC01CB0198
:10DA8000880D991DAA1DBB1D4881552747FD50953E
:10DA9000652F752F840F951FA61FB71FBC01CD01E1
:10DAA0006C0D7D1D8E1D9F1DDF91CF911F910F91DC
:10DAB000FF90EF90DF90CF90BF90AF909F908F90AE
:10DAC00008959C0123703327232B59F464E670E0FA
:10DAD0000E946C73892B39F46370772781E0672B80
:10DAE00019F080E0089581E008950E9420048DE2FD
:10DAF00098E10E94E0600E943F6A0E94B6670E941F
:10DB00003A120E943654F3CF2F923F924F925F9277
:10DB10006F927F928F929F92AF92BF92CF92DF923D
:10DB2000EF92FF920F931F93CF93DF93CDB7DEB7A2
:10DB300063970FB6F894DEBF0FBECDBF6C014B01EB
:10DB40002A01FC0117821682838181FF43C3AE0143
:10DB50004F5F5F4F3A01F6019381F40193FD859188
:10DB600093FF81914F01882309F430C3853239F442
:10DB700093FD859193FF81914F01853239F4B60170
:10DB800090E00E946F7652012501E5CF10E0F12C64
:10DB900020E02032A0F48B3269F030F4803259F06A
:10DBA000833269F420612CC08D3239F0803339F42E
:10DBB000216026C02260246023C0286021C027FD88
:10DBC00027C030ED380F3A3078F426FF06C0FAE06F
:10DBD0001F9F300D1124132F13C04AE0F49E300D07
:10DBE0001124F32E20620CC08E3221F426FDEEC2E9
:10DBF000206406C08C3611F4206802C0883641F4D7
:10DC0000F40193FD859193FF81914F018111C1CF63
:10DC10009BEB980F933018F42061805E06C09BE95F
:10DC2000980F933008F071C12F7E26FF16E02F73F6
:10DC3000322E853619F42064322E08C0863621F43F
:10DC4000F22FF0683F2E02C01111115037FE07C0AD
:10DC50001C3350F4EE24E394E10E27E00BC018309F
:10DC600038F027E017E005C027E04CE3E42E02C0BF
:10DC7000212FE12C520144E0A40EB11CF20160817D
:10DC80007181828193810E2DA3010E94F0742C0179
:10DC9000098100FF02C003FF07C031FC08C032FE4B
:10DCA00009C030E2232E07C02DE2222E04C09BE2E1
:10DCB000292E01C0212C802F8C7019F0211068C2F0
:10DCC000A8C237FE0FC0E40C04FF04C08A81813370
:10DCD00009F4EA941E1474F5F8E0FE1578F588E06E
:10DCE000E82E2CC036FC2AC0812F90E084159505C3
:10DCF0009CF02CEF42162FEF520674F0432D406833
:10DD0000342E0AC0E2E0F0E0EC0FFD1FE10FF11D40
:10DD10008081803319F411501111F4CF37FE0EC0F9
:10DD2000EE24E394E10E812F90E0481659062CF47E
:10DD3000141904C0EE24E39401C010E037FE06C0BD
:10DD40001414150434F4C201019605C085E090E076
:10DD500002C081E090E021100196112331F0212FC3
:10DD600030E02F5F3F4F820F931F2F2D30E082173F
:10DD7000930714F4F81A01C0F12C832D897049F42B
:10DD8000FF2039F0B60180E290E00E946F76FA94AD
:10DD9000F7CF222029F0B601822D90E00E946F7605
:10DDA00033FC09C0FF2039F0B60180E390E00E9407
:10DDB0006F76FA94F7CF37FE5AC0942D852D57FE13
:10DDC00002C090E080E0292E382E20E030E0A20151
:10DDD0004E1951095D874C87A201421953095F878B
:10DDE0004E87612F70E044275527461B570B598BF0
:10DDF000488B5FEF2516350649F4B6018EE290E0B8
:10DE00002A8B3B8B0E946F763B892A8942145304EC
:10DE10006CF04C855D854215530544F4EE85FF8515
:10DE2000E20FF31FE60DF71D818101C080E351E091
:10DE3000251A31082F5F3F4F488959892416350626
:10DE40004CF0B60190E02A8B3B8B0E946F762A89BA
:10DE50003B89CFCF2414350439F49A81963318F4D2
:10DE6000953311F404FF81E3B60190E04BC08A8141
:10DE7000813309F00F7EB60190E00E946F76111198
:10DE800005C034FC18C085E690E017C0B6018EE2EC
:10DE900090E00E946F7682E0EE24E394E80EF301B6
:10DEA000E80FF11D8081B60190E00E946F7611505D
:10DEB0008E2D91F7E6CF85E490E0B6010E946F7653
:10DEC00057FC05C04114510439F404FF05C05194B6
:10DED000419451088DE201C08BE2B60190E00E94AE
:10DEE0006F7680E39AE0491651042CF08F5F5AE078
:10DEF000451A5108F7CFB60190E00E946F76B6013F
:10DF0000C201C0960E946F7657C1833631F08337C5
:10DF100079F0833509F058C021C05201E2E0AE0E1D
:10DF2000B11CF2018081898301E010E0230114C05B
:10DF30005201F2E0AF0EB11CF2014080518026FF89
:10DF400003C0612F70E002C06FEF7FEFC2012A8B28
:10DF50000E94E7758C012A892F7715C05201F2E0E3
:10DF6000AF0EB11CF2014080518026FF03C0612F2B
:10DF700070E002C06FEF7FEFC2012A8B0E94C8756C
:10DF80008C012A892068322E23FD1AC08F2D90E043
:10DF900008171907A8F4B60180E290E00E946F7696
:10DFA000FA94F4CFF20137FC859137FE81912F016D
:10DFB000B60190E00E946F76F110FA9401501109B9
:10DFC0000115110579F7F8C0843611F0893659F535
:10DFD000520127FF09C0F4E0AF0EB11CF2016081CD
:10DFE0007181828193810AC0F2E0AF0EB11CF2010F
:10DFF00060817181882777FD8095982F2F76322E4A
:10E0000097FF09C090958095709561957F4F8F4FD0
:10E010009F4F2068322E2AE030E0A3010E9428772B
:10E02000E82EE6183FC0022F853721F40F7E2AE044
:10E0300030E01DC0097F8F3691F018F4883559F013
:10E04000C5C0803719F0883711F0C0C0006104FFE7
:10E0500009C0046007C024FF08C0066006C028E0AD
:10E0600030E005C020E130E002C020E132E05201A2
:10E0700007FF09C0F4E0AF0EB11CF20160817181AD
:10E080008281938108C0F2E0AF0EB11CF201608181
:10E09000718180E090E0A3010E942877E82EE618C5
:10E0A0000F77302E36FE0BC0332D3E7FE11650F435
:10E0B00034FE0AC032FC08C0332D3E7E05C00E2D52
:10E0C000332D03C00E2D01C0012F34FF0CC0FE0103
:10E0D000EE0DF11D8081803311F4397E08C032FFCE
:10E0E00005C00E5F04C0832F867809F00F5F33FDF3
:10E0F00013C030FF06C01E2D0F1518F41F0D101B86
:10E100000F2D0F1568F4B60180E290E03B8B0E9462
:10E110006F760F5F3B89F5CF0F1510F4F01A01C031
:10E12000F12C34FF12C0B60180E390E03B8B0E94DB
:10E130006F763B8932FF17C031FD03C088E790E05E
:10E1400002C088E590E0B6010CC0832F867859F0B4
:10E1500031FF02C08BE201C080E237FD8DE2B601E3
:10E1600090E00E946F76E11638F4B60180E390E00B
:10E170000E946F761150F7CFEA94F301EE0DF11D76
:10E180008081B60190E00E946F76E110F5CF14C057
:10E19000F4E0FF1558F584E0F81A33FE1EC0211094
:10E1A00026C003FF2AC00CEB10E0F32DF0713F2EC8
:10E1B000F8018491811124C0FF2009F4E5CCB60157
:10E1C00080E290E00E946F76FA94F6CFF6018681A5
:10E1D000978126C08FEF9FEF23C0B60180E290E0C9
:10E1E0000E946F76FA94F110F8CFD9CFF12CB601D6
:10E1F000822D90E00E946F76D4CF00EC10E0D5CF56
:10E2000031108052B60190E00E946F760F5F1F4F71
:10E21000CFCF23E02F1510F483E0BECFF12CC1CF78
:10E2200063960FB6F894DEBF0FBECDBFDF91CF91DE
:10E230001F910F91FF90EF90DF90CF90BF90AF9024
:10E240009F908F907F906F905F904F903F902F9016
:10E2500008955058BB27AA270E9441710C948B72D5
:10E260000E947D7238F00E94847220F039F49F3F42
:10E2700019F426F40C947A720EF4E095E7FB0C94F2
:10E280007472E92F0E949C7258F3BA1762077307E1
:10E290008407950720F079F4A6F50C94BE720EF46D
:10E2A000E0950B2EBA2FA02D0B01B90190010C01A6
:10E2B000CA01A0011124FF27591B99F0593F50F4BE
:10E2C000503E68F11A16F040A22F232F342F442716
:10E2D000585FF3CF469537952795A795F04053950E
:10E2E000C9F77EF41F16BA0B620B730B840BBAF0DE
:10E2F0009150A1F0FF0FBB1F661F771F881FC2F749
:10E300000EC0BA0F621F731F841F48F4879577955C
:10E310006795B795F7959E3F08F0B0CF9395880F16
:10E3200008F09927EE0F9795879508950E94AA7196
:10E330000C948B720E94847258F00E947D7240F09F
:10E3400029F45F3F29F00C94747251110C94BF7240
:10E350000C947A720E949C7268F39923B1F355234E
:10E3600091F3951B550BBB27AA27621773078407E8
:10E3700038F09F5F5F4F220F331F441FAA1FA9F37E
:10E3800035D00E2E3AF0E0E832D091505040E6956C
:10E39000001CCAF72BD0FE2F29D0660F771F881FCD
:10E3A000BB1F261737074807AB07B0E809F0BB0BC0
:10E3B000802DBF01FF2793585F4F3AF09E3F5105D4
:10E3C00078F00C9474720C94BF725F3FE4F3983E43
:10E3D000D4F3869577956795B795F7959F5FC9F7BD
:10E3E000880F911D9695879597F90895E1E0660F3E
:10E3F000771F881FBB1F621773078407BA0720F0B7
:10E40000621B730B840BBA0BEE1F88F7E09508951F
:10E410000E94A47288F09F5798F0B92F9927B7519E
:10E42000B0F0E1F0660F771F881F991F1AF0BA95B8
:10E43000C9F714C0B13091F00E94BE72B1E00895E6
:10E440000C94BE72672F782F8827B85F39F0B93FD8
:10E45000CCF3869577956795B395D9F73EF490956B
:10E460008095709561957F4F8F4F9F4F0895E894E9
:10E4700009C097FB3EF490958095709561957F4F0C
:10E480008F4F9F4F9923A9F0F92F96E9BB279395BA
:10E49000F695879577956795B795F111F8CFFAF4CA
:10E4A000BB0F11F460FF1BC06F5F7F4F8F4F9F4FFB
:10E4B00016C0882311F096E911C0772321F09EE859
:10E4C000872F762F05C0662371F096E8862F70E0BF
:10E4D00060E02AF09A95660F771F881FDAF7880F99
:10E4E0009695879597F9089597F99F6780E870E06A
:10E4F00060E008959FEF80EC089500240A941616BA
:10E50000170618060906089500240A941216130621
:10E51000140605060895092E0394000C11F48823AF
:10E5200052F0BB0F40F4BF2B11F460FF04C06F5FCB
:10E530007F4F8F4F9F4F089557FD9058440F551FA1
:10E5400059F05F3F71F04795880F97FB991F61F075
:10E550009F3F79F087950895121613061406551FEC
:10E56000F2CF4695F1DF08C0161617061806991F58
:10E57000F1CF86957105610508940895E894BB274D
:10E5800066277727CB0197F908950E94D8720C94DB
:10E590008B720E947D7238F00E94847220F0952365
:10E5A00011F00C9474720C947A7211240C94BF7252
:10E5B0000E949C7270F3959FC1F3950F50E0551F18
:10E5C000629FF001729FBB27F00DB11D639FAA27C8
:10E5D000F00DB11DAA1F649F6627B00DA11D661F17
:10E5E000829F2227B00DA11D621F739FB00DA11D38
:10E5F000621F839FA00D611D221F749F3327A00DF2
:10E60000611D231F849F600D211D822F762F6A2F8D
:10E6100011249F5750409AF0F1F088234AF0EE0FF2
:10E62000FF1FBB1F661F771F881F91505040A9F71F
:10E630009E3F510580F00C9474720C94BF725F3F42
:10E64000E4F3983ED4F3869577956795B795F7955B
:10E65000E7959F5FC1F7FE2B880F911D96958795D3
:10E6600097F90895A29FB001B39FC001A39F700DB9
:10E67000811D1124911DB29F700D811D1124911DCA
:10E6800008950E943273A59F900DB49F900DA49F92
:10E69000800D911D11240895991B79E004C0991FE4
:10E6A000961708F0961B881F7A95C9F780950895EC
:10E6B000AA1BBB1B51E107C0AA1FBB1FA617B707A8
:10E6C00010F0A61BB70B881F991F5A95A9F78095C4
:10E6D0009095BC01CD01089597FB072E16F4009488
:10E6E00007D077FD09D00E94587307FC05D03EF48F
:10E6F000909581959F4F0895709561957F4F0895EE
:10E70000A1E21A2EAA1BBB1BFD010DC0AA1FBB1F35
:10E71000EE1FFF1FA217B307E407F50720F0A21BA7
:10E72000B30BE40BF50B661F771F881F991F1A9414
:10E7300069F760957095809590959B01AC01BD013E
:10E74000CF010895689401C0E8948F929F92CF936F
:10E75000DF930E94B073DF91CF919F908F900895C7
:10E7600088249924F401E401B0E49F93AA279A1520
:10E770008B049C04ED05FE05CF05D007A10798F496
:10E78000AD2FDC2FCF2FFE2FE92D982C892E982F1F
:10E79000872F762F652F542F432F322F2227B850E3
:10E7A00031F7BF9127C01B2EBF91BB27220F331F0C
:10E7B000441F551F661F771F881F991F881C991CAF
:10E7C000EE1FFF1FCC1FDD1FAA1FBB1F8A149B0457
:10E7D000EC05FD05CE05DF05A007B10748F08A1856
:10E7E0009B08EC09FD09CE09DF09A00BB10B2160E4
:10E7F0001A94E1F62EF49401AF01BE01CD01000C94
:10E800000895EE0FFF1F0024001C0BBE0790F69129
:10E81000E02D09940F93083090F0982F872F762FD2
:10E82000652F542F432F322F22270850F4CF220F69
:10E83000331F441F551F661F771F881F991F0A9596
:10E84000B2F70F91089597FB10F8169400080F93F4
:10E85000083098F00850232F342F452F562F672F5C
:10E86000782F892F902DF4CF0594979587957795DC
:10E87000679557954795379527950A95AAF70F916C
:10E8800008952A0D3B1D4C1D5D1D6E1D7F1D801FB3
:10E89000911F08950024A7FD00942A0F301D401DEC
:10E8A000501D601D701D801D901D08952A193B0983
:10E8B0004C095D096E097F09800B910B08952A159B
:10E8C0003B054C055D056E057F05800791070895A2
:10E8D0000024A7FD00942A17300540055005600567
:10E8E00070058005900508958F929F92AF92BF9218
:10E8F000CF92DF92EF92FF92CF93DF93EC0168818A
:10E9000079818A819B81611571058105910521F4C9
:10E9100064E279ED8BE597E02DE133EF41E050E0E3
:10E920000E94617949015A019B01AC01A7EAB1E457
:10E930000E9441736B017C01ACEEB4EFA501940120
:10E940000E944C79DC01CB018C0D9D1DAE1DBF1DBD
:10E95000B7FF03C00197A109B04888839983AA83B0
:10E96000BB83BC01CD019F77DF91CF91FF90EF90EA
:10E97000DF90CF90BF90AF909F908F9008950C94B0
:10E98000747484E091E00C94747460930401709347
:10E990000501809306019093070108956627772764
:10E9A0000C948677FC0188279927E89421912032DE
:10E9B000E9F3293010F02E30C8F32B3241F02D321C
:10E9C00039F4689404C00E940C76820F911D219145
:10E9D00020532A30C0F31EF4909581959F4F0895DF
:10E9E000283008F027E03327DA01990F311D87FD21
:10E9F000916000966105710539F432602E5F3D9398
:10EA000030E32A95E1F708959F3F30F08038710593
:10EA1000610509F03C5F3C5F3D93913008F08068F0
:10EA2000911DDF93CF931F930F93FF92EF92192FB6
:10EA3000987F9695E92F96959695E90FFF27E25EC8
:10EA4000FE4F99273327EE24FF24A701E701059005
:10EA50000894079428F4360FE71EF81E491F511D2D
:10EA6000660F771F881F991F0694A1F705900794DA
:10EA700028F4E70EF81E491F561FC11D770F881F87
:10EA8000991F661F0694A1F70590079428F4F80EC5
:10EA9000491F561FC71FD11D880F991F661F771F5B
:10EAA0000694A1F70590079420F4490F561FC71F3D
:10EAB000D81F990F661F771F881F0694A9F78491A6
:10EAC0001095177041F0D695C79557954795F794CF
:10EAD000E7941A95C1F7E4ECF0E06894159015916D
:10EAE00035916591959105907FE27395E118F10A52
:10EAF000430B560BC90BD009C0F7E10CF11E431FA5
:10EB0000561FC91FD01D7EF4703311F48A95E6CFCD
:10EB1000E894015030F0080F0AF40027021708F4B7
:10EB2000202F2395022F7A3328F079E37D932A95BD
:10EB3000E9F710C07D932A9589F606949795679515
:10EB4000379517951794E118F10A430B560BC90B2B
:10EB5000D00998F023957E9173957A3308F070E38D
:10EB60007C932013B8F77E9170617D9330F083958C
:10EB700071E37D9370E32A95E1F71124EF90FF9004
:10EB80000F911F91CF91DF91992787FD909508955F
:10EB9000FC010590615070400110D8F78095909568
:10EBA0008E0F9F1F0895FB01DC0102C001900D92A2
:10EBB00041505040D8F70895FC018191861721F00B
:10EBC0008823D9F7992708953197CF010895FC013B
:10EBD0006150704001900110D8F7809590958E0F8C
:10EBE0009F1F0895FB0151915523A9F0BF01DC013E
:10EBF0004D9145174111E1F759F4CD0101900020E5
:10EC000049F04D9140154111C9F3FB014111EFCF7E
:10EC100081E090E0019708957AE0979F902D879F7B
:10EC2000802D910D11240895CF93DF93EC012B815A
:10EC300020FF33C026FF0AC02F7B2B838E819F814C
:10EC400001969F838E838A8190E029C022FF0FC0A6
:10EC5000E881F9818081992787FD9095009719F4C3
:10EC600020622B831AC03196F983E8830EC0EA85AF
:10EC7000FB85099597FF09C02B81019611F080E271
:10EC800001C080E1822B8B8308C02E813F812F5FE2
:10EC90003F4F3F832E83992702C08FEF9FEFDF9175
:10ECA000CF9108950F931F93CF93DF93CDB7DEB726
:10ECB0000F811885F801838188608383AE01455FE9
:10ECC0005F4F69857A85C8010E94846DF8012381B0
:10ECD000277F2383DF91CF911F910F9108950F9389
:10ECE0001F93CF93DF93FB01238121FD03C08FEF9F
:10ECF0009FEF28C022FF16C04681578124813581AD
:10ED00004217530744F4A081B1819D012F5F3F4F0B
:10ED1000318320838C93268137812F5F3F4F378348
:10ED2000268310C0EB01092F182F0084F185E02DF8
:10ED30000995892BE1F68E819F8101969F838E83B1
:10ED4000812F902FDF91CF911F910F910895CF9335
:10ED5000DF93CDB7DEB7AE014B5F5F4FFA01619134
:10ED60007191AF018091CC3A9091CD3A0E94846D1F
:10ED7000DF91CF9108950F931F93CF93DF93E0918D
:10ED8000CC3AF091CD3A238121FF1BC08C01D0E019
:10ED9000C0E0F80181918F016091CC3A7091CD3A39
:10EDA000DB011896ED91FC911997882331F00995B4
:10EDB000892B79F3DFEFCFEFECCF8AE00995892B30
:10EDC00019F08FEF9FEF02C08D2F9C2FDF91CF9115
:10EDD0001F910F9108950F931F93CF93DF93CDB79A
:10EDE000DEB72E970FB6F894DEBF0FBECDBF0D89EC
:10EDF0001E898F89988D26E02C831A83098397FFBB
:10EE000002C080E090E801979E838D83AE01455E4D
:10EE10005F4F698D7A8DCE0101960E94846D4D8180
:10EE20005E8157FD0AC02F813885421753070CF4C5
:10EE30009A01F801E20FF31F10822E960FB6F89494
:10EE4000DEBF0FBECDBFDF91CF911F910F9108950F
:10EE5000FA01AA27283051F1203181F1E8946F930B
:10EE60006E7F6E5F7F4F8F4F9F4FAF4FB1E03ED0B1
:10EE7000B4E03CD0670F781F891F9A1FA11D680F4F
:10EE8000791F8A1F911DA11D6A0F711D811D911D82
:10EE9000A11D20D009F468943F912AE0269F1124F7
:10EEA0003019305D3193DEF6CF010895462F47705B
:10EEB000405D4193B3E00FD0C9F7F6CF462F4F70B6
:10EEC000405D4A3318F0495D31FD4052419302D014
:10EED000A9F7EACFB4E0A6959795879577956795BA
:10EEE000BA95C9F700976105710508959B01AC01BA
:10EEF0000A2E06945795479537952795BA95C9F7E1
:10EF0000620F731F841F951FA01D08956F927F923B
:10EF10008F929F92AF92BF92CF92DF92EF92FF9229
:10EF20000F931F93CF93DF93EC017B016115710564
:10EF300019F0DB018D939C938E010F5F1F4F78803A
:10EF4000872D90E00E94F578892B11F0E801F4CF2D
:10EF5000BDE27B1205C00F5F1F4F7980C1E008C082
:10EF6000EBE27E1204C08E010E5F1F4F7980C0E07D
:10EF70006801F1E0CF1AD10843E050E066EC71E09F
:10EF8000C6010E94FE78892BF1F4680122E0C20ECE
:10EF9000D11C45E050E061EC71E0C6010E94FE78B2
:10EFA000892B21F4680187E0C80ED11CE114F1041B
:10EFB00019F0D701CD92DC92C111FFC060E070E082
:10EFC00080E89FE703C143E050E06EEB71E0C601CB
:10EFD0000E94FE78892B51F4E114F10409F4F2C087
:10EFE0000E5F1F4FF70111830083ECC0680160E0E2
:10EFF00070E0CB0100E010E0F601D0EDD70DDA3083
:10F0000058F52C2F2260622E2C2F2870C2FF05C0CD
:10F01000211128C00F5F1F4F25C0222311F001507E
:10F020001109A5E0B0E09B01AC010E9441734B01C6
:10F030005C01880C991CAA1CBB1CC501B4016D0F96
:10F04000711D811D911D6839A9E97A078A07A9E117
:10F050009A0740F0C66005C0DE3F51F4C3FD44C0CE
:10F06000C8606C2EBFEFCB1ADB0A7080C62DC4CFF0
:10F070002D2F2F7D2531C1F540814D3211F4C06116
:10F0800006C04B3221F0319621E030E006C03296C6
:10F09000D60111964C9122E030E0A0EDA40FAA30E9
:10F0A00018F0E21BF30B20C040E050E04038BCE019
:10F0B0005B075CF49A01220F331F220F331F420FAC
:10F0C000531F440F551F4A0F511D3196DF011197F1
:10F0D0002C91A0EDA20FAA3048F3C4FF03C05195B4
:10F0E00041955109040F151FC1FF07C0E114F10438
:10F0F00021F03197D701ED93FC930E943772C370D2
:10F10000C33019F06B017C0106C06B017C01F7FA7A
:10F11000F094F7F8F09420E030E0A901C701B601BF
:10F120000E941679882309F445C017FF06C011957F
:10F1300001951109CDEDD1E002C0C5EFD1E05E012E
:10F14000B8E1AB1AB1084601BE2DAF2D90E2E92E11
:10F15000F12C0E151F0584F0FE0125913591459186
:10F160005491B4018B2F9A2F0E94C5724B01B82F76
:10F17000A92F0E191F09EDCF2497F594E794CA150E
:10F18000DB0539F76401EB2EFA2E8E2D880F8F2DBB
:10F19000881F8F3F49F020E030E0A901C701B60188
:10F1A0000E941679811106C082E290E09093D73ACE
:10F1B0008093D63AC701B60109C060E070E080E8EC
:10F1C0009FEF04C060E070E080EC9FE7DF91CF919B
:10F1D0001F910F91FF90EF90DF90CF90BF90AF9075
:10F1E0009F908F907F906F90089591110C943F792C
:10F1F000803219F089508550C8F70895FB01DC0171
:10F200004150504088F08D9181341CF08B350CF4C6
:10F21000805E659161341CF06B350CF4605E861B7A
:10F22000611171F3990B0895881BFCCF0E941B7923
:10F2300008F481E00895990F0008550FAA0BE0E843
:10F24000FEEF16161706E807F907C0F012161306A8
:10F25000E407F50798F0621B730B840B950B39F4E8
:10F260000A2661F0232B242B252B21F408950A264E
:10F2700009F4A140A6958FEF811D811D089599275E
:10F28000882708950E943273B7FF0895821B930B5D
:10F290000895B7FF0C9441730E944173821B930B36
:10F2A0000895DB018F939F930E944173BF91AF91AB
:10F2B000A29F800D911DA39F900DB29F900D1124D0
:10F2C0000895052E97FB1EF400940E94787957FD4F
:10F2D00007D00E94807307FC03D04EF40C94787919
:10F2E00050954095309521953F4F4F4F5F4F089572
:10F2F00090958095709561957F4F8F4F9F4F0895A2
:04F30000F894FFCFAF
:10F30400FF0101FE01000000808183848687898AD1
:10F314008C8E8F9192949597989A9B9D9EA0A2A370
:10F32400A5A6A7A9AAACADAFB0B2B3B5B6B7B9BAE2
:10F33400BCBDBEC0C1C2C4C5C6C8C9CACBCDCECF70
:10F34400D0D2D3D4D5D6D7D9DADBDCDDDEDFE0E129
:10F35400E2E3E4E5E6E7E8E9EAEAEBECEDEEEEEF1A
:10F36400F0F1F1F2F3F3F4F5F5F6F6F7F8F8F9F94C
:10F37400FAFAFAFBFBFCFCFCFDFDFDFDFEFEFEFEC5
:10F38400FEFFFFFFFFFFFFFF2B2E2C3B3D5B5D2F9E
:10F394005C222A3A3C3E3F7C7F00809A90418E4119
:10F3A4008F804545454949498E8F9092924F994F98
:10F3B400555559999A9B9C9D9E9F41494F55A5A58A
:10F3C400A6A7A8A9AAABACADAEAFB0B1B2B3B4B561
:10F3D400B6B7B8B9BABBBCBDBEBFC0C1C2C3C4C551
:10F3E400C6C7C8C9CACBCCCDCECFD0D1D2D3D4D541
:10F3F400D6D7D8D9DADBDCDDDEDFE0E1E2E3E4E531
:10F40400E6E7E8E9EAEBECEDEEEFF0F1F2F3F4F520
:10F41400F6F7F8F9FAFBFCFDFEFF01030507090EF8
:10F4240010121416181C1E7D1D0100632C001E965C
:10F4340001A01E5A01001F0806101F0606201F08FF
:10F4440006301F0806401F0606511F0700591F52A9
:10F454001F5B1F541F5D1F561F5F1F601F08067030
:10F464001F0E00BA1FBB1FC81FC91FCA1FCB1FDA3C
:10F474001FDB1FF81FF91FEA1FEB1FFA1FFB1F807A
:10F484001F0806901F0806A01F0806B01F0400B836
:10F494001FB91FB21FBC1FCC1F0100C31FD01F0206
:10F4A40006E01F0206E51F0100EC1FF31F0100FC2C
:10F4B4001F4E21010032217021100284210100839A
:10F4C40021D0241A05302C2F04602C0201672C064D
:10F4D40001752C0201802C6401002D260841FF1ABD
:10F4E40003000061001A03E0001703F8000703FF9C
:10F4F40000010078010001300132010601390110D8
:10F50400014A012E017901060180014D0043028167
:10F5140001820182018401840186018701870189B6
:10F52400018A018B018B018D018E018F0190019164
:10F5340001910193019401F60196019701980198B4
:10F54400013D029B019C019D0120029F01A001A09D
:10F5540001A201A201A401A401A601A701A701A976
:10F5640001AA01AB01AC01AC01AE01AF01AF01B125
:10F5740001B201B301B301B501B501B701B801B8D6
:10F5840001BA01BB01BC01BC01BE01F701C001C14C
:10F5940001C201C301C401C501C401C701C801C737
:10F5A40001CA01CB01CA01CD011001DD0101008EA8
:10F5B40001DE011201F3010300F101F401F401F889
:10F5C400012801220212013A020900652C3B023B88
:10F5D400023D02662C3F0240024102410246020AF9
:10F5E400015302400081018601550289018A0158B4
:10F5F400028F015A0290015C025D025E025F029377
:10F604000161026202940164026502660267029764
:10F614000196016A02622C6C026D026E029C0170FA
:10F624000271029D01730274029F017602770278CF
:10F634000279027A027B027C02642C7E027F02A69B
:10F644000181028202A9018402850286028702AE38
:10F65400014402B101B20145028D028E028F029073
:10F66400029102B7017B030300FD03FE03FF03AC19
:10F674000304008603880389038A03B1031103C2C8
:10F68400030200A303A303C4030803CC0303008CF5
:10F69400038E038F03D8031801F2030A00F903F35E
:10F6A40003F403F503F603F703F703F903FA03FA84
:10F6B400033004200350041007600422018A043636
:10F6C40001C1040E01CF040100C004D0044401614F
:10F6D4000526040000C700FC00E900E200E400E0A5
:10F6E40000E500E700EA00EB00E800EF00EE00ECC4
:10F6F40000C400C500C500E600C600F400F600F230
:10F7040000FB00F900FF00D600DC00F800A300D8DD
:10F7140000A7209201E100ED00F300FA00F100D10E
:10F7240000AA00BA00BF001023AC00BD00BC00A1B9
:10F7340000AB00A400912592259325022524256180
:10F74400256225562555256325512557255D255CBC
:10F754002558251025142534252C251C2500253C49
:10F76400255E255F255A2554256925662560255083
:10F77400256C256725682564256525592558255256
:10F784002553256B256A2518250C25882584258C69
:10F794002590258025B103DF009303C003A303C391
:10F7A40003B500C403A6039803A903B4031E22C629
:10F7B40003B50329226122B100652264222023219A
:10F7C40023F7004822B0001922B7001A227F20B282
:10F7D40000A025A00001020408102040801B363A36
:10F7E4005C675C8E5CA95C53797374656D2073747B
:10F7F40061727420686173206265656E2068616C53
:10F804007465640D00EB76904558464154202020E1
:10F814000046415400464154333200222A3A3C3EC9
:10F824003F7C7F002B2C3B3D5B5D0041542B4641CC
:10F8340043544F525952455345540D0041542B479C
:10F8440041504445564E414D453D4F70656E4D6F98
:10F8540064656D0D0041542B4D4F44455357495435
:10F864004348454E3D626C652C300D0041542B4D90
:10F874004F4445535749544348454E3D6C6F63616B
:10F884006C2C300D0041542B48574D4F44454C458A
:10F89400443D300D0041542B424C45504F57455286
:10F8A4004C4556454C3D340D0041545A0D002573CA
:10F8B4000A0D0024475047474100244750524D4306
:10F8C400004F70656E4D6F64656D2F656E74726F59
:10F8D40070792E696E646578004F70656E4D6F6443
:10F8E400656D2F656E74726F70792E736F757263A8
:10F8F40065004F70656E4D6F64656D2F6165733182
:10F9040032382E64697361626C65004F70656E4DA8
:10F914006F64656D2F6165733132382E6B657900C4
:10F924004F70656E4D6F64656D2F4C6F672F7061FE
:10F93400636B65742E696E646578004F70656E4DF7
:10F944006F64656D004F70656E4D6F64656D2F4C0F
:10F954006F670025732F256C752E7063617000002E
:00000001FF
